:020000040800F2
:10000000B0A7002069020008E1BA0008519F00086B
:10001000E5B70008A934000889F2000800000000D4
:1000200000000000000000000000000011C60008F1
:10003000394500080000000051C00008A5D900089B
:10004000830200088302000883020008830200087C
:1000500083020008830200083D450008830200086F
:10006000830200084945000855450008830200083E
:10007000414300085143000883020008830200083E
:10008000830200088302000883020008CD340008C0
:10009000AD340008BD340008830200086145000843
:1000A000830200088302000883020008830200081C
:1000B000830200088302000883020008830200080C
:1000C00083020008830200088302000883020008FC
:1000D00083020008830200088302000883020008EC
:1000E00083020008830200088302000883020008DC
:1000F00083020008830200088302000883020008CC
:1001000083020008830200088302000883020008BB
:1001100083020008830200088302000883020008AB
:10012000830200086143000871430008814300080E
:10013000830200088302000883020008FD340008DF
:10014000DD340008ED340008830200088302000853
:100150008302000891430008830200086DF2000842
:10016000830200088302000883020008830200085B
:1001700083020008830200088302000800000000D8
:10018000830200088302000800F002F800F05CF827
:100190000AA090E8000C82448344AAF10107DA45E2
:1001A00001D100F051F8AFF2090EBAE80F0013F0D8
:1001B000010F18BFFB1A43F0010318474C620100FE
:1001C0006C6201000A444FF0000C10F8013B13F080
:1001D000070408BF10F8014B1D1108BF10F8015BA0
:1001E000641E05D010F8016B641E01F8016BF9D193
:1001F00013F0080F1EBF10F8014BAD1C0C1B09D1EA
:100200006D1E58BF01F801CBFAD505E014F8016B5B
:1002100001F8016B6D1EF9D59142D6D370470000ED
:100220000023002400250026103A28BF78C1FBD8FF
:10023000520728BF30C148BF0B6070471FB515F08B
:1002400006FF1FBD10B510BD00F062F91146FFF7A3
:10025000F5FF0FF0B9FE00F080F903B4FFF7F2FFED
:1002600003BC00F083F900000948804709480047B3
:10027000FEE7FEE7FEE7FEE7FEE7FEE7FEE7FEE756
:10028000FEE7FEE704480549054A064B70470000B3
:1002900079DA000889010008B0870020B0A70020A3
:1002A000B0970020B097002053EA020C00F069805C
:1002B0002DE9F04B4FF00006002B1FBFB3FA83F57A
:1002C00003FA05F424FA05F65E4012BF1643B2FAAB
:1002D00082F502FA05F4C5F120051EBF22FA05FCDD
:1002E00044EA0C04203556EA044C4FEA144418BF83
:1002F000641C4FF000084FF00009904271EB030CB2
:1003000039D3002919BFB1FA81F701FA07F6B0FA1B
:1003100080F700FA07F6C7F120071EBF20FA07FC96
:1003200046EA0C062037B6FBF4FCA7EB0507103FA6
:1003300007F01F0BCBF120062CFA06F60CFA0BFB8C
:1003400044BFB3460026202FA4BF5E464FF0000BEB
:100350005BEA060C08BF4FF0010B19EB0B0948EBE9
:100360000608ABFB027C06FB02CC0BFB03CCC01BDC
:1003700071EB0C01C1E70B46024641464846BDE819
:10038000F08B13B5084318BF4FF0FF300146AFF3B1
:100390000080BDE81C407047032A40F2308010F016
:1003A000030C00F0158011F8013BBCF1020F624410
:1003B00098BF11F801CB00F8013B38BF11F8013BA1
:1003C000A2F1040298BF00F801CB38BF00F8013B4E
:1003D00011F0030300F02580083AC0F0088051F8BE
:1003E000043B083A51F804CBA0E80810F5E7121DC9
:1003F0005CBF51F8043B40F8043BAFF30080D207E8
:1004000024BF11F8013B11F801CB48BF11F8012BB3
:1004100024BF00F8013B00F801CB48BF00F8012BD6
:10042000704710B5203AC0F00B80B1E81850A0E832
:100430001850B1E81850A0E81850203ABFF4F5AFB2
:100440005FEA027C24BFB1E81850A0E8185044BF0E
:1004500018C918C0BDE810405FEA827C24BF51F87B
:10046000043B40F8043B08BF7047D20728BF31F86F
:10047000023B48BF11F8012B28BF20F8023B48BFC0
:1004800000F8012B704702F0FF0343EA032242EA1F
:10049000024200F002B84FF0000200B51346944645
:1004A0009646203922BFA0E80C50A0E80C50B1F1CC
:1004B0002001BFF4F7AF090728BFA0E80C5048BFE0
:1004C0000CC05DF804EB890028BF40F8042B08BF7E
:1004D000704748BF20F8022B11F0804F18BF00F87A
:1004E000012B704770477047704710B500F008F84F
:1004F000006810BD10B5044600F002F8046010BD9D
:1005000000487047700200200048704770020020C9
:100510007546FFF7F9FFAE4605006946534620F0E1
:100520000700854618B020B5FFF7ACFEBDE82040B7
:100530004FF000064FF000074FF000084FF0000B9F
:10054000AC46ACE8C009ACE8C009ACE8C009ACE80E
:10055000C00921F007018D46704710B50446AFF37E
:1005600000802046BDE81040FFF777BE0149182003
:10057000ABBEFEE7260002007047000080B58AB0DF
:1005800008900791089820B9FFE7FF208DF8270011
:100590009BE0079820B9FFE7FF208DF8270094E043
:1005A000079890ED000A90ED013A90ED021A90ED57
:1005B000032A20EE030A21EE021A30EE010A30EE81
:1005C000000A8DED060A079890ED010A90ED021AD7
:1005D00020EE000A21EE011A30EE010A30EE001A78
:1005E000B7EE000A8DED010A30EE410A8DED050AE5
:1005F0009DED060ADDED050A14F00EFA9DED011AD7
:10060000089880ED010A079890ED000A90ED013AF4
:1006100090ED024A90ED032A20EE040A22EE032A0E
:1006200030EE420A30EE000A8DED040A9DED040A18
:10063000B0EEC00AB4EE410AF1EE10FA0ADBFFE7B1
:10064000DDED040A9FED230A0FF006FC089880ED0B
:10065000020A07E09DED040A13F0DAFE089880ED27
:10066000020AFFE7079890ED000A90ED011A90ED5D
:10067000022A90ED033A20EE030A21EE021A30EE30
:10068000010A30EE000A8DED030A079890ED020A88
:1006900090ED031A20EE000A21EE011A30EE010A55
:1006A00030EE001AB7EE000A30EE410A8DED020A74
:1006B0009DED030ADDED020A14F0AEF9089880ED15
:1006C000000A00208DF82700FFE79DF927000AB0F7
:1006D00080BD00BFDB0FC93F80B58CB00A90099187
:1006E0008DED080A0A9820B9FFE7FF208DF82F004A
:1006F00029E19DED081AB7EE000A80EE010A0A987A
:1007000080ED040A0A994FF07E5008600A99002093
:1007100048600A9988600A99C8600998002800F022
:100720000E81FFE7099801680091406815F0C4FB4D
:100730000246009801920A46019942EC101B8DED89
:10074000020B15F0B9FB9DED020B41EC110B14F0FF
:1007500063F88DED040B9DF8170080F080008DF894
:1007600017000498059914F07BFE0790099890ED06
:10077000000AB5EE400AF1EE10FA2BD1FFE7099816
:1007800090ED010AB5EE400AF1EE10FA22D1FFE732
:10079000099890ED020AB5EE400AF1EE10FA19D16F
:1007A000FFE70A9940F2C560C3F64D7008600A99E8
:1007B00044F62D20C3F60D4048600A994AF256408F
:1007C000CBF6393088600A9944F2AD70C3F61970DF
:1007D000C860B3E09DED070A9FED5D1AB4EE410AD3
:1007E000F1EE10FA08DBFFE79DED070AB5EE400ACF
:1007F000F1EE10FA19DDFFE70A9945F66E10C3F61F
:100800007F7008600A9945F20C30C3F6B01048605A
:100810000A9948F6AB00CBF6BB3088600A9949F2DA
:100820008550C3F69750C86087E09DED070A9FED9D
:10083000491AB4EE410AF1EE10FA0ADBFFE79DED2A
:10084000070A9FED431AB4EE410AF1EE10FA19DDE2
:10085000FFE70A9940F2C560C3F64D7008600A9937
:1008600044F62D20C3F60D4048600A994AF25640DE
:10087000CBF6393088600A9944F2AD70C3F619702E
:10088000C86059E09DED070A9FED331AB4EE410AA6
:10089000F1EE10FA0ADBFFE79DED070A9FED2D1A36
:1008A000B4EE410AF1EE10FA19DDFFE70A9940F2C1
:1008B000C560C3F64D7008600A9944F62D20C3F652
:1008C0000D4048600A994AF25640CBF639308860AC
:1008D0000A9944F2AD70C3F61970C8602BE09DED23
:1008E000070A9FED1D1AB4EE410AF1EE10FA08DB7B
:1008F000FFE79DED070AB5EE400AF1EE10FA19DDAB
:10090000FFE70A9940F2C560C3F64D7008600A9986
:1009100044F62D20C3F60D4048600A994AF256402D
:10092000CBF6393088600A9944F2AD70C3F619707D
:10093000C860FFE7FFE7FFE7FFE7FFE7FFE700200B
:100940008DF82F00FFE79DF92F000CB080BD00BF90
:10095000DB0FC93FDB0F49400000B44281B000907B
:100960000099002088604860086001B0704700006E
:1009700080B52DED048BB2B030902F912E922D9337
:10098000309828B9FFE7FF208DF8C70000F0F7BDC9
:100990002F9828B9FFE7FF208DF8C70000F0EFBDC2
:1009A0002E9828B9FFE7FF208DF8C70000F0E7BDBB
:1009B00040F20401C2F200014EF69E70C3F62750C9
:1009C00008602D9848B9FFE730982F992E9A00F0CB
:1009D000DDFD8DF8C70000F0D2BD2D9800680990AC
:1009E0002D98406808902D98806807909DED090A21
:1009F000B5EE400AF1EE10FA19D1FFE79DED080AB5
:100A0000B5EE400AF1EE10FA11D1FFE79DED070AAD
:100A1000B5EE400AF1EE10FA09D1FFE730982F99B0
:100A20002E9A00F0B3FD8DF8C70000F0A8BD2F98F6
:100A3000006806902F98406805902F988068049071
:100A40002E98006803902E98406802902E98806837
:100A5000019030989DED033A90ED010A90ED022A45
:100A600090ED031A20EE430A9DED023A22EE032A8E
:100A700030EE420A9DED012A21EE021A30EE410AC3
:100A8000B6EE001A20EE010A8DED270A30989DED92
:100A9000034A90ED000A90ED023A90ED032A20EE11
:100AA000040A9DED014A23EE043A30EE030A9DED5F
:100AB000023A22EE032A30EE420A20EE010A8DEDC0
:100AC000260A30989DED024A90ED000A90ED013A19
:100AD00090ED032A20EE040A9DED014A23EE043A2C
:100AE00030EE430A9DED033A22EE032A30EE020A6D
:100AF00020EE010A8DED250A30989DED014A90ED1A
:100B0000000A90ED013A90ED022A20EE040A9DEDD4
:100B1000024A23EE043A30EE030A9DED033A22EE38
:100B2000032A30EE420A20EE010A8DED240A9DEDE3
:100B3000060AB5EE400AF1EE10FA11D1FFE79DED7D
:100B4000050AB5EE400AF1EE10FA09D1FFE79DED76
:100B5000040AB5EE400AF1EE10FA00F09984FFE7BE
:100B60009DED060A20EE000A9DED051A21EE011A00
:100B700030EE010A9DED041A21EE011A30EE010A51
:100B800009F0E8F98DED2C0A9DED2C1A9DED060A71
:100B900020EE010A8DED060A9DED2C1A9DED050A49
:100BA00020EE010A8DED050A9DED2C1A9DED040A3B
:100BB00020EE010A8DED040A9DED090A20EE000ADF
:100BC0009DED081A21EE011A30EE010A9DED071A7B
:100BD00021EE011A30EE010A09F0BCF98DED2C0A64
:100BE0009DED2C1A9DED090A20EE010A8DED090AF2
:100BF0009DED2C1A9DED080A20EE010A8DED080AE4
:100C00009DED2C1A9DED070A20EE010A8DED070AD5
:100C1000309890ED000A30EE000A9DED091A20EEA2
:100C2000010A8DED210A309890ED000A30EE000A9D
:100C30009DED081A20EE010A8DED200A309890ED06
:100C4000000A30EE000A9DED071A20EE010A8DED34
:100C50001F0A309890ED010A30EE000A9DED091A46
:100C600020EE010A8DED1E0A309890ED000A30EE5C
:100C7000000A8DED190A309890ED010A30EE000A55
:100C80008DED180A309890ED020A30EE000A8DEDD5
:100C9000170A309890ED030A30EE000A8DED160A1F
:100CA000309890ED000A90ED021A30EE000A20EE26
:100CB000010A8DED150A309890ED020A90ED031AA5
:100CC00030EE000A20EE010A8DED140A309890ED06
:100CD000000A20EE000A8DED130A309890ED000A0C
:100CE00090ED011A20EE010A8DED120A309890ED78
:100CF000000A90ED021A20EE010A8DED110A3098DB
:100D000090ED000A90ED031A20EE010A8DED100A15
:100D1000309890ED010A20EE000A8DED0F0A309810
:100D200090ED010A90ED021A20EE010A8DED0E0AF7
:100D3000309890ED010A90ED031A20EE010A8DED36
:100D40000D0A309890ED020A20EE000A8DED0C0A93
:100D5000309890ED020A90ED031A20EE010A8DED15
:100D60000B0A309890ED030A20EE000A8DED0A0A76
:100D70009DED091A9DED130A21EE000A9DED202A32
:100D8000309890ED025A90ED033A22EE032A30EEAD
:100D9000420A9DED1F2A22EE052A30EE020A9DED41
:100DA0000F2A21EE022A30EE020A9DED182A9DED4F
:100DB000084A22EE044A24EE054A30EE040A9DED6C
:100DC000074A22EE042A22EE032A30EE020A9DEDA3
:100DD0000C2A21EE022A30EE420A9DED0A2A21EE6B
:100DE000021A30EE410A8DED230A9DED210A30985A
:100DF00090ED015A90ED024A90ED033A20EE030A7D
:100E00009DED081A9DED132A21EE022A30EE020A0A
:100E10009DED1F2A22EE052A30EE420A9DED1E2A84
:100E200022EE042A30EE020A9DED0F2A21EE022A5C
:100E300030EE420A9DED0C2A21EE022A30EE020A23
:100E40009DED172A9DED074A22EE042A22EE032A81
:100E500030EE020A9DED0A2A21EE021A30EE410A16
:100E60008DED220A9DED230A20EE000A9DED221A47
:100E700021EE011A30EE010A09F06CF8B7EE006AB3
:100E800086EE000A8DED1D0A9DED210A309890ED49
:100E9000012A90ED021A90ED033A20EE011A9DED21
:100EA000200A20EE020A30EE412A9DED071A9DED40
:100EB000130A21EE000A30EE022A9DED1E0A20EEF2
:100EC000030A30EE020A9DED0F2A21EE022A30EECF
:100ED000420A9DED172A9DED084A22EE042A22EED1
:100EE000032A30EE020A9DED0C2A21EE022A30EE92
:100EF000420A9DED0A2A21EE021A30EE010A8DED1A
:100F00001C0A9DED1D0A30EE000A8DED1B0A9DEDB9
:100F10001C0A30EE000A8DED1A0A9DED170ADDED70
:100F20000D0A30EEA02A9DED151A31EE422A9DEDF4
:100F3000061A31EE021A20EE010A9DED181ADDEDB7
:100F4000123A33EEA32A9DED143A32EE032A9DEDB8
:100F5000053A32EE432A21EE021A70EE014A9DED67
:100F60001C3A309890ED011A90ED020AD0ED032A58
:100F700063EE001A9DED1D2A9DED0C7AB6EE004A37
:100F80008DED004A77EE445A9DED0A5A35EE255A0A
:100F900062EE055A9DED115A75EE606A63EE266A9F
:100FA00075EEA66ADDED095A75EEA65A61EEA51A30
:100FB00071EEA41A62EE222A23EE011A31EE621AB1
:100FC000DDED0E2ADDED104A72EEE42A62EE222AF1
:100FD000DDED0B4A73EEA43A63EE233A72EEA32AD8
:100FE000DDED083A72EEE32A21EE221A31EE211AE3
:100FF00022EE000A35EE205A22EE052A9DED0F5A08
:1010000034EE455A35EE475A23EE053A32EE032ABE
:101010009DED073A32EE432A20EE020A30EE010A35
:101020008DED2B0A9DED160ADDED0D2A32EEA21A8A
:101030009DED152A31EE421A9DED062A31EE421A37
:1010400020EE010A9DED191ADDED126A36EEA62A90
:101050009DED143A32EE032A9DED053A32EE432A15
:1010600021EE021A30EE011A3098D0ED005AD0ED80
:10107000014AD0ED023A90ED032AB1EE000A24EEC7
:10108000803A9DED0F7A37EE075A75EE461ADDED80
:101090000C0A30EEA05A75EE211A9DED045A35EE79
:1010A000215A23EE053A31EE031A9DED1C5A65EEE6
:1010B000027A9DED1D3A74EE601A9DED0A8A71EE7A
:1010C000C81A23EE218ADDED111A32EEE19A25EEDF
:1010D000099A38EE098A9DED099A38EE498A67EE39
:1010E000887A31EE271A63EE233A65EE255A73EEBD
:1010F000A53ADDED0E5ADDED107A75EEE75A63EE96
:10110000255ADDED0B7A76EEA76A65EE266A75EE56
:10111000A65ADDED086A75EEE65A63EEA53A31EEA1
:10112000231A23EE022ADDED1A3A63EEA43A32EED8
:10113000632A71EEA21A23EE213A34EE477A37EE93
:10114000607A25EE075A33EE053A9DED075A33EEE5
:10115000453A22EE032A31EE021A8DED2A1A9DED50
:10116000191ADDED0D0A30EEA03A9DED152A32EE8A
:10117000433A9DED062A32EE032A21EE021A9DED36
:10118000162ADDED124A34EEA43A9DED145A33EEE0
:10119000053A9DED055A33EE453A22EE032A31EE2B
:1011A000022A309890ED001AD0ED011AD0ED022AF3
:1011B000D0ED033A22EE800A9DED0F5A35EE053A46
:1011C00033EE467A9DED0C6A36EE063A33EE077A38
:1011D0009DED043A33EE073A20EE030A70EE025A10
:1011E0009DED1B0A20EE620A9DED1C3A23EE012ABA
:1011F00030EE420A9DED1D2A34EE467ADDED0A6A94
:1012000037EE667A62EE076A9DED117A70EEC77A64
:1012100063EE277A76EEA76ADDED097A76EEE76A65
:1012200020EE260A30EE250A62EE211A63EE233AFA
:1012300071EEA31ADDED0E3ADDED105A73EEE53ACC
:1012400062EE233ADDED0B5A74EEA54A63EE244AB2
:1012500073EEA43ADDED084A73EEE43A61EEA31AA8
:1012600030EE210A22EE011ADDED1A1A61EEA21A01
:1012700031EE611A37EE207A22EE072A34EE455A13
:1012800035EE465A23EE053A32EE032A9DED073A33
:1012900032EE432A21EE021A30EE010A8DED290AC0
:1012A0009DED180A9DED0D7A37EE071A9DED152A72
:1012B00031EE421A9DED062A31EE421A20EE010A65
:1012C0009DED171ADDED122A32EEA22A9DED143A99
:1012D00032EE032A9DED053A32EE432A21EE021A40
:1012E00070EE013A9DED1B1A3098D0ED001A90ED8A
:1012F000010AD0ED020A90ED032A21EE022A9DEDAB
:101300001C3A23EE001A31EE421A9DED1D2A9DED86
:101310000C5A34EE456ADDED0A4A36EE646A62EE36
:10132000064A9DED116A77EE465A63EE255A74EE31
:10133000A54ADDED095A74EEE54A21EE241A31EE94
:10134000231A62EE211A63EE200A70EEE10ADDED47
:101350000E1ADDED103A71EEE31A62EE211ADDEDA0
:101360000B3A72EEA32A63EE222A71EEA21ADDED89
:10137000082A71EEE21A60EEA10A31EE201A22EE7E
:10138000000A36EE076A22EE062A9DED0F6A34EE59
:10139000464A34EE454A23EE043A32EE032A9DEDE6
:1013A000073A32EE432A20EE020A30EE010A8DEDB2
:1013B000280A9DED2B0A20EE000A9DED2A1A21EE47
:1013C000011A30EE010A9DED291A21EE011A30EEC4
:1013D000010A9DED281A21EE011A30EE010A08F0EB
:1013E000B9FD8DED2C0A9DED2C1A9DED2B0A20EEFA
:1013F000010A8DED2B0A9DED2C1A9DED2A0A20EE97
:10140000010A8DED2A0A9DED2C1A9DED290A20EE88
:10141000010A8DED290A9DED2C1A9DED280A20EE7A
:10142000010A8DED280A40F20400C2F2000090ED9E
:10143000000A9DED2B1A20EE011A9DED270A30EED1
:10144000410A8DED270A90ED000A9DED2A1A20EE43
:10145000011A9DED260A30EE410A8DED260A90ED27
:10146000000A9DED291A20EE011A9DED250A30EEA5
:10147000410A8DED250A90ED000A9DED281A20EE17
:10148000011A9DED240A30EE410A8DED240AFFE792
:101490009DED271A309890ED000A90ED042A21EE78
:1014A000021A30EE010A80ED000A9DED261A3098EE
:1014B00090ED010A90ED042A21EE021A30EE010AA5
:1014C00080ED010A9DED251A309890ED020A90ED0D
:1014D000042A21EE021A30EE010A80ED020A9DED87
:1014E000241A309890ED030A90ED042A21EE021A96
:1014F00030EE010A80ED030A309890ED000A90ED7D
:10150000013A90ED022A90ED031A20EE000A23EE34
:10151000033A30EE030A22EE022A30EE020A21EEEE
:10152000011A30EE010A08F015FD8DED2C0A9DED33
:101530002C1A309890ED000A20EE010A80ED000A86
:101540009DED2C1A309890ED010A20EE010A80EDF5
:10155000010A9DED2C1A309890ED020A20EE010A46
:1015600080ED020A9DED2C1A309890ED030A20EED2
:10157000010A80ED030A00208DF8C700FFE79DF9FE
:10158000C70032B0BDEC048B80BD000080B5A0B0B8
:101590001E901D911C921E9820B9FFE7FF208DF828
:1015A0007F00D3E21D9820B9FFE7FF208DF87F0070
:1015B000CCE21C9820B9FFE7FF208DF87F00C5E240
:1015C00040F20401C2F2000142F60230C3F60750B5
:1015D00008601D9800681B901D9840681A901D981F
:1015E000806819901C98006818901C9840681790A3
:1015F0001C98806816901E989DED183A90ED010A8F
:1016000090ED022A90ED031A20EE430A9DED173A61
:1016100022EE032A30EE420A9DED162A21EE021A2E
:1016200030EE410AB6EE001A20EE010A8DED100AE6
:101630001E989DED184A90ED000A90ED023A90ED4B
:10164000032A20EE040A9DED164A23EE043A30EEFA
:10165000030A9DED173A22EE032A30EE420A20EEED
:10166000010A8DED0F0A1E989DED174A90ED000AB4
:1016700090ED013A90ED032A20EE040A9DED164A02
:1016800023EE043A30EE430A9DED183A22EE032A87
:1016900030EE020A20EE010A8DED0E0A1E989DED35
:1016A000164A90ED000A90ED013A90ED022A20EEE4
:1016B000040A9DED174A23EE043A30EE030A9DED2D
:1016C000183A22EE032A30EE420A20EE010A8DED8E
:1016D0000D0A9DED1B0AB5EE400AF1EE10FA11D18C
:1016E000FFE79DED1A0AB5EE400AF1EE10FA09D1B6
:1016F000FFE79DED190AB5EE400AF1EE10FA00F091
:10170000AE81FFE79DED1B0A20EE000A9DED1A1A3F
:1017100021EE011A30EE010A9DED191A21EE011A8F
:1017200030EE010A08F016FC8DED150A9DED151A34
:101730009DED1B0A20EE010A8DED1B0A9DED151A89
:101740009DED1A0A20EE010A8DED1A0A9DED151A7B
:101750009DED190A20EE010A8DED190A1E9890EDF3
:10176000000A30EE000A8DED0C0A1E9890ED010A79
:1017700030EE000A8DED0B0A1E9890ED020A30EE55
:10178000000A8DED0A0A1E9890ED030A30EE000A59
:101790008DED090A1E9890ED000AB1EE003A20EE98
:1017A000030A8DED080A1E9890ED010A20EE030A47
:1017B0008DED070A1E9890ED020A20EE030A8DEDCA
:1017C000060A1E9890ED010AB2EE001A20EE010AF8
:1017D0008DED050A1E9890ED020A20EE010A8DEDAE
:1017E000040A1E9890ED000A20EE000A8DED030A0F
:1017F0001E9890ED010A20EE000A8DED020A1E9857
:1018000090ED020A20EE000A8DED010A1E9890ED7F
:10181000030A20EE000A8DED000A9DED081A9DEDE9
:10182000010A21EE000A9DED0A2A9DED1B4A22EED7
:10183000042A30EE020A9DED022A21EE021A30EE51
:10184000010A9DED0B1A9DED1A2A21EE021A30EEC7
:10185000410A8DED140A9DED071A9DED000A21EE57
:10186000000A9DED092A9DED1B4A22EE042A30EE66
:10187000420A9DED032A22EE032A1E9890ED014AAA
:1018800022EE042A30EE020A9DED0C2A9DED1A4A42
:1018900022EE042A30EE420A30EE410A9DED052A7E
:1018A0009DED024A22EE044A30EE040A9DED014A03
:1018B00022EE042A30EE020A9DED192A21EE021AC8
:1018C00030EE010A8DED130A9DED030A20EE030AA6
:1018D0001E9890ED021A20EE010A9DED0C1A9DED66
:1018E0001B2A21EE021A30EE010A9DED061A9DED2B
:1018F000002A21EE022A30EE020A9DED092A9DED12
:101900001A4A22EE042A30EE420A30EE410A9DEDD8
:10191000042A9DED024A22EE044A30EE040A9DEDAF
:10192000014A22EE042A30EE020A9DED192A21EE28
:10193000021A30EE010A8DED120A9DED020A20EE28
:10194000030A1E9890ED032A20EE020A9DED0B1A61
:101950009DED1B4A21EE041A30EE410A9DED011A5D
:1019600021EE031A21EE021A30EE010A9DED0A1A49
:101970009DED1A2A21EE021A30EE410A8DED110A70
:101980009DED140A20EE000A9DED131A21EE011AB6
:1019900030EE010A9DED121A21EE011A30EE010A15
:1019A0009DED111A21EE011A30EE010A08F0D2FA6B
:1019B0008DED150A9DED151A9DED140A20EE010A14
:1019C0008DED140A9DED151A9DED130A20EE010A06
:1019D0008DED130A9DED151A9DED120A20EE010AF8
:1019E0008DED120A9DED151A9DED110A20EE010AEA
:1019F0008DED110A40F20400C2F2000090ED000AE1
:101A00009DED141A20EE011A9DED100A30EE410AE8
:101A10008DED100A90ED000A9DED131A20EE011ACB
:101A20009DED0F0A30EE410A8DED0F0A90ED000A90
:101A30009DED121A20EE011A9DED0E0A30EE410ABC
:101A40008DED0E0A90ED000A9DED111A20EE011A9F
:101A50009DED0D0A30EE410A8DED0D0AFFE79DED7B
:101A6000101A1E9890ED000A90ED042A21EE021A39
:101A700030EE010A80ED000A9DED0F1A1E9890EDE0
:101A8000010A90ED042A21EE021A30EE010A80EDDF
:101A9000010A9DED0E1A1E9890ED020A90ED042A9F
:101AA00021EE021A30EE010A80ED020A9DED0D1AB8
:101AB0001E9890ED030A90ED042A21EE021A30EEF2
:101AC000010A80ED030A1E9890ED000A90ED013A9C
:101AD00090ED022A90ED031A20EE000A23EE033A5D
:101AE00030EE030A22EE022A30EE020A21EE011A3B
:101AF00030EE010A08F02EFA8DED150A9DED151A4B
:101B00001E9890ED000A20EE010A80ED000A9DED7E
:101B1000151A1E9890ED010A20EE010A80ED010AC7
:101B20009DED151A1E9890ED020A20EE010A80ED37
:101B3000020A9DED151A1E9890ED030A20EE010A87
:101B400080ED030A00208DF87F00FFE79DF97F00FC
:101B500020B080BD84B08DED030ACDED020A9DED6D
:101B6000030A9DED021AB1EE411AB4EE410AF1EEFC
:101B700010FA07DAFFE79DED020AB1EE400A8DED9B
:101B8000010A18E09DED030A9DED021AB4EE410A28
:101B9000F1EE10FA05DDFFE79DED020A8DED000A7A
:101BA00004E09DED030A8DED000AFFE79DED000ABC
:101BB0008DED010AFFE79DED010A04B070470000BA
:101BC00080B541F2AC70C2F20000006804210EF052
:101BD000E1FD80BD80B582B040F28842C2F20002D1
:101BE000002001901221132300F030FA019802B076
:101BF00080BD000080B501214FF0FF3208460EF095
:101C00001BFE80BD81B000909FED010A01B07047BE
:101C10000000C84380B541F2AC70C2F20000006819
:101C200008210EF0B7FD80BD80B540F28840C2F2B9
:101C30000000C21D01200221062300F007FA002047
:101C400080BD000080B5022001214FF0FF320EF070
:101C5000F3FD80BD80B58AB008900791089820B93F
:101C6000FFE7FE208DF82700B4E0079820B9FFE7D2
:101C7000FE208DF82700ADE040F61A40C2F20000C9
:101C80000078C00720B1FFE7FD208DF82700A1E014
:101C90000EF060FE41F2AC71C2F20001086020B9A2
:101CA000FFE7FE208DF8270094E007980899C862A6
:101CB000002006907E21B622049200F05DFA049A7C
:101CC0000120142100F058FA1E20059001F0C6FAF8
:101CD0000599069800F0F6F90699084600F0F2F921
:101CE0001E2804D0FFE7FC208DF8270072E00120B9
:101CF000002100F0E7F90F2804D0FFE7FC208DF861
:101D0000270067E00320019001F018F804200290FA
:101D100001F014F841F6E972C0F6000200200390C9
:101D20000121009101F038FA019841F6C131C0F665
:101D3000000101F081F8029841F61541C0F600015A
:101D400001F07AF803984021AA2200F015FA009ACF
:101D50000398412100F010FA03985321082200F063
:101D60000BFA029A0398582100F006FA029A039897
:101D70007D2100F001FA322001F070FA009A0F2163
:101D8000104600F0F9F90098019A102100F0F4F9DA
:101D90000098039A162100F0EFF9009A18211046D6
:101DA00000F0EAF900981521802200F0E5F90A20F8
:101DB00001F054FA0099019840F61A42C2F200026A
:101DC000117000F0E7FF029800F0E4FF03988DF82F
:101DD0002700FFE79DF927000AB080BD84B002907C
:101DE000029820B9FFE7FE208DF80F006AE040F26C
:101DF0008841C2F20001B1F80100ADF80600B1F867
:101E00000300ADF80400B1F80500ADF80200BDF91B
:101E1000060000EE100AB8EEC00A029880ED040A2F
:101E2000BDF9040000EE100AB8EEC00A029880ED79
:101E3000050ABDF9020000EE100AB8EEC00A0298C9
:101E400080ED060A029890ED040A9FED201A80EEBC
:101E5000010A80ED040A029890ED050A80EE010A5D
:101E600080ED050A029890ED060A80EE010A80EDE9
:101E7000060A487C897CC00040EA5110ADF8000099
:101E8000BDF90000B0F5806F07DBFFE7BDF800008B
:101E9000A0F50060ADF80000FFE7BDF9000000EE1E
:101EA000100AB8EEC00AB4EE001A20EE010AB3EE32
:101EB000071A30EE010A029880ED0A0A00208DF818
:101EC0000F00FFE79DF90F0004B0704700A0AA457E
:101ED00084B00290029820B9FFE7FE208DF80F0031
:101EE0007AE040F28840C2F20000B0F80710ADF886
:101EF0000610B0F80910ADF80410B0F80B00ADF8FA
:101F00000200BDF9060000EE100AB8EEC00A029801
:101F100080ED070ABDF9040000EE100AB8EEC00A11
:101F2000029880ED080ABDF9020000EE100AB8EE32
:101F3000C00A029880ED090A029890ED070A9FED09
:101F4000281A80EE010A80ED070A029890ED080A2F
:101F500080EE010A80ED080A029890ED090A80EEF1
:101F6000010A80ED090A029890ED070A9FED1D1AFB
:101F700020EE010A80ED070A029890ED080A20EE93
:101F8000010A80ED080A029890ED090A20EE010A84
:101F900080ED090A0298C16A91ED001A90ED070AD6
:101FA00030EE410A80ED070A0298C16A91ED011AEC
:101FB00090ED080A30EE410A80ED080A0298C16AE5
:101FC00091ED021A90ED090A30EE410A80ED090AFE
:101FD000FE208DF80F00FFE79DF90F0004B0704759
:101FE0006F12034235FA8E3C80B582B0012000F0BA
:101FF000FDFE70B9FFE701210191084600F064FF82
:10200000019941F2AC70C2F2000000680EF0C2FB10
:10201000FFE7022000F0EAFE70B9FFE7022000901F
:10202000012100F051FF009941F2AC70C2F20000B2
:1020300000680EF0AFFBFFE702B080BD80B50C205A
:1020400001214FF0FF320EF0F7FB80BD80B586B066
:102050008DF817008DF8161004928DF80F30049843
:1020600008B9FFE72BE09DF817000146029120B167
:10207000FFE70298012805D009E00120002100F0C7
:1020800023FF04E00220002100F01EFFFFE79DF87F
:10209000160040F0800040F29B41C2F2000108703F
:1020A0000122009200230193184601F097F8009B4B
:1020B000019804999DF80F2001F02EF8FFE706B073
:1020C00080BD000080B586B08DF816008DF8151023
:1020D000012001F0C3F89DF816000146049120B1DB
:1020E000FFE70498012805D009E00120002100F055
:1020F000EBFE04E00220002100F0E6FEFFE79DF881
:10210000150040F0800040F29B41C2F200010191B5
:102110000870012200230293184601F05FF801992C
:10212000029B0222184600F0F7FF9DF816000146B8
:10213000039120B1FFE7039801280CD017E001219B
:10214000084600F0C1FE40F29B40C2F20000407819
:102150008DF817000BE00220012100F0B5FE40F2DF
:102160009B40C2F2000000788DF81700FFE79DF851
:10217000170006B080BD000080B584B08DF80F0058
:102180008DF80E108DF80D209DF80E0000F07F00E8
:1021900040F29B41C2F2000108709DF80D004870AA
:1021A000012001F05BF89DF80F000146029120B17B
:1021B000FFE70298012805D009E00120002100F086
:1021C00083FE04E00220002100F07EFEFFE740F2E3
:1021D0009B41C2F2000102220023184600F0FEFFDC
:1021E0009DF80F000146019120B1FFE701980128F9
:1021F00005D009E00121084600F066FE04E0022057
:10220000012100F061FEFFE704B080BD80B586B01B
:102210008DF8160004918DF80F209DF80F0020B95D
:10222000FFE70A208DF80F00FFE741F21C50C2F2D1
:102230000000006864210EF089F920B1FFE7FB205F
:102240008DF8170070E041F21850C2F200000068EB
:102250000290FFE70298E0B1FFE7029800789DF84E
:102260001610884211D1FFE702984068049988420D
:102270000BD1FFE741F21C50C2F2000000680EF0E3
:1022800049FAFF208DF817004EE00298006902908D
:10229000E0E7142000F040FE0190019858B9FFE7F4
:1022A00041F21C50C2F2000000680EF033FAFE202A
:1022B0008DF8170038E09DF80F001C2100220EF069
:1022C00043F8019988600198806870B9FFE7019828
:1022D00000F02CFD41F21C50C2F2000000680EF02C
:1022E00019FAFF208DF817001EE09DF816000199DD
:1022F00008700498019948609DF80F0001990873CF
:1023000041F21851C2F200010868019A1061019867
:10231000086041F21C50C2F2000000680EF0FAF9A9
:1023200000208DF81700FFE79DF9170006B080BD6B
:1023300082B001908DF80310019802B07047000040
:1023400084B08DF80B00019141F21850C2F20000E8
:1023500000680090FFE70098A8B1FFE700980078B8
:102360009DF80B1088420AD1FFE700984068019958
:10237000884204D1FFE700988068039006E0009847
:1023800000690090E7E700200390FFE7039804B09E
:102390007047000082B000900098C068022809D100
:1023A000FFE7009881680220042908BF03208DF808
:1023B000070008E0009880680438B0FA80F040090F
:1023C0008DF80700FFE79DF8070002B07047000096
:1023D00083B08DF807009DF80700022803DBFFE7B4
:1023E0000020029018E09DF807000146009120B1FE
:1023F000FFE70098012806D00BE040F23470C2F2EB
:102400000000029008E040F25C70C2F2000002900E
:1024100002E000200290FFE7029803B0704700003E
:1024200080B586B08DF8160004910392029340F6B1
:102430001840C2F200000078C00720B9FFE7FD2075
:102440008DF8170037E0039820B9FFE7FE208DF8DC
:10245000170030E041F21C50C2F200000068642115
:102460000EF074F820B1FFE7FB208DF8170022E092
:102470009DF816000499FFF763FF019041F21C508C
:10248000C2F2000000680EF045F9019820B9FFE79C
:10249000FC208DF817000EE001980399029B0022A2
:1024A0000DF0F2FE00900098002818BF4FF0FF30AA
:1024B0008DF81700FFE79DF9170006B080BD0000FA
:1024C00080B596B040F61840C2F200000078C00710
:1024D00020B1FFE7FD208DF85700A7E040F2D020A3
:1024E000C2F200006821FDF7D6FF00201490FFE73C
:1024F0001498012809DCFFE79DF8500000F01CFB50
:10250000FFE7149801301490F2E740F6D831C2F298
:10251000000142F23130C0F60000086000200EF0E9
:1025200065F8014641F21C50C2F2000001600068EB
:1025300020B9FFE7FF208DF8570077E040F61841FB
:10254000C2F2000107910120089008700AA80390C8
:102550002821FDF7A0FF0399089A002009900F9009
:102560000A900B90109011920C900D9012920E22E6
:10257000029213920E9040F23470C2F20000019069
:1025800002F04EFC019803F049FB099842F24172B7
:10259000C0F60002062100F06FF8099942F6C12248
:1025A000C0F600020592084600F066F8059A089900
:1025B000099800F061F8059A09980221049100F049
:1025C0005BF80198032102F055FB029A03990898E1
:1025D0000F920E9040F25C70C2F20000069002F082
:1025E0001FFC069803F01AFB089842F62502C0F675
:1025F0000002082100F040F8059A0999089800F0B7
:102600003BF8059A0899084600F036F80499059AAF
:10261000089800F031F80698112102F02BFB079A78
:102620000899099811708DF85700FFE79DF9570038
:1026300016B080BD80B584B002908DF8071040F6CA
:10264000D830C2F20000006858B1FFE740F6D83039
:10265000C2F20000026802989DF8071090470390AC
:1026600006E002989DF80710FFF762FE0390FFE76F
:10267000039804B080BD000082B08DF806008DF88C
:102680000510009240F61840C2F200000078C00722
:1026900020B9FFE7FD208DF807002AE0009820B957
:1026A000FFE7FE208DF8070023E09DF806000228D2
:1026B00004DBFFE7FF208DF807001AE09DF8050016
:1026C0000D2804DBFFE7FF208DF8070011E00098DC
:1026D0009DF8061040F2D023C2F20003342211FB11
:1026E00002319DF8052041F8220000208DF80700F6
:1026F000FFE79DF9070002B07047000080B584B085
:102700008DF80E0002918DF8072040F61840C2F2B5
:1027100000000078C00720B9FFE7FD208DF80F000A
:1027200009E09DF80E0002999DF80720FFF76EFD65
:102730008DF80F00FFE79DF90F0004B080BD000089
:1027400080B598B000200E90FFE70E98012867DC56
:10275000FFE79DF83800FFF73BFE0D900D9808B994
:10276000FFE759E0FFE70D98002102F051FC002837
:1027700051D0FFE70D98002111AA0FAB02F072FCB7
:10278000002847D1FFE7139818B9FFE71198019087
:1027900002E012980190FFE701980C9011A8FFF752
:1027A000F9FD8DF82F000C989DF82F10FFF742FFD0
:1027B0000A909DF838000A99FFF7C2FD0990099820
:1027C00038B3FFE70020089007900690059004902A
:1027D000039002909DF82F008DF808000C9803904C
:1027E0000A98049015988DF81400149838B9FFE7EA
:1027F00002A80D30159A0FA9FDF7CEFDFFE704F0F2
:1028000029F90890099802A900231A460DF01CFE28
:10281000FFE7FFE7A7E7FFE70E9801300E9094E788
:1028200018B080BD80B598B000200E90FFE70E98DC
:10283000012867DCFFE79DF83800FFF7C9FD0D9020
:102840000D9808B9FFE759E0FFE70D98012102F064
:10285000DFFB002851D0FFE70D98012111AA0FAB33
:1028600002F000FC002847D1FFE7139818B9FFE7F2
:102870001198019002E012980190FFE701980C90E6
:1028800011A8FFF787FD8DF82F000C989DF82F10E9
:10289000FFF7D0FE0A909DF838000A99FFF750FD27
:1028A0000990099838B3FFE7002008900790069038
:1028B00005900490039002909DF82F008DF8080079
:1028C0000C9803900A98049015988DF814001498A9
:1028D00038B9FFE702A80D30159A0FA9FDF75CFD86
:1028E000FFE704F0B7F80890099802A900231A46F8
:1028F0000DF0AAFDFFE7FFE7A7E7FFE70E9801301D
:102900000E9094E718B080BD80B592B084461498BC
:102910008DF846C08DF8451010920F938DF83B004E
:1029200040F61840C2F200000078C00720B9FFE767
:10293000FD208DF847009EE09DF84600022804DB4C
:10294000FFE7FF208DF8470095E00F9870B9FFE78B
:102950009DF84500022809D0FFE79DF845000328AF
:1029600004D0FFE7FE208DF8470084E09DF83B008F
:10297000092804DBFFE7FF208DF847007BE09DF886
:102980004600FFF725FD0D900D9820B9FFE7FE20CA
:102990008DF847006FE0002001900C900B900A909A
:1029A000099008900790069005909DF84500014613
:1029B000029103281FD80299DFE801F002080F16E0
:1029C0001098059000200790089018E01098069045
:1029D000042007900020089011E010980590002036
:1029E0000790022008900AE01098069004200790B3
:1029F0000220089003E0FF208DF847003BE09DF89F
:102A00003B00099000208DF828000F9868B1FFE77F
:102A10009DF83B00012808DBFFE705A818300F9957
:102A20009DF83B20FDF7B8FCFFE70D9802F024FC71
:102A300090B1FFE70D9805A901F1180204AB02F06F
:102A400043F98DF80F009DF80F0020B9FFE7002033
:102A50008DF847000FE0FFE79DF8460005A900F05C
:102A60000FF920B1FFE700208DF8470003E0FF20B9
:102A70008DF84700FFE79DF9470012B080BD0000C8
:102A800080B584B08DF80E000291029820B9FFE75E
:102A9000FE208DF80F000EE09DF80E0002990A68E6
:102AA0004B1D0979EC46CCF800100021FFF72CFFF4
:102AB0008DF80F00FFE79DF90F0004B080BD000006
:102AC00080B58CB000200B90FFE70B98012831DC1B
:102AD000FFE70B988DF82B009DF82B00FFF778FC93
:102AE0000990099808B9FFE720E0FFE79DF82B005F
:102AF00000F044F8C8B9FFE7099802F0BDFB08B937
:102B0000FFE712E09DF82B0001A900F063F808B977
:102B1000FFE70AE0099801A901F118026B4602F0EB
:102B2000D3F808B1FFE700E0E0E7FFE70B980130DA
:102B30000B90CAE70CB080BD81B08DF803009DF802
:102B40000300022801DBFFE715E09DF8030000EB1E
:102B5000C01041F2B071C2F2000101EBC0020020CE
:102B6000C2F800049DF8032002EBC21201EBC2017F
:102B7000C1F80404FFE701B07047000081B08DF890
:102B800002009DF80200022804DBFFE701208DF817
:102B900003001AE09DF8020000EBC01041F2B07192
:102BA000C2F2000101EBC000D0F800049DF8022041
:102BB00002EBC21201EBC201D1F80414401AB0FAC0
:102BC00080F040098DF80300FFE79DF8030001B095
:102BD00070470000B0B584B08DF80E0002919DF8EA
:102BE0000E00012803DCFFE7029820B9FFE7002070
:102BF0008DF80F0040E09DF80E0000EBC01141F28F
:102C0000B070C2F2000000EBC10001900198D0F852
:102C100000040199D1F80414884204D1FFE7002090
:102C20008DF80F0028E0029900910198D0F8043443
:102C300000EB43125B01C0585368D2F808C0D2F8C9
:102C40000CE0146955694D610C61C1F80CE0C1F8E4
:102C500008C04B6008609069D269CA6188610198B8
:102C6000D0F80404013000F01F000199C1F80404F9
:102C700001208DF80F00FFE79DF80F0004B0B0BDF4
:102C8000F0B585B08DF8120003919DF8120001286F
:102C900003DCFFE7039820B9FFE700208DF813005D
:102CA00040E09DF8120000EBC01141F2B070C2F29A
:102CB000000000EBC10002900298D0F8000401303F
:102CC00000F01F00019001980299D1F80414884285
:102CD00004D1FFE700208DF8130023E0029ED6F810
:102CE000000406EB40114701039A0092D2F810E06D
:102CF0005469156850689368D2F80CC0F5514C615E
:102D0000C1F810E0C1F80CC08B6048609069D269CE
:102D1000CA61886101980299C1F8000401208DF808
:102D20001300FFE79DF8130005B0F0BD80B582B039
:102D3000019001980FF012F902B080BD80B582B009
:102D40008DF806009DF8060001460091052815D86B
:102D50000099DFE801F0031313070B0F062004F0BE
:102D6000FDF80FE00A2004F0F9F80BE0172004F05A
:102D7000F5F807E0092004F0F1F803E0FF208DF8F2
:102D8000070003E000208DF80700FFE79DF907002A
:102D900002B080BD80B582B08DF806009DF80600B7
:102DA00001460091052815D80099DFE801F00313CA
:102DB00013070B0F062004F0DBF80FE00A2004F0E5
:102DC000D7F80BE0172004F0D3F807E0092004F04F
:102DD000CFF803E0FF208DF8070003E000208DF816
:102DE0000700FFE79DF9070002B080BD80B582B003
:102DF0008DF806009DF80600072804DBFFE7002099
:102E00008DF8070013E09DF8062046F2E011C0F6A9
:102E1000010101EBC200406831F8321003F0EAFD15
:102E20000138B0FA80F040098DF80700FFE79DF8FF
:102E3000070002B080BD000083B08DF80A00019148
:102E4000019820B9FFE7FE208DF80B0038E09DF8CF
:102E50000A00072804DBFFE7FF208DF80B002FE0B6
:102E60009DF80A1046F2E010C0F6010030F831007B
:102E7000ADF8020000208DF80100FFE79DF8010089
:102E80000F2819DCFFE7BDF802009DF80110C840CB
:102E9000C00750B1FFE701989DF8012040F238319A
:102EA000C2F2000141F8220006E0FFE79DF80100B0
:102EB00001308DF80100E1E700208DF80B00FFE7FD
:102EC0009DF90B0003B0704780B582B08DF8060005
:102ED0008DF805109DF80600072804DBFFE7FF20AA
:102EE0008DF8070014E09DF8062046F2E011C0F6C8
:102EF000010101EBC200406831F832109DF8052055
:102F000002F0010203F08EFD00208DF80700FFE7BC
:102F10009DF9070002B080BD80B582B00190019894
:102F20000EF07AFD02B080BD86B08DF816008DEDF2
:102F3000040A9DF81600052804DBFFE7FF208DF842
:102F400017008CE09DED040AB7EE001AB4EE410ABA
:102F5000F1EE10FA04DDFFE74FF07E500490FFE73A
:102F60009DED040AB5EE400AF1EE10FA03DAFFE730
:102F700000200490FFE79DF8161046F21820C0F6D6
:102F8000010050F831100968C96A03919DED040AE7
:102F90000399013101EE101AB8EE411A20EE010A30
:102FA000BCEEC00A8DED020A9DF8161000EBC100C0
:102FB000808860B9FFE702989DF8162046F2182134
:102FC000C0F6010151F832100968486343E09DF8EA
:102FD000161046F21820C0F6010000EBC1008088F0
:102FE00004280DD1FFE702989DF8162046F218211B
:102FF000C0F6010151F8321009688863019028E099
:103000009DF8161046F21820C0F6010000EBC10032
:10301000808808280DD1FFE702989DF8162046F217
:103020001821C0F6010151F832100968C8630090F8
:103030000CE002989DF8162046F21821C0F6010116
:1030400051F83210096808640090FFE70098019079
:10305000FFE70198FFE700208DF81700FFE79DF9D3
:10306000170006B07047000080B582B08DF80600EA
:103070009DF80600052804DBFFE7FF208DF8070018
:1030800010E09DF8062046F21820C0F6010000EB83
:10309000C20150F83200898806F088F900208DF8C6
:1030A0000700FFE79DF9070002B080BD80B582B040
:1030B0008DF806009DF80600052804DBFFE7FF20D9
:1030C0008DF8070010E09DF8062046F21820C0F6A3
:1030D000010000EBC20150F83200898806F04CFA7A
:1030E00000208DF80700FFE79DF9070002B080BDC2
:1030F00082B08DF803009DF8030030B9FFE740F679
:103100001820C2F20000019002E000200190FFE7C9
:10311000019802B07047000080B584B08DF80E00B1
:103120000291ADF806208DF805309DF80E000128BB
:1031300004DBFFE7FF208DF80F0029E09DF80E006B
:10314000FFF7D6FF0090009820B9FFE7FF208DF829
:103150000F001DE09DF80500C00760B1FFE7009873
:103160000299BDF8062004F0F7FE002818BF0120E0
:103170008DF80F000CE000980299BDF8062014238A
:1031800004F0C2FD002818BF01208DF80F00FFE7F2
:103190009DF90F0004B080BD82B08DF806008DF857
:1031A00005100092009820B9FFE7FE208DF8070077
:1031B00010E000989DF8062040F28031C2F2000134
:1031C00001EB42119DF8052041F8220000208DF806
:1031D0000700FFE79DF9070002B0704780B584B093
:1031E0008DF80E000291ADF806208DF805309DF89F
:1031F0000E00012804DBFFE7FF208DF80F0029E017
:103200009DF80E00FFF774FF0090009820B9FFE7CB
:10321000FF208DF80F001DE09DF80500C00760B18C
:10322000FFE700980299BDF8062005F0E3FB0028AF
:1032300018BF01208DF80F000CE000980299BDF82E
:103240000620142304F0A8FF002818BF01208DF8E1
:103250000F00FFE79DF90F0004B080BD80B586B078
:1032600004900CF05BFF01464FF47A70B0FBF1F074
:10327000039004980399B0FBF1F002900CF010FF5A
:103280000146481C019198B1FFE70198022820D31C
:10329000FFE7019802280FD0FFE7019803380228C2
:1032A00006D3FFE701986FF00041884215D1FFE790
:1032B000FF208DF8170014E0029818B1FFE702987C
:1032C000009002E001200090FFE700980CF0A2FEC1
:1032D00003E0049803F040F9FFE700208DF81700A1
:1032E000FFE79DF9170006B080BD000080B58AB0E9
:1032F0000CF014FF079010F02BFC079A4FF47A7132
:103300000191B1FBF2F1484306904EF21800CEF263
:10331000000002900068059010F01AFC019A014626
:103320000298079BB2FBF3F25143049100680390AB
:1033300006980499884215D1FFE704984FF47A72F1
:103340005043059951434EF21402CEF20002126826
:103350000132B1FBF2F1401A00F57A7000210991B7
:10336000089014E004984FF47A7250430399514343
:103370004EF21402CEF2000212680132B1FBF2F1F9
:10338000401A00F57A70002109910890FFE708982B
:1033900009990AB080BD000083B08DF807009DF840
:1033A00007000146009120B1FFE70098012806D0F0
:1033B0000BE040F64830C2F20000029008E040F610
:1033C0009030C2F20000029002E000200290FFE77D
:1033D000029803B07047000080B582B00190019858
:1033E00000680068C00600282AD5FFE7FFE7002034
:1033F000009001980068006800900198006840689B
:1034000000900098FFE701980BF0D8FC00EBC0019A
:1034100040F2A430C2F2000000EB8100006A70B1FB
:10342000FFE701980BF0CAFC00EBC00140F2A430AA
:10343000C2F2000000EB8100006A8047FFE7FFE76F
:1034400002B080BD82B08DF806008DF805100092A4
:10345000009820B9FFE7FE208DF8070020E09DF8D6
:103460000600012805DCFFE79DF80500092804DBBC
:10347000FFE7FF208DF8070012E000989DF8061086
:1034800001EBC10240F2A431C2F2000101EB820162
:103490009DF8052041F8220000208DF80700FFE785
:1034A0009DF9070002B07047FFE7FEE780B540F2E4
:1034B0003470C2F2000001F017FF80BD80B540F209
:1034C0003470C2F2000001F00FFF80BD80B540F201
:1034D0003470C2F2000001F007FF80BD80B540F2F9
:1034E0005C70C2F2000001F0FFFE80BD80B540F2CA
:1034F0005C70C2F2000001F0F7FE80BD80B540F2C2
:103500005C70C2F2000001F0EFFE80BD82B000905E
:10351000009820B9FFE703208DF807001DE0009810
:10352000006846F20041C4F20001884204D1FFE77E
:1035300000208DF8070010E00098006846F60001B2
:10354000C4F20001884204D1FFE701208DF8070092
:1035500003E003208DF80700FFE79DF8070002B0A5
:103560007047000083B001900091019820B9FFE7F7
:10357000FF208DF80B005BE0009820B9FFE7FF20EB
:103580008DF80B0054E0019840680099486001985C
:103590008068009988600198C0680099C8600198A7
:1035A000006900990861009890ED030AB6EE001AD0
:1035B00020EE010A80ED050A009890ED040A20EE45
:1035C000010A80ED060A01980078C00720B1FFE7E4
:1035D0000198007D20B9FFE70099002048701DE0A8
:1035E0000198007E022804D1FFE70099012048706D
:1035F00013E00198007E032804D1FFE70099022020
:10360000487009E00198007E012804D1FFE7009985
:1036100003204870FFE7FFE7FFE7FFE70198007826
:10362000009900F00100087000208DF80B00FFE702
:103630009DF90B0003B0704784B003908DED020A32
:10364000CDED010A039890ED000A9DED021A30EECF
:10365000010A8DED000A9DED010AB5EE400AF1EE7A
:1036600010FA26DDFFE79DED000A9DED011AB4EE8C
:10367000410AF1EE10FA09DBFFE79DED011A9DED1D
:10368000000A30EE410A8DED000A11E09DED000ABE
:10369000B5EE400AF1EE10FA09DAFFE79DED011AE6
:1036A0009DED000A30EE010A8DED000AFFE7FFE70D
:1036B000FFE700980399086004B0704785B08DED6E
:1036C000040ACDED030A8DED021A9DED040A9DED6D
:1036D000031A30EE410A8DED010A9DED020AB5EEA6
:1036E000400AF1EE10FA32DDFFE79DED020AB0EE7E
:1036F000001A80EE010A8DED000A9DED010A9DED94
:10370000001AB4EE410AF1EE10FA09DDFFE79DED73
:10371000021A9DED010A30EE410A8DED010A15E015
:103720009DED010A9DED001AB1EE411AB4EE410A79
:10373000F1EE10FA09DAFFE79DED021A9DED010A9C
:1037400030EE010A8DED010AFFE7FFE7FFE79DED8F
:10375000010A05B07047000040F2B400C2F2000058
:103760007047000080B58AB040F2B400C2F2000099
:1037700003904168089180690790089800EB8000E9
:103780004000FFF7C9FB01460398C162C06A58B9FF
:10379000FFE740F2B400C2F20000C06AFFF7C6FAC9
:1037A000FF208DF8270070E007988000FFF7B4FB3A
:1037B000014640F2B400C2F20000C161C06958B9CC
:1037C000FFE740F2B400C2F20000C069FFF7AEFAB2
:1037D000FF208DF8270058E000208DF81B00FFE740
:1037E0009DF81B00089988423CDAFFE740F2B400DC
:1037F000C2F20000C06A9DF81B1001EB810100EBD2
:103800004100009001208DF810009DF81B1001F27E
:103810000121ADF812108DF8140004A905310191B1
:103820009DF81B100129029008D0FFE79DF81B00AE
:103830000238B0FA80F040090290FFE70099019A3F
:10384000029800F00100107000208DF81600049816
:10385000059A4A600860FFE79DF81B0001308DF86B
:103860001B00BDE740F2B400C2F20000C26A0121B1
:103870001172C26A9174C26A1177C1694FF07E50A9
:10388000086000208DF82700FFE79DF927000AB0A7
:1038900080BD000080B584B00290029820B9FFE797
:1038A000FE208DF80F002BE040F61940C2F2000018
:1038B0000078C00720B1FFE7FD208DF80F001FE062
:1038C0000DF048F841F2A871C2F20001086020B979
:1038D000FFE7FE208DF80F0012E044F2E122C0F66F
:1038E0000002002001900321FFF7ACFD019840F693
:1038F0001942C2F20002012111708DF80F00FFE79A
:103900009DF90F0004B080BD80B59CB01B901A914A
:103910001B994878897840EA01216FF3DF2141F251
:103920002050C2F20000199001801B9A9178D27841
:10393000C90841EA42116FF3DF2141801B9AD17817
:1039400013795279890941EA830141EA82216FF3AF
:10395000DF2181801B9A51799279490841EAC2118D
:103960006FF3DF21C1801B9A9179D279090941EA6D
:1039700002116FF3DF2101811B9AD179137A527AF8
:10398000C90941EA430141EA42216FF3DF21418144
:103990001B9A517A927A890841EA82116FF3DF21EA
:1039A00081811B9A917AD27A490941EAC201C18187
:1039B0001B9A117B527B41EA02216FF3DF210182C6
:1039C0001B9A517B927BC90841EA42116FF3DF21B8
:1039D00041821B9A917BD37B127C890941EA830146
:1039E00041EA82216FF3DF2181821B9A117C527C94
:1039F000490841EAC2116FF3DF21C182B0F9061014
:103A000000EE101AB8EEC00A9FEDDA1A30EE010A85
:103A100030EE000A9FEDD82A80EE020AB7EE001AB7
:103A200030EE410A1A9981ED010AB0F9041000EE56
:103A3000101AB8EEC00A9FEDD13A30EE030A30EE0C
:103A4000000A9FEDCF3A80EE030A30EE410A1A9940
:103A500081ED020AB0F9001000EE101AB8EEC00AAB
:103A60009FEDC83A30EE030A30EE000A9FEDC63AE9
:103A700080EE030A30EE410A1A9981ED030AB0F98B
:103A8000020000EE100AB8EEC00A9FEDC03A30EE18
:103A9000030A30EE000A80EE020A30EE410A1A985C
:103AA00080ED040A1A98406812F006FA41EC100BF7
:103AB0009FEDB71B50EC111BC20F51EC100B62F3C2
:103AC000DF7141EC100B51EC100B9FEDB30B53EC7D
:103AD000102B12F02AFA20B9FFE71A99002048604B
:103AE000FFE71A98806812F0E7F941EC100B9FEDA0
:103AF000A81B50EC111BC20F51EC100B62F3DF71CD
:103B000041EC100B51EC100B9FEDA50B53EC102B5F
:103B100012F00BFA20B9FFE71A9900208860FFE73E
:103B20001A98C06812F0C8F941EC100B9FED981B71
:103B300050EC111BC20F51EC100B62F3DF7141EC22
:103B4000100B51EC100B9FED940B53EC102B12F05B
:103B5000ECF920B9FFE71A990020C860FFE71A982E
:103B6000006912F0A9F941EC100B9FED891B50EC94
:103B7000111BC20F51EC100B62F3DF7141EC100B03
:103B800051EC100B9FED840B53EC102B12F0CDF980
:103B900020B9FFE71A9900200861FFE71A984068EA
:103BA00012F08AF941EC100B9FED791B50EC111BC0
:103BB000C20F51EC100B62F3DF7141EC100B51ECB2
:103BC000100B9FED790B53EC102B12F0C3F988B951
:103BD000FFE71A9890ED012AB7EE001ABFEE000A2F
:103BE000B5EE402AF1EE10FAC8BFB0EE410A80ED02
:103BF000010AFFE71A98806812F05EF941EC100B99
:103C00009FED631B50EC111BC20F51EC100B62F3C4
:103C1000DF7141EC100B51EC100B9FED630B53EC7B
:103C2000102B12F097F988B9FFE71A9890ED022A45
:103C3000B7EE001ABFEE000AB5EE402AF1EE10FA18
:103C4000C8BFB0EE410A80ED020AFFE71A98C068CB
:103C500012F032F941EC100B9FED4D1B50EC111B93
:103C6000C20F51EC100B62F3DF7141EC100B51EC01
:103C7000100B9FED4D0B53EC102B12F06BF988B924
:103C8000FFE71A9890ED032AB7EE001ABFEE000A7C
:103C9000B5EE402AF1EE10FAC8BFB0EE410A80ED51
:103CA000030AFFE71A98006912F006F941EC100BBD
:103CB0009FED371B50EC111BC20F51EC100B62F340
:103CC000DF7141EC100B51EC100B9FED370B53ECF7
:103CD000102B12F03FF988B9FFE71A9890ED042AEB
:103CE000B7EE001ABFEE000AB5EE402AF1EE10FA68
:103CF000C8BFB0EE410A80ED040AFFE741F2205050
:103D0000C2F20000B0F90800B0F5967F0DDDFFE7C4
:103D100041F22050C2F20000B0F90800B0F5FA7F7D
:103D200003DAFFE7012018905BE041F22050C2F275
:103D30000000B0F90800B0F5FA7F0EDBFFE741F2B2
:103D40002050C2F20000B0F9080040F2DB51884276
:103D500003DCFFE70320179040E041F22050C2F25D
:103D60000000B0F90810002040F2DC529142169099
:103D70002CDB1DE0000051C30060AD44000032C3E5
:103D80000020AC44000052C30040AD4400005DC3BD
:103D90000000000000000000000000A09999A93F69
:103DA000000000A09999C93F000000000000F03F0A
:103DB00041F22050C2F20000B0F9081040F2A462B3
:103DC00000209142B8BF01201690FFE7169800F03E
:103DD0000100002818BF02201790FFE717981890DD
:103DE000FFE718981A99087541F22050C2F20000B6
:103DF000B0F90A00B0F5967F0DDDFFE741F22050E3
:103E0000C2F20000B0F90A00B0F5FA7F03DAFFE76A
:103E1000012015903DE041F22050C2F20000B0F9BF
:103E20000A00B0F5FA7F0EDBFFE741F22050C2F244
:103E30000000B0F90A0040F2DB51884203DCFFE7E2
:103E40000320149022E041F22050C2F20000B0F9A9
:103E50000A10002040F2DC52914213900EDBFFE783
:103E600041F22050C2F20000B0F90A1040F2A46200
:103E700000209142B8BF01201390FFE7139800F093
:103E80000100002818BF02201490FFE71498159035
:103E9000FFE715981A99487541F22050C2F20000C8
:103EA000B0F90C00B0F5967F0DDDFFE741F2205030
:103EB000C2F20000B0F90C00B0F5FA7F03DAFFE7B8
:103EC000012012903DE041F22050C2F20000B0F912
:103ED0000C00B0F5FA7F0EDBFFE741F22050C2F292
:103EE0000000B0F90C0040F2DB51884203DCFFE730
:103EF0000320119022E041F22050C2F20000B0F9FC
:103F00000C10002040F2DC52914210900EDBFFE7D3
:103F100041F22050C2F20000B0F90C1040F2A4624D
:103F200000209142B8BF01201090FFE7109800F0E8
:103F30000100002818BF02201190FFE7119812908D
:103F4000FFE712981A99887541F22050C2F20000DA
:103F5000B0F90E00B0F5967F0DDDFFE741F220507D
:103F6000C2F20000B0F90E00B0F5FA7F03DAFFE705
:103F700002200F903AE041F22050C2F20000B0F966
:103F80000E00B0F5FA7F0EDBFFE741F22050C2F2DF
:103F90000000B0F90E0040F2DB51884203DCFFE77D
:103FA00003200E901FE041F22050C2F20000B0F951
:103FB0000E10002040F2DC5291420D900EDBFFE724
:103FC00041F22050C2F20000B0F90E1040F2A4629B
:103FD00000209142B8BF01200D90FFE70D9800F03E
:103FE00001000E90FFE70E980F90FFE70F981A99C7
:103FF000C87541F22050C2F20000B0F91000B0F5CF
:10400000967F0DDDFFE741F22050C2F20000B0F9CB
:104010001000B0F5FA7F03DAFFE702200C903AE0D7
:1040200041F22050C2F20000B0F91000B0F5FA7F62
:104030000EDBFFE741F22050C2F20000B0F91000A1
:1040400040F2DB51884203DCFFE703200B901FE0C6
:1040500041F22050C2F20000B0F91010002040F2EE
:10406000DC5291420A900EDBFFE741F22050C2F28F
:104070000000B0F9101040F2A46200209142B8BFD5
:1040800001200A90FFE70A9800F001000B90FFE77B
:104090000B980C90FFE70C981A99087641F2205083
:1040A000C2F20000B0F91200B0F5967F0DDDFFE717
:1040B00041F22050C2F20000B0F91200B0F5FA7FD0
:1040C00003DAFFE7022009903AE041F22050C2F201
:1040D0000000B0F91200B0F5FA7F0EDBFFE741F205
:1040E0002050C2F20000B0F9120040F2DB518842C9
:1040F00003DCFFE7032008901FE041F22050C2F2EA
:104100000000B0F91210002040F2DC5291420790FA
:104110000EDBFFE741F22050C2F20000B0F91210AE
:1041200040F2A46200209142B8BF01200790FFE74F
:10413000079800F001000890FFE708980990FFE752
:1041400009981A99487641F22050C2F20000B0F95D
:104150001400B0F5967F0DDDFFE741F22050C2F26A
:104160000000B0F91400B0F5FA7F03DAFFE7012090
:1041700006903DE041F22050C2F20000B0F9140078
:10418000B0F5FA7F0EDBFFE741F22050C2F20000EB
:10419000B0F9140040F2DB51884203DCFFE7032052
:1041A000059022E041F22050C2F20000B0F9141054
:1041B000002040F2DC52914204900EDBFFE741F216
:1041C0002050C2F20000B0F9141040F2A4620020A6
:1041D0009142B8BF01200490FFE7049800F001006D
:1041E000002818BF02200590FFE705980690FFE71A
:1041F00006981A99887641F22050C2F20000B0F970
:104200001600B0F5967F0DDDFFE741F22050C2F2B7
:104210000000B0F91600B0F5FA7F03DAFFE70220DC
:1042200003903AE041F22050C2F20000B0F91600CB
:10423000B0F5FA7F0EDBFFE741F22050C2F200003A
:10424000B0F9160040F2DB51884203DCFFE703209F
:1042500002901FE041F22050C2F20000B0F91610A7
:10426000002040F2DC52914201900EDBFFE741F268
:104270002050C2F20000B0F9161040F2A4620020F3
:104280009142B8BF01200190FFE7019800F00100C2
:104290000290FFE702980390FFE703981A99C87607
:1042A00041F22050C2F20000B0F916100020B1F522
:1042B000967F00900CD0FFE741F22050C2F2000040
:1042C000B0F90000B0F57A7018BF01200090FFE748
:1042D00000981A9900F0010008701CB080BD000021
:1042E00080B541F2A870C2F20000006880210CF095
:1042F00051FA80BD80B582B000900020FFF74CF8E5
:104300000099192205F07AFD20B9FFE700208DF809
:10431000070003E0FF208DF80700FFE79DF9070085
:1043200002B080BD80B582B00190019A8020012149
:104330000CF082FA8038B0FA80F0400902B080BDFB
:1043400080B540F6A400C2F2000001F05BFE80BD23
:1043500080B540F28470C2F2000001F053FE80BDCF
:1043600080B540F60410C2F2000001F04BFE80BDA3
:1043700080B540F2E470C2F2000001F043FE80BD5F
:1043800080B540F64400C2F2000001F03BFE80BD63
:1043900080B540F66410C2F2000001F033FE80BD2B
:1043A00082B001900198007810384AF6AB21CAF625
:1043B000AA21A0FB011000090090009946F2D81034
:1043C000C0F60100405C0199C8650098042807D335
:1043D000FFE701990868042262F30900886506E096
:1043E0000199086840F2FF3290438865FFE7019821
:1043F000806D02B07047000086B0059000208DF8F7
:1044000013000598806A03900598806910BBFFE748
:104410000398029003281BD80299DFE801F0020DEF
:104420000218059890F82F00C00720B1FFE701207F
:104430008DF81300FFE70CE00598C06AB0F1C07F6B
:1044400004D1FFE701208DF81300FFE701E000E051
:10445000FFE745E005988069B0F5005F25D1FFE7EB
:104460000398019003281ED80199DFE801F00206A5
:10447000021101208DF8130016E0059890F82F0026
:10448000C00720B1FFE701208DF81300FFE70BE024
:104490000598C06AB0F1C07F04D1FFE701208DF814
:1044A0001300FFE700E0FFE719E0039800900328FE
:1044B00004D3FFE70098032804D00EE001208DF814
:1044C00013000BE0059890F82F00C00720B1FFE71C
:1044D00001208DF81300FFE700E0FFE7FFE7FFE7AB
:1044E0009DF8130006B0704784B0039002910192CA
:1044F000009303980168086820F480200860009801
:1045000003990968486003988068402809D1FFE74B
:104510000198039909688860029803990968C8603E
:1045200008E002980399096888600198039909686E
:10453000C860FFE704B070477047000080B50120F5
:1045400002F060F880BD000080B5082002F05AF843
:1045500080BD000080B5102002F054F880BD00003E
:1045600080B5202002F04EF880BD000072B6FFE753
:10457000FEE7000080B592B010900F91109818B12E
:10458000FFE70F9820B9FFE7FF208DF84700C0E153
:10459000FEF7ACFE109A049213685268C01A91415B
:1045A00011F0DFFC0146049800EE101A9FEDDB1AB3
:1045B00080EE010A80ED020AFEF798FE0A46109985
:1045C0004A60086010980F99097800F07DFA0F98FA
:1045D00090ED010A109890ED021A20EE010AB7EE54
:1045E000081A20EE010A8DED0E0A1098C06890EDB1
:1045F000280AB5EE400AF1EE10FA72DDFFE71098D6
:1046000090ED5D1A90ED600A30EE410A8DED0D0AD5
:104610009DED0D0A9FEDC21AB4EE410AF1EE10FABB
:1046200009DDFFE79DED0D0A9FEDBE1A30EE010A90
:104630008DED0D0AFFE79DED0D0A9FEDBB1AB4EE5F
:10464000410AF1EE10FA09DAFFE79DED0D0A9FED40
:10465000B71A30EE010A8DED0D0AFFE7109890EDC4
:10466000051A90ED440A9DED0D2A31EE021A9DEDDA
:104670000E2A71EE020A9FEDAD1A8DED031AFFF7B7
:104680001DF89DED031A8DED0C0A109890ED052A8A
:1046900090ED450A9DED0D3A32EE032A9DED0E3A5E
:1046A00072EE030AFFF70AF88DED0B0A9DED0E0A74
:1046B0009DED0C1AB4EE410AF1EE10FA03DDFFE7AE
:1046C0000C980E90FFE79DED0E0A9DED0B1AB4EECF
:1046D000410AF1EE10FA03DAFFE70B980E90FFE7BC
:1046E000FFE7109814309DED0E0ADFED900AFEF7FB
:1046F000A3FF0F9890ED020A109890ED021A20EE99
:10470000010A8DED0A0A1098C06890ED290AB5EEED
:10471000400AF1EE10FA6BDDFFE7002009909DEDF5
:10472000090A9FED7F1AB4EE410AF1EE10FA09DD95
:10473000FFE79DED090A9FED7B1A30EE010A8DED32
:10474000090AFFE79DED090A9FED771AB4EE410AC9
:10475000F1EE10FA09DAFFE79DED090A9FED731AF1
:1047600030EE010A8DED090AFFE7109890ED061A68
:1047700090ED460A9DED092A31EE021A9DED0A2AB6
:1047800071EE020A9FED691A8DED021AFEF796FF8F
:104790009DED021A8DED080A109890ED062A90ED15
:1047A000470A9DED093A32EE032A9DED0A3A72EE70
:1047B000030AFEF783FF8DED070A9DED0A0A9DEDC2
:1047C000081AB4EE410AF1EE10FA03DDFFE708988B
:1047D0000A90FFE79DED0A0A9DED071AB4EE410A23
:1047E000F1EE10FA03DAFFE707980A90FFE7FFE718
:1047F000109818309DED0A0ADFED4C0AFEF71CFFF9
:104800000F9890ED020AB0EE081A80EE010A9FEDB3
:10481000481A30EE010A9FED471A30EE010A10984F
:1048200080ED060A1098007C0146019140B1FFE737
:10483000019801280CD0FFE7019802285DD064E0C0
:1048400010990020C1F860011099C1F864015CE082
:10485000109901F12000D1ED021A91ED050AD1ED78
:104860005D0A9FED351A8DED001A07F071F99DED87
:10487000001A8DED060A109901F1D4009DED060A8B
:10488000D1ED021AD1ED5C0A07F062F99DED001A34
:10489000109880ED580A109901F19800D1ED021A94
:1048A00091ED060AD1ED640A07F052F99DED001A68
:1048B0008DED050A109901F1D4009DED050AD1EDA9
:1048C000021AD1ED5A0A07F043F9109880ED590AFF
:1048D000109901F5907091ED580A05F0B7FB10980A
:1048E00080ED580A109901F5A07091ED590A05F074
:1048F000ADFB109880ED590A07E010990020C1F82F
:1049000060011099C1F86401FFE700208DF84700AD
:10491000FFE79DF9470012B080BD00BF0024744935
:10492000DB0F4940DB0FC9C0DB0F49C0DB0FC940BB
:1049300052B83E40ABAAAA3E0000000080B586B047
:10494000049003918DED020A049820B9FFE7FF203F
:104950008DF817007BE003980499C8600498002143
:1049600001910174049A02F120009DED020AD268BF
:10497000303207F065FA049901F15C009DED020AFE
:10498000C96801F110020121009107F059FA01995B
:10499000049A02F198009DED020AD268703207F085
:1049A0004FFA0099049A02F1D4009DED020AD268F0
:1049B000503207F045FA049901F590709DED020A16
:1049C000C968D1ED240A05F09DFB049901F5A0709A
:1049D0009DED020AC968D1ED240A05F093FB049805
:1049E000C16891ED260A91ED281A30EE010A80ED9A
:1049F000440A0499C868D0F89800C1F814010498D2
:104A0000C16891ED270A91ED291A30EE010A80ED77
:104A1000460A0499C868D0F89C00C1F81C01FDF74B
:104A20004FFD0498C06805F00BFE0498C06808307C
:104A300005F006FE0498C06805F098FC0498C0686C
:104A4000083005F093FC01988DF81700FFE79DF9F9
:104A5000170006B080BD000080B58CB00B90002020
:104A600000900A9009900890079006900B9890ED9E
:104A7000590AB1EE041A20EE010A8DED060A4FF034
:104A80007E500A900B98C06806A905F009FD0098B1
:104A9000059004900390029001900B9890ED580AB5
:104AA000B2EE001A20EE010A8DED010A49F69A10C5
:104AB000C3F6996005900B98C068083001A905F00D
:104AC000EFFC0CB080BD000080B584B002908DF882
:104AD0000710029820B9FFE7FF208DF80F0047E08C
:104AE0009DF807000299097C884204D1FFE7002065
:104AF0008DF80F003CE00298203007F06DFA029824
:104B00005C3007F069FA0298983007F065FA02986D
:104B1000D43007F061FA029800F590709FED160A04
:104B20008DED000A05F08CFB9DED000A029800F562
:104B3000A07005F085FB0298C068083005F016FCEF
:104B40000298C06805F012FC02981430FBF706FFCB
:104B50000299D1F8900188610299D1F874014861F5
:104B60009DF807000299087400208DF80F00FFE7F8
:104B70009DF90F0004B080BD0000000080B584B036
:104B80000290029820B9FFE7FF208DF80F0045E062
:104B90000298C06805F08CFE0298C06805F03CFCE5
:104BA00001900198A0B1FFE70299DDF804C0DCF89C
:104BB0001C00DCF82020DCF82430DCF828C0C1F828
:104BC0009CC1C1F89831C1F89421C1F89001FFE768
:104BD0000298C068083005F06BFE0298C068083083
:104BE00005F01AFC00900098A0B1FFE70299DDF8EB
:104BF00000C0DCF81C00DCF82020DCF82430DCF8F5
:104C000028C0C1F88CC1C1F88831C1F88421C1F82D
:104C10008001FFE700208DF80F00FFE79DF90F00EE
:104C200004B080BD83B001900091019820B9FFE7E6
:104C3000FF208DF80B0019E00199009B18685A6855
:104C40009B68C1F87031C1F86C21C1F86801019905
:104C5000009BD8681A695B69C1F87C31C1F878217A
:104C6000C1F8740100208DF80B00FFE79DF90B00DF
:104C700003B0704784B002900191029890F8200030
:104C80008DF803009DF80300012805D0FFE79DF88B
:104C9000030002280AD1FFE7019A029801684869D7
:104CA0001043486100208DF80F0008E00299486A1F
:104CB00040F48020486201208DF80F00FFE79DF846
:104CC0000F0004B07047000088B006900591049270
:104CD0000393069890F820008DF807000698006866
:104CE000806800900598806808B9FFE700E0FFE75A
:104CF0009DF80700012806D0FFE79DF8070002286D
:104D000040F08080FFE79DF80300400700280CD4A6
:104D1000FFE79DF803000007002806D4FFE79DF891
:104D20000300C006002864D5FFE70098C0F30160C7
:104D300002900299012088400399086005988068D4
:104D400068B9FFE705980168C06840EA41500699D4
:104D50000968029A01EB0211C1F880010EE0059981
:104D60004A688868C96840EAC20008430699096829
:104D7000029A01EB0211C1F88001FFE70598006972
:104D800006990968029A01EB0211C1F8840105989D
:104D9000007D01280CD1FFE706980068029900EB1E
:104DA0000111D1F8840140F48070C1F88401FFE75B
:104DB0000498406806990968029A01EB0211C1F84B
:104DC0008C010498006806990968029A01EB0211A7
:104DD000C1F8880106980068029900EB0111D1F82A
:104DE000800140F00100C1F8800100208DF81F0013
:104DF00011E00699486A40F40010486201208DF8DD
:104E00001F0008E00699486A40F4802048620120AB
:104E10008DF81F00FFE79DF81F0008B070470000E5
:104E200086B004900391049890F820008DF8030058
:104E30009DF80300012806D0FFE79DF80300022833
:104E400040F0B080FFE746F20040C4F2000001905D
:104E50000199D1F8000240F00100C1F80002019967
:104E6000D1F8000220F47C50C1F800020398426A95
:104E70000199D1F8000240EA0220C1F8000203982B
:104E8000406900F01F01012088400290029A0199B8
:104E9000D1F81C029043C1F81C020398C069F0B914
:104EA000FFE7029A0199D1F80C029043C1F80C0275
:104EB000039A9088D168526940EA0140019901EB58
:104EC000C201C1F84002039A10889168526940EA11
:104ED0000140019901EBC201C1F84402FFE70398C8
:104EE000C06901281ED1FFE7029A0199D1F80C028E
:104EF0001043C1F80C02039A90881168526940EA85
:104F00000140019901EBC201C1F84002039A908966
:104F10009168526940EA0140019901EBC201C1F870
:104F20004402FFE70398806940B9FFE7029A0199BC
:104F3000D1F804029043C1F8040207E0029A0199F3
:104F4000D1F804021043C1F80402FFE70398006996
:104F500040B9FFE7029A0199D1F814029043C1F8D1
:104F6000140207E0029A0199D1F814021043C1F823
:104F70001402FFE70398006A012808D1FFE7029AAC
:104F80000199D1F81C021043C1F81C02FFE70199F6
:104F9000D1F8000220F00100C1F8000200208DF8D5
:104FA000170008E00499486A40F480204862012014
:104FB0008DF81700FFE79DF8170006B07047000056
:104FC00080B582B001900198FEF7A0FA8DF8030039
:104FD0009DF80300032819D0FFE79DF8030040F275
:104FE000D022C2F20002342110FB0120006B60B11C
:104FF000FFE79DF8030040F2D022C2F20002342104
:1050000010FB0120006B8047FFE7FFE702B080BD87
:1050100084B00390029100200190039890F8200042
:105020008DF803009DF80300012805D0FFE79DF8E7
:105030000300022812D1FFE7029838B9FFE703986E
:105040000068C06800F00300019006E00398006863
:10505000006900F003000190FFE7FFE7019804B04A
:105060007047000086B00490039102920193049867
:1050700090F820008DF803009DF80300012806D069
:10508000FFE79DF80300022840F0E880FFE703985F
:1050900080B9FFE704980068C068800748B9FFE757
:1050A0000499486A40F40010486201208DF8170006
:1050B000DDE00FE0049800680069800748B9FFE769
:1050C0000499486A40F40010486201208DF81700E6
:1050D000CDE0FFE704980068039900EB0110D0F8D9
:1050E000B00100F00400029988600298806858B905
:1050F000FFE704980068039900EB0110D0F8B001B5
:10510000400D029908600AE004980068039900EBDA
:105110000110D0F8B001C00802994860FFE7049878
:105120000068039900EB0110D0F8B00100F0020014
:105130000299C86004980068039900EB0110D0F848
:10514000B40100F00F00082804D3FFE702990820FB
:1051500008610BE004980068039900EB0110D0F897
:10516000B40100F00F0002990861FFE7049800689D
:10517000039900EB0110D0F8B40180B2000A029943
:10518000886104980068039900EB0110D0F8B4011D
:10519000000C0299486104980068039900EB011023
:1051A000D0F8B8010199087004980068039900EBE1
:1051B0000110D0F8B801000A0199487004980068FD
:1051C000039900EB0110D0F8B801000C0199887028
:1051D00004980068039900EB0110D0F8B801000EA4
:1051E0000199C87004980068039900EB0110D0F889
:1051F000BC010199087104980068039900EB011043
:10520000D0F8BC01000A019948710498006803991C
:1052100000EB0110D0F8BC01000C019988710498D2
:105220000068039900EB0110D0F8BC01000E019951
:10523000C871039838B9FFE704980168C86840F05E
:105240002000C86006E004980168086940F020006A
:105250000861FFE700208DF8170008E00499486A0C
:1052600040F48020486201208DF81700FFE79DF888
:10527000170006B07047000083B002900020019034
:10528000029890F820008DF803009DF80300012893
:1052900005D0FFE79DF80300022822D1FFE702981E
:1052A000006880684001002804D5FFE701980130BC
:1052B0000190FFE70298006880680001002804D58B
:1052C000FFE7019801300190FFE7029800688068CD
:1052D000C000002804D5FFE7019801300190FFE7E6
:1052E000FFE7019803B0704780B58AB009900020AD
:1052F000089009980068406907900998006840681C
:105300000690099800688068059009980068C06850
:105310000490099800680069039009980068806902
:1053200002909DF81C00C007002800F09480FFE761
:105330009DF81400C00758B3FFE7099801680120E1
:1053400088609DF814008007002804D5FFE70998BD
:1053500000F0D2FC1BE09DF814004007002805D5A2
:10536000FFE7089840F4006008900FE09DF81400F3
:105370000007002805D5FFE7089840F48050089002
:1053800003E0099800F090FCFFE7FFE7FFE7FFE785
:105390009DF81500C00760B3FFE7099801684FF456
:1053A000807088609DF815008007002804D5FFE70D
:1053B000099800F0EFFC1BE09DF81500400700285D
:1053C00005D5FFE7089840F4005008900FE09DF8DD
:1053D00015000007002805D5FFE7089840F4804035
:1053E000089003E0099800F0ADFCFFE7FFE7FFE756
:1053F000FFE79DF81600C00760B3FFE70998016852
:105400004FF4803088609DF816008007002804D58E
:10541000FFE7099800F00EFD1BE09DF8160040071D
:10542000002805D5FFE7089840F4004008900FE0F9
:105430009DF816000007002805D5FFE7089840F4FE
:105440008030089003E0099800F0CCFCFFE7FFE70C
:10545000FFE7FFE7FFE79DF81C000007002810D5D5
:10546000FFE79DF81000C006002809D5FFE708985F
:1054700040F400700890099801681020C860FFE7A8
:10548000FFE79DF81C00400700280FD5FFE79DF8B7
:1054900010000007002808D5FFE7099801680820D8
:1054A000C860099800F0F2FAFFE7FFE79DF81C00DA
:1054B000800700280BD5FFE709980068C0688007BF
:1054C00020B1FFE7099800F009FBFFE7FFE79DF82F
:1054D0001C004006002810D5FFE79DF80C00C00610
:1054E000002809D5FFE7089840F4806008900998E3
:1054F000016810200861FFE7FFE79DF81C008006A7
:1055000000280FD5FFE79DF80C000007002808D5FC
:10551000FFE70998016808200861099800F006FB78
:10552000FFE7FFE79DF81C00C00600280BD5FFE74A
:10553000099800680069800720B1FFE7099800F02A
:105540001DFBFFE7FFE79DF81E00800700280FD531
:10555000FFE79DF81800C006002808D5FFE7099866
:10556000016810204860099800F030FBFFE7FFE772
:105570009DF81E00C00778B1FFE79DF818000007EE
:10558000002808D5FFE709980168082048600998B5
:1055900000F078FCFFE7FFE79DF81D0000060028FB
:1055A00040F18D80FFE79DF818004007002840F18A
:1055B0008180FFE79DF81D00C00750B1FFE79DF80F
:1055C0000800C00728B1FFE7089840F001000890E4
:1055D000FFE79DF81D00800700280BD5FFE79DF829
:1055E00008008007002805D5FFE7089840F0020072
:1055F0000890FFE79DF81D00400700280BD5FFE746
:105600009DF808004007002805D5FFE7089840F0FE
:1056100004000890FFE79DF81D000007002848D50A
:10562000FFE79DF8080010F0700F42D0FFE70298E6
:1056300000F0700001460191102814D0FFE7019896
:10564000202815D0FFE70198302816D0FFE70198F1
:10565000402817D0FFE70198502818D0FFE701989D
:10566000602819D01DE0089840F00800089019E063
:10567000089840F01000089014E0089840F02000CE
:1056800008900FE0089840F0400008900AE0089861
:1056900040F08000089005E0089840F48070089081
:1056A00000E0FFE709980168886920F070008861D0
:1056B000FFE7FFE70998016804204860FFE70898C2
:1056C00048B1FFE7089A0999486A10434862099867
:1056D000FFF776FCFFE70AB080BD000080B584B01C
:1056E0000290029820B9FFE701208DF80F00E0E05A
:1056F000029890F8200020B9FFE7029800F0DEF849
:10570000FFE702980168086840F00100086001F0B6
:10571000A1F90190FFE7029800684068C007A8B9A6
:10572000FFE701F097F90199401A0B280DD3FFE725
:105730000299486A40F4003048620299052081F8D5
:10574000200001208DF80F00B3E0E4E70298016823
:10575000086820F00200086001F07CF90190FFE782
:105760000298006840688007002815D5FFE701F01F
:1057700071F90199401A0B280DD3FFE70299486A85
:1057800040F4003048620299052081F82000012091
:105790008DF80F008DE0E3E70298007E012807D125
:1057A000FFE702980168086840F08000086006E0A2
:1057B00002980168086820F080000860FFE70298FE
:1057C000407E012807D1FFE702980168086840F091
:1057D0004000086006E002980168086820F0400078
:1057E0000860FFE70298807E012807D1FFE7029852
:1057F0000168086840F02000086006E0029801682F
:10580000086820F020000860FFE70298C07E0128A9
:1058100007D1FFE702980168086820F010000860CF
:1058200006E002980168086840F010000860FFE791
:105830000298007F012807D1FFE7029801680868F5
:1058400040F00800086006E002980168086820F04F
:1058500008000860FFE70298407F012807D1FFE7B2
:1058600002980168086840F00400086006E00298A9
:105870000168086820F004000860FFE7029B1968CF
:105880005A689868D3F80CC040EA0C00D3F810C0EE
:1058900040EA0C005B691843013A1043C861029961
:1058A00000204862029A012182F820108DF80F0032
:1058B000FFE79DF80F0004B080BD000080B596B0F2
:1058C000159000201490139012901190109015983C
:1058D000006846F20041C4F2000188425CD1FFE753
:1058E00040F27830C2F200000168013101600068C6
:1058F000012812D1FFE7FFE700200F9043F6400098
:10590000C4F20200016841F000710160006800F01B
:1059100000700F900F98FFE7FFE7FFE700200E9061
:1059200043F63000C4F20200016841F00801016052
:10593000006800F008000E900E98FFE7032010901A
:1059400002211191002109911291139009201490C4
:1059500040F60040C4F2020010A900F06FFE099A60
:10596000132006900521089101F00CFB069801F028
:10597000FFFA0899099A1420079001F003FB079891
:1059800001F0F6FA0899099A15200A9001F0FAFA3E
:105990000A9801F0EDFA77E01598006846F60001E4
:1059A000C4F2000188426ED1FFE7FFE700200D90AE
:1059B00043F64000C4F20200016841F080610160DA
:1059C000006800F080600D900D98FFE740F278309D
:1059D000C2F200000168013101600068012812D1A3
:1059E000FFE7FFE700200C9043F64000C4F20200FE
:1059F000016841F000710160006800F000700C90D7
:105A00000C98FFE7FFE7FFE700200B9043F630001C
:105A1000C4F20200016841F002010160006800F078
:105A200002000B900B98FFE760201090022011906D
:105A3000002004901290032013900920149040F24B
:105A40000040C4F2020010A900F0F8FD049A3F20C3
:105A500001900521039101F095FA019801F088FA6F
:105A60000399049A4020029001F08CFA029801F008
:105A70007FFA0399049A4120059001F083FA059872
:105A800001F076FAFFE7FFE716B080BD80B582B07F
:105A900001900198FDF73AFD8DF803009DF8030091
:105AA000032819D0FFE79DF8030040F2D022C2F28C
:105AB0000002342110FB0120C06960B1FFE79DF8AE
:105AC000030040F2D022C2F20002342110FB012078
:105AD000C0698047FFE7FFE702B080BD80B582B0B4
:105AE00001900198FDF712FD8DF803009DF8030069
:105AF000032819D0FFE79DF8030040F2D022C2F23C
:105B00000002342110FB0120806960B1FFE79DF89D
:105B1000030040F2D022C2F20002342110FB012027
:105B200080698047FFE7FFE702B080BD80B582B0A3
:105B300001900198FDF7EAFC8DF803009DF8030041
:105B4000032819D0FFE79DF8030040F2D022C2F2EB
:105B50000002342110FB0120406A60B1FFE79DF88C
:105B6000030040F2D022C2F20002342110FB0120D7
:105B7000406A8047FFE7FFE702B080BD80B582B092
:105B800001900198FDF7C2FC8DF803009DF8030019
:105B9000032819D0FFE79DF8030040F2D022C2F29B
:105BA0000002342110FB0120006A60B1FFE79DF87C
:105BB000030040F2D022C2F20002342110FB012087
:105BC000006A8047FFE7FFE702B080BD80B582B082
:105BD00001900198FDF79AFC8DF803009DF80300F1
:105BE000032819D0FFE79DF8030040F2D022C2F24B
:105BF0000002342110FB0120806A60B1FFE79DF8AC
:105C0000030040F2D022C2F20002342110FB012036
:105C1000806A8047FFE7FFE702B080BD80B584B0AF
:105C20000290029890F8200001282FD1FFE70299F6
:105C3000022081F8200002980168086820F0010025
:105C4000086000F007FF0190FFE7029800684068D5
:105C5000C007A8B1FFE700F0FDFE0199401A0B282C
:105C60000DD3FFE70299486A40F400304862029978
:105C7000052081F8200001208DF80F000FE0E4E7F7
:105C80000299002048628DF80F0008E00299486AE6
:105C900040F40020486201208DF80F00FFE79DF8D6
:105CA0000F0004B080BD000080B582B00190019863
:105CB000FDF72CFC8DF803009DF80300032819D094
:105CC000FFE79DF8030040F2D022C2F20002342127
:105CD00010FB0120C06860B1FFE79DF8030040F2AF
:105CE000D022C2F20002342110FB0120C06880479C
:105CF000FFE7FFE702B080BD80B582B00190019858
:105D0000FDF704FC8DF803009DF80300032817D06D
:105D1000FFE79DF803003421414340F2D020C2F256
:105D20000000405858B1FFE79DF80300342141437B
:105D300040F2D020C2F2000040588047FFE7FFE762
:105D400002B080BD80B582B001900198FDF7DEFB06
:105D50008DF803009DF80300032819D0FFE79DF894
:105D6000030040F2D022C2F20002342110FB0120D5
:105D7000006960B1FFE79DF8030040F2D022C2F253
:105D80000002342110FB012000698047FFE7FFE794
:105D900002B080BD80B582B001900198FDF7B6FBDE
:105DA0008DF803009DF80300032819D0FFE79DF844
:105DB000030040F2D022C2F20002342110FB012085
:105DC000406860B1FFE79DF8030040F2D022C2F2C4
:105DD0000002342110FB012040688047FFE7FFE705
:105DE00002B080BD80B582B001900198FDF78EFBB6
:105DF0008DF803009DF80300032819D0FFE79DF8F4
:105E0000030040F2D022C2F20002342110FB012034
:105E1000406960B1FFE79DF8030040F2D022C2F272
:105E20000002342110FB012040698047FFE7FFE7B3
:105E300002B080BD80B582B001900198FDF766FB8D
:105E40008DF803009DF80300032819D0FFE79DF8A3
:105E5000030040F2D022C2F20002342110FB0120E4
:105E6000806860B1FFE79DF8030040F2D022C2F2E3
:105E70000002342110FB012080688047FFE7FFE724
:105E800002B080BD80B582B001900198FDF73EFB65
:105E90008DF803009DF80300032819D0FFE79DF853
:105EA000030040F2D022C2F20002342110FB012094
:105EB000C06A60B1FFE79DF8030040F2D022C2F251
:105EC0000002342110FB0120C06A8047FFE7FFE792
:105ED00002B080BD80B584B002900298806D0190C0
:105EE00000F0B8FD0090029890F8350002280DD01F
:105EF000FFE7029980204865FFE70299002081F8BA
:105F00003400FFE701208DF80F0055E0029801688A
:105F1000086820F01600086002980168486920F0BF
:105F2000800048610298006C20B9FFE70298806CFD
:105F300038B1FFE702980168086820F0080008609F
:105F4000FFE702980168086820F001000860FFE799
:105F5000029800680068C007C8B1FFE700F07AFD4A
:105F60000099401A062811D3FFE7029920204865BE
:105F70000299032081F83500FFE70299002081F89B
:105F80003400FFE703208DF80F0015E0E0E70298EA
:105F9000C16D3F208840019988600299012081F8F5
:105FA0003500FFE70299002081F83400FFE7FFE7A2
:105FB00000208DF80F00FFE79DF80F0004B080BDB2
:105FC00082B00090009890F83500022807D0FFE7D3
:105FD00000998020486501208DF807000EE00099A7
:105FE000052081F8350000980168086820F001005C
:105FF0000860FFE700208DF80700FFE79DF8070025
:1060000002B0704780B586B005900020039040F242
:106010000000C2F20000006848F2B511C1F64E312E
:10602000A0FB0110800A02900598806D01900198F4
:106030000068049004980599C96DC84000070028BD
:106040001AD5FFE70598006800684007002812D5B8
:10605000FFE705980168086820F0040008600598CB
:10606000C16D08208840019988600599486D40F00D
:1060700001004865FFE7FFE704980599C96DC8402E
:10608000C007A0B1FFE70598006840690006002836
:106090000CD5FFE70598C16D012088400199886003
:1060A0000599486D40F002004865FFE7FFE7049856
:1060B0000599C96DC8404007002814D5FFE7059829
:1060C00000680068800700280CD5FFE70598C16DBF
:1060D00004208840019988600599486D40F00400CB
:1060E0004865FFE7FFE704980599C96DC840C006F9
:1060F000002847D5FFE705980068006800070028DA
:106100003FD5FFE70598C16D102088400199886050
:10611000059800680068400300281AD5FFE7059835
:10612000006800680003002809D4FFE70598006CA8
:1061300020B1FFE70598016C8847FFE708E0059864
:10614000806C20B1FFE70598816C8847FFE7FFE787
:1061500016E0059800680068C005002807D4FFE72E
:1061600005980168086820F008000860FFE70598B6
:10617000006C20B1FFE70598016C8847FFE7FFE757
:10618000FFE7FFE704980599C96DC840800600281D
:1061900040F18D80FFE7059800680068C006002880
:1061A00040F18480FFE70598C16D20208840019967
:1061B0008860059890F83500052834D1FFE70598E8
:1061C0000168086820F016000860059801684869B1
:1061D00020F0800048610598006C20B9FFE7059821
:1061E000806C38B1FFE705980168086820F0080066
:1061F0000860FFE70598C16D3F20884001998860DD
:106200000599012081F83500FFE70599002081F804
:106210003400FFE70598006D20B1FFE70598016D98
:106220008847FFE77BE00598006800684003002886
:106230001AD5FFE70598006800680003002809D414
:10624000FFE70598406C20B1FFE70598416C88474F
:10625000FFE708E00598C06B20B1FFE70598C16B28
:106260008847FFE7FFE720E0059800680068C00561
:10627000002811D4FFE705980168086820F0100095
:1062800008600599012081F83500FFE70599002095
:1062900081F83400FFE7FFE70598C06B20B1FFE706
:1062A0000598C16B8847FFE7FFE7FFE7FFE7059821
:1062B000406DA0B3FFE70598406DC00730B3FFE71E
:1062C0000599052081F8350005980168086820F0D7
:1062D00001000860FFE703980130039002998842AB
:1062E00001D9FFE707E0FFE7059800680068C007ED
:1062F0000028F0D1FFE70599012081F83500FFE77C
:106300000599002081F83400FFE7FFE70598C06C8D
:1063100020B1FFE70598C16C8847FFE7FFE706B0AB
:1063200080BD000080B586B004900020039000F08E
:1063300091FB0290049820B9FFE701208DF8170027
:10634000A3E00498406A08B1FFE7FFE70499022040
:1063500081F83500FFE70499002081F83400FFE759
:1063600004980168086820F001000860FFE70498BD
:1063700000680068C00790B1FFE700F06BFB02996E
:10638000401A06280AD3FFE704992020486504999B
:10639000032081F835008DF8170076E0E7E70498D0
:1063A000006800680390039848F23F01CFF21001A3
:1063B00008400390049900914868D1F808C0CB6860
:1063C0000A6940EA0C00184310434A6910438A697D
:1063D0001043CA691043096A0143039808430390B4
:1063E0000498406A042808D1FFE70499C86A096B39
:1063F0000143039808430390FFE703980499096851
:1064000008600498006840690390039820F0070032
:1064100003900498416A0398084303900498406AE3
:1064200004281AD1FFE70498816A0398084303906F
:106430000498C06A80B1FFE70498FDF7DDFF50B112
:10644000FFE70499402048650499012081F8350050
:106450008DF8170019E0FFE7FFE703980499096832
:1064600048610498FDF79CFF01900498C16D3F209E
:10647000884001998860049900204865049A0121A8
:1064800082F835108DF81700FFE79DF8170006B069
:1064900080BD000080B588B00690059104920393FA
:1064A00000208DF80B000698806D0190FFE706989C
:1064B00090F83400012804D1FFE702208DF81F0076
:1064C00045E00699012081F83400FFE7FFE70698D0
:1064D00090F8350001282BD1FFE70699022081F8BA
:1064E000350006990020486506980599049A039B93
:1064F000FDF7FAFF0698C16D3F208840019988603A
:1065000006980168086840F0160008600698006C5C
:1065100038B1FFE706980168086840F00800086095
:10652000FFE706980168086840F00100086009E08C
:10653000FFE70699002081F83400FFE702208DF87C
:106540000B00FFE79DF80B008DF81F00FFE79DF89B
:106550001F0008B080BD000080B584B0039000F03B
:1065600079FA0290039801900198013048B1FFE751
:1065700040F26420C2F200000178019808440190C2
:10658000FFE7FFE700F066FA0299401A0199884296
:1065900001D2FFE7F6E704B080BD000080B582B00D
:1065A000ADF8060000208DF80500FFE79DF8050016
:1065B0000F2824DCFFE7BDF806009DF80510C84051
:1065C000C007A8B1FFE79DF8051040F23830C2F2CD
:1065D000000050F8210050B1FFE79DF8051040F28F
:1065E0003830C2F2000050F821008047FFE7FFE793
:1065F000FFE79DF8050001308DF80500D6E702B0F1
:1066000080BD000080B582B0ADF8060043F61440AE
:10661000C4F201000068BDF8061008420CD0FFE784
:10662000BDF8060043F61441C4F201010860BDF84C
:106630000600FFF7B3FFFFE702B080BD8EB00D90FC
:106640000C9100200A90099008900B90FFE70B989E
:106650000F2800F2CC81FFE70B99012088400A90B7
:106660000C9800680A990840099009980A9988428C
:1066700040F0B881FFE70C98406800F00300012863
:1066800007D0FFE70C98406800F0030002282FD1E4
:10669000FFE70D98806808900B984100032000FAEE
:1066A00001F10898884308900C98C0680B9949003C
:1066B00000FA01F108980843089008980D9988603D
:1066C0000D98406808900B99012000FA01F1089894
:1066D000884308900C984068C0F300100B9900FAAA
:1066E00001F108980843089008980D994860FFE761
:1066F0000C98406800F00300032818D0FFE70D98BD
:10670000C06808900B984100032000FA01F1089836
:10671000884308900C9880680B99490000FA01F1B1
:1067200008980843089008980D99C860FFE70C98EE
:10673000406800F00300022826D1FFE70D980B996E
:106740006FF0030202EA51010844006A08900B98B6
:1067500000F0070081000F2000FA01F1089888433B
:1067600008900C9800690B9901F00701890000FA64
:1067700001F108980843089008980D990B9B02EACC
:10678000530211440862FFE70D98006808900B98C7
:106790004100032000FA01F10898884308900C9802
:1067A000406800F003000B99490000FA01F10898D5
:1067B0000843089008980D9908600C988079800724
:1067C000002800F00E81FFE7FFE70020079043F666
:1067D0004400C4F20200016841F480410160006895
:1067E00000F4804007900798FFE70B9820F0030023
:1067F00043F60801C4F20101405808900B9800F0DC
:10680000030081000F2000FA01F1089888430890E6
:106810000D980021C4F20201884203D1FFE7002055
:1068200006905EE00D9840F20041C4F202018842F9
:1068300003D1FFE70120059050E00D9840F60001DC
:10684000C4F20201884203D1FFE70220049042E033
:106850000D9840F60041C4F20201884203D1FFE7DF
:106860000320039034E00D9841F20001C4F20201CC
:10687000884203D1FFE70420029026E00D9841F200
:106880000041C4F20201884203D1FFE705200190D4
:1068900018E00D9841F60001C4F20201884203D1CC
:1068A000FFE7062000900AE00D9941F60042C4F28D
:1068B00002020820914208BF07200090FFE70098DD
:1068C0000190FFE701980290FFE702980390FFE72D
:1068D00003980490FFE704980590FFE70598069059
:1068E000FFE70698C0B20B9901F00301890000FA96
:1068F00001F108980843089008980B9921F00301CA
:1069000043F60802C4F20102885043F60840C4F27C
:1069100001000068089009990898884308900C982D
:106920008079C006002805D5FFE709990898084333
:106930000890FFE7089843F60841C4F20101086097
:1069400043F60C40C4F201000068089009990898C9
:10695000884308900C9880798006002805D5FFE7C9
:106960000999089808430890FFE7089843F60C41F6
:10697000C4F20101086043F60440C4F2010000685B
:10698000089009990898884308900C9880798007A6
:10699000002805D5FFE70999089808430890FFE704
:1069A000089843F60441C4F20101086043F6004030
:1069B000C4F201000068089009990898884308907B
:1069C0000C988079C00728B1FFE709990898084317
:1069D0000890FFE7089843F60041C4F201010860FF
:1069E000FFE7FFE7FFE70B9801300B902FE60EB0B3
:1069F0007047000082B00190ADF802100198006964
:106A0000BDF80210084204D0FFE701208DF8010014
:106A100003E000208DF80100FFE79DF8010002B0BF
:106A20007047000082B00190ADF802108DF801208F
:106A30009DF8010028B1FFE7BDF8020001998861C7
:106A400005E0BDF80200000401998861FFE702B08B
:106A50007047000047F6C870C2F200000068704737
:106A600080B58EB00C900C9820B9FFE701208DF80E
:106A7000370043E10C9890F83D0040B9FFE70C99CE
:106A8000002081F83C000C9800F03CF9FFE70C99DD
:106A9000242081F83D000C980168086820F001006E
:106AA00008600C980168086840F4004008600C9881
:106AB0000168086820F40040086000F0BDFB0A90FF
:106AC0000C98406848F2A061C0F2010188420BD8DE
:106AD000FFE70A9948F28042C0F21E02002091426C
:106AE00038BF012009900AE00A9940F60012C0F26E
:106AF0003D020020914238BF01200990FFE709982C
:106B0000012804D1FFE701208DF83700F6E00A984C
:106B10004DF68361C4F21B31A0FB0110800C0B9079
:106B20000C980068406820F03F000B9908430C99CE
:106B3000096848600C980068006A20F03F000890DF
:106B40000C98406848F2A061C0F20101884204D864
:106B5000FFE70B98013007900EE00B984FF4967109
:106B6000484344F6D351C1F26201A0FB0101012068
:106B700000EB91100790FFE70898079908430C99DC
:106B8000096808620C980068C0694CF6FF71884378
:106B900006900C98406848F2A061C0F2010188425A
:106BA0001FD8FFE70A9801380C9949684900B0FBE3
:106BB000F1F001306FF31F30032803D8FFE7042002
:106BC00005900BE00A9801380C9949684900B0FB20
:106BD000F1F001306FF31F300590FFE70598049046
:106BE0004CE00C98806868B9FFE70A9801380C9966
:106BF000496801EB4101B0FBF1F001306FF31F3048
:106C000003900DE00A9801380C9949681922514304
:106C1000B0FBF1F00130042161F31F300390FFE776
:106C20000398000518B9FFE70120029023E00C98B3
:106C3000806868B9FFE70A9801380C99496801EB48
:106C40004101B0FBF1F001306FF31F3001900DE016
:106C50000A9801380C99496819225143B0FBF1F0A8
:106C60000130042161F31F300190FFE7019840F4E7
:106C700000400290FFE702980490FFE7069804990D
:106C800008430C990968C8610C980068006820F0F6
:106C9000C0000C9B1968DA691B6A1A43104308602C
:106CA0000C980068806848F2FF3188430C9A11689C
:106CB000D36812691A43104388600C980068C06852
:106CC00020F0FF000C9B19685A699B691A43104316
:106CD000C8600C980168086840F0010008600C99D1
:106CE000002008640C9A202182F83D100C9908635A
:106CF0000C9981F83E008DF83700FFE79DF83700CA
:106D00000EB080BD80B590B00F9000200E900D9019
:106D10000C900B900A900F98006845F60041C4F261
:106D20000001884240F08980FFE7FFE700200990DA
:106D300043F63000C4F20200016841F00401016032
:106D4000006800F0040009900998FFE7FFE70020C1
:106D5000089043F63000C4F20200016841F00101DE
:106D60000160006800F0010008900898FFE74FF408
:106D700000700A90122002900B90002003900C905B
:106D8000032004900D90042005900E9040F6000022
:106D9000C4F202000AA90691FFF750FCDDF808C012
:106DA000039B049A059806994FF4807ECDF828E05D
:106DB000CDF82CC00C930D920E900020C4F202006E
:106DC000FFF73CFCFFE70020079043F64000C4F2C9
:106DD0000200016841F400010160006800F4000055
:106DE00007900798FFE740F28470C2F2000001901C
:106DF00046F24001C4F2020101604FF0C0614160FF
:106E000000218160C1604FF4806202614161816153
:106E1000C16101624162FFF785FA18B1FFE7FDF732
:106E2000A5FBFFE7FFE70F9840F28471C2F2000173
:106E300081630F988863FFE7FFE710B080BD000013
:106E400040F26420C2F20000027847F6C871C2F234
:106E500000010868104408607047000080B543F6E0
:106E60000041C4F20201086840F40070086008683C
:106E700040F480600860086840F480700860032077
:106E800000F09AF80F2000F005F800F03BF8002021
:106E900080BD000080B582B0009040F20000C2F2D8
:106EA0000000006840F26421C2F200010A784FF449
:106EB0007A71B1FBF2F1B0FBF1F001F0F3FE20B119
:106EC000FFE701208DF8070018E000980F280DD883
:106ED000FFE700994FF0FF30002200F053F80098D0
:106EE00040F26821C2F20001086003E001208DF841
:106EF000070003E000208DF80700FFE79DF807007A
:106F000002B080BD80B582B0FFE70020019043F65B
:106F10004400C4F20200016841F48041016000684D
:106F200000F4804001900198FFE7FFE70020009007
:106F300043F64000C4F20200016841F08051016054
:106F4000006800F0805000900098FFE76FF00100AB
:106F50000F21002200F016F802B080BD80B582B08B
:106F60008DF807009DF9070008F0F0F902B080BD28
:106F700080B582B08DF807009DF9070008F002FA8D
:106F800002B080BD80B586B08DF8170004910392E1
:106F90000020029008F00EFA02909DF9170001906F
:106FA00002980499039A04F09DFD0146019808F0A7
:106FB00009FA06B080BD000080B582B0019001984A
:106FC00008F044FA02B080BD80B584B0029001910F
:106FD000029820B9FFE701208DF80F0021E1019808
:106FE00043F60041C4F20201096801F0070188423A
:106FF00012D9FFE7019943F60040C4F20200017084
:10700000006800F007000199884204D0FFE70120E2
:107010008DF80F0005E1FFE702980078800700284F
:107020002AD5FFE7029800784007002809D5FFE736
:1070300043F60801C4F20201086840F4E050086019
:10704000FFE7029800780007002809D5FFE743F61C
:107050000801C4F20201086840F460400860FFE7DC
:1070600043F60801C4F20201086820F0F000029A19
:10707000926810430860FFE702980078C007002874
:107080006ED0FFE702984068012811D1FFE743F670
:107090000000C4F20200006800F400310020B0EBF0
:1070A000514F04D1FFE701208DF80F00B9E02CE02B
:1070B00002984068022805D0FFE70298406803283C
:1070C00011D1FFE743F60000C4F20200006800F0AF
:1070D00000710020B0EB516F04D1FFE701208DF863
:1070E0000F009EE010E043F60000C4F202000068CA
:1070F00000F002010020B0EB510F04D1FFE70120A6
:107100008DF80F008DE0FFE7FFE743F60801C4F2BA
:107110000201086820F00300029A526810430860D8
:10712000FFF798FC0090FFE743F60800C4F2020066
:10713000006800F00C0002994968B0EB810F0ED096
:10714000FFE7FFF787FC0099401A41F28931884236
:1071500004D3FFE703208DF80F0062E0E4E7FFE7C8
:10716000019843F60041C4F20201096801F00701E9
:10717000884212D2FFE7019943F60040C4F20200B0
:107180000170006800F007000199884204D0FFE711
:1071900001208DF80F0044E0FFE7029800784007D7
:1071A00000280CD5FFE743F60801C4F20201086885
:1071B00020F4E050029AD26810430860FFE702987A
:1071C0000078000700280DD5FFE743F60801C4F258
:1071D0000201086820F46040029A126940EAC20085
:1071E0000860FFE700F04CF843F60801C4F2020122
:1071F0000968C9B20A0946F2C011C0F60101895CEA
:10720000C84040F20001C2F20001086040F268206C
:10721000C2F200000068FFF73DFE00208DF80F006D
:10722000FFE79DF80F0004B080BD000040F20000B1
:10723000C2F200000068704780B5FFF7F7FF43F621
:107240000801C4F202010968C1F3822246F2D0119A
:10725000C0F60101895CC84080BD000080B5FFF721
:10726000E5FF43F60801C4F20201096889B24A0B3E
:1072700046F2D011C0F60101895CC84080BD000013
:1072800080B586B00020059004900390029043F6EC
:107290000800C4F20200006800F00C0001460191F1
:1072A00040B1FFE7019804280AD0FFE701980828B9
:1072B0000CD04FE042F20040C0F2F40002904FE0E8
:1072C00041F60030C0F2B700029049E043F60400F6
:1072D000C4F20200016801F03F010591006840021C
:1072E000002813D5FFE743F60400C4F2020000684B
:1072F000C0F3881041F60031C0F2B701A0FB0101D4
:10730000059A0023F8F7D0FF049012E043F604003A
:10731000C4F202000068C0F3881042F20041C0F2DB
:10732000F401A0FB0101059A0023F8F7BDFF0490CA
:10733000FFE743F60400C4F20200006800F44031A5
:10734000022000EBD130039004980399B0FBF1F0D8
:10735000029005E042F20040C0F2F4000290FFE724
:10736000029806B080BD000080B586B004900498F5
:1073700020B9FFE701208DF8170050E3049800784A
:10738000C007002800F0A580FFE743F60800C4F21C
:107390000200006800F00C00042813D0FFE743F659
:1073A0000800C4F20200006800F00C0008281ED19A
:1073B000FFE743F60400C4F2020000684002002820
:1073C00015D5FFE743F60000C4F20200006800F4A0
:1073D00000310020B0EB514F08D0FFE7049840681F
:1073E00020B9FFE701208DF8170018E370E0FFE7F0
:1073F00004984068B0F5803F09D1FFE743F60001EB
:10740000C4F20201086840F48030086020E004986B
:107410004068B0F5A02F0DD1FFE743F60001C4F29C
:107420000201086840F480200860086840F4803059
:1074300008600CE043F60001C4F20201086820F481
:1074400080300860086820F480200860FFE7FFE7CC
:10745000FFE704984068E8B1FFE7FFF7FBFA039005
:10746000FFE743F60000C4F20200006800F40031B8
:107470000020B0EB514F0CD1FFE7FFF7EBFA039977
:10748000401A652804D3FFE703208DF81700C6E2F1
:10749000E7E71CE0FFF7DEFA0390FFE743F60000A2
:1074A000C4F20200006800F400310020B0EB514F3C
:1074B0000CD0FFE7FFF7CEFA0399401A652804D3F2
:1074C000FFE703208DF81700A9E2E7E7FFE7FFE7F2
:1074D000FFE7049800788007002840F19680FFE7D6
:1074E00043F60800C4F20200006810F00C0F13D03D
:1074F000FFE743F60800C4F20200006800F00C0049
:1075000008282CD1FFE743F60400C4F2020000680B
:107510004002002823D4FFE743F60000C4F2020033
:10752000006800F002010020B0EB510F09D0FFE726
:107530000498C068012804D0FFE701208DF81700E7
:107540006DE243F60001C4F20201086820F0F80081
:10755000049A126940EAC2000860FFE754E0049808
:10756000C06870B3FFE70021C4F247210120086022
:10757000FFF770FA0390FFE743F60000C4F2020041
:10758000006800F002010020B0EB510F0CD1FFE7C2
:10759000FFF760FA0399401A032804D3FFE703209A
:1075A0008DF817003BE2E7E743F60001C4F2020161
:1075B000086820F0F800049A126940EAC2000860E6
:1075C00021E00021C4F2472100200860FFF742FAC1
:1075D0000390FFE743F60000C4F20200006800F0E9
:1075E00002010020B0EB510F0CD0FFE7FFF732FA99
:1075F0000399401A032804D3FFE703208DF81700EE
:107600000DE2E7E7FFE7FFE7FFE7049800780007F0
:1076100000284BD5FFE70498406918B3FFE740F610
:107620008061C4F2472101200860FFF713FA03903C
:10763000FFE743F67400C4F20200006800F00201A4
:107640000020B0EB510F0CD1FFE7FFF703FA0399CD
:10765000401A032804D3FFE703208DF81700DEE16A
:10766000E7E722E040F68061C4F24721002008608D
:10767000FFF7F0F90390FFE743F67400C4F202004D
:10768000006800F002010020B0EB510F0CD0FFE7C2
:10769000FFF7E0F90399401A032804D3FFE703201A
:1076A0008DF81700BBE1E7E7FFE7FFE704980078F4
:1076B0004007002840F1CE80FFE700208DF807004A
:1076C00043F64000C4F202000068C000002815D450
:1076D000FFE7FFE70020009043F64000C4F20200FD
:1076E000016841F080510160006800F08050009016
:1076F0000098FFE701208DF80700FFE747F2000040
:10770000C4F200000068C005002822D4FFE747F259
:107710000001C4F20001086840F480700860FFF7BF
:1077200099F90390FFE747F20000C4F200000068F7
:10773000C00500280CD4FFE7FFF78CF90399401A25
:10774000032804D3FFE703208DF8170067E1EAE779
:10775000FFE7FFE704988068012809D1FFE743F6B7
:107760007001C4F20201086840F0010008601FE0E7
:107770000498806805280DD1FFE743F67001C4F234
:107780000201086840F004000860086840F0010049
:1077900008600CE043F67001C4F20201086820F0B2
:1077A00001000860086820F004000860FFE7FFE7B8
:1077B000FFE704988068F8B1FFE7FFF74BF9039003
:1077C000FFE743F67000C4F20200006800F0020117
:1077D0000020B0EB510F0ED1FFE7FFF73BF9039903
:1077E000401A41F28931884204D3FFE703208DF823
:1077F000170014E1E5E71EE0FFF72CF90390FFE71F
:1078000043F67000C4F20200006800F0020100209C
:10781000B0EB510F0ED0FFE7FFF71CF90399401AA8
:1078200041F28931884204D3FFE703208DF8170025
:10783000F5E0E5E7FFE79DF80700012809D1FFE73C
:1078400043F64001C4F20201086820F0805008604D
:10785000FFE7FFE704988069002800F0DC80FFE77D
:1078600043F60800C4F20200006800F00C0008288B
:1078700000F08580FFE70498806902285CD1FFE76B
:107880006021C4F2472100200860FFF7E3F803906D
:10789000FFE743F60000C4F20200006800F0007148
:1078A0000020B0EB516F0CD0FFE7FFF7D3F803993E
:1078B000401A032804D3FFE703208DF81700AEE039
:1078C000E7E70499C869D1F820C04B6A8A6A40EAA0
:1078D0000C0040EA8310D2034FF6FF739A43A2F5DF
:1078E00080321043C96A40EA016043F60401C4F2E1
:1078F000020108606021C4F2472101200860FFF7FF
:10790000A9F80390FFE743F60000C4F20200006804
:1079100000F000710020B0EB516F0CD1FFE7FFF7D2
:1079200099F80399401A032804D3FFE703208DF840
:10793000170074E0E7E721E06021C4F2472100204E
:107940000860FFF787F80390FFE743F60000C4F2F2
:107950000200006800F000710020B0EB516F0CD005
:10796000FFE7FFF777F80399401A032804D3FFE7EE
:1079700003208DF8170052E0E7E7FFE74AE004989C
:107980008069012804D1FFE701208DF8170046E047
:1079900043F60400C4F20200006802900498806973
:1079A000012831D0FFE7029800F480000499C969EA
:1079B000884229D1FFE7029800F03F000499096A44
:1079C000884221D1FFE7029847F6C0710840049928
:1079D000496AB0EB811F17D1FFE7029800F44030ED
:1079E0000499896AC9034FF6FF729143A1F580316A
:1079F000884209D1FFE7029800F070600499C96AD3
:107A0000B0EB016F04D0FFE701208DF8170006E00E
:107A1000FFE7FFE7FFE700208DF81700FFE79DF87D
:107A2000170006B080BD000080B582B001900198BB
:107A300004F040FD8DF803009DF8030002281BD0E0
:107A4000FFE7019804F036FD014640F28030C2F2B3
:107A5000000000EB4110806968B1FFE7019804F075
:107A600029FD014640F28030C2F2000000EB4110D7
:107A700080698047FFE7FFE702B080BD80B584B032
:107A80000290029820B9FFE701208DF80F0071E005
:107A90000298406A60B9FFE702984068B0F5827FBB
:107AA00001D1FFE703E002990020C861FFE705E08C
:107AB00002990020086102994861FFE702990020BD
:107AC0008862029890F8510040B9FFE702990020BF
:107AD00081F85000029800F051F8FFE70299022067
:107AE00081F8510002980168086820F040000860A1
:107AF000029A019211685068D2F808C0D36800F465
:107B000082700CF4044C604403F40063184413695D
:107B100003F002031844536903F001031844936906
:107B200003F400731844D36903F038031844136A4C
:107B300003F080031843926A02F400521043086075
:107B4000029A508B00F004001168526A02F0100291
:107B50001044486002980168C86920F40060C86158
:107B6000029900204865029A012182F851108DF88F
:107B70000F00FFE79DF80F0004B080BD80B590B006
:107B80000F9000200E900D900C900B900A900F9883
:107B9000006843F20001C4F20101884240F0B28063
:107BA000FFE7FFE70020099043F64400C4F202001B
:107BB000016841F480510160006800F48050099030
:107BC0000998FFE7FFE70020089043F63000C4F271
:107BD0000200016841F002010160006800F002004B
:107BE00008900898FFE7FFE70020079043F6300071
:107BF000C4F20200016841F001010160006800F078
:107C0000010007900798FFE718200A9002200190D2
:107C10000B90002005900C90032002900D90052001
:107C200003900E9040F20040C4F202000AA90491B1
:107C3000FEF704FDDDF804C0029A03980499059B41
:107C40004FF0800ECDF828E0CDF82CC00C930D92AB
:107C50000E900020C4F20200FEF7F0FC059940F2FD
:107C6000E470C2F20000069046F24042C4F2020202
:107C700002604FF0C06242608160C1604FF4806278
:107C8000026141618161C16101624162FEF74AFBAB
:107C900018B1FFE7FCF76AFCFFE7FFE70F9840F237
:107CA000E471C2F20001C1640F988863FFE740F6F7
:107CB0004400C2F20000009046F25841C4F20201B2
:107CC00001604FF0C0614160402181600021C160CE
:107CD0004FF48062026141618161C1610162416270
:107CE000FEF720FB18B1FFE7FCF740FCFFE7FFE7DA
:107CF0000F9840F64401C2F2000181640F98886336
:107D0000FFE7FFE710B080BD80B588B00690059111
:107D1000ADF812200393069890F85100012804D082
:107D2000FFE702208DF81F0011E1059820B1FFE761
:107D3000BDF8120020B9FFE701208DF81F0006E111
:107D400006984068B0F5827F16D1FFE706988068F4
:107D500090B9FFE70699042081F851000698059A2A
:107D6000BDF812300399EC46CCF80010114600F033
:107D700065FB8DF81F00EAE0FEF76CFE0290FFE75E
:107D8000069890F85000012804D1FFE702208DF8F2
:107D90001F00DCE00699012081F85000FFE7FFE7B3
:107DA0000699042081F8510006990020486505993C
:107DB000069A9163BDF81210069A9187BDF81210C9
:107DC000069AD18706990863069988860699C88617
:107DD000069908640699486406988068B0F5004FD3
:107DE0000DD1FFE706980168086820F040000860A0
:107DF00006980168086820F480400860FFE706984C
:107E00000068006800F04000402807D0FFE70698AF
:107E10000168086840F040000860FFE70698C06805
:107E2000D0BBFFE7FFE70698C08FA0B3FFE7069837
:107E300000688068C00778B1FFE706980068007B9B
:107E40000699896B08700699886B013088630699DA
:107E5000C88F0138C8871DE0FEF7FCFD0299401A63
:107E60000399884204D3FFE70398013018B9FFE76C
:107E7000039870B9FFE70699012081F85100FFE7E8
:107E80000699002081F85000FFE703208DF81F00BD
:107E90005DE0FFE7C7E739E0FFE70698C08FA0B3D2
:107EA000FFE7069800688068C00778B1FFE706988A
:107EB0000068C0680699896B08800699886B023053
:107EC00088630699C88F0138C8871DE0FEF7C2FD98
:107ED0000299401A0399884204D3FFE703980130BE
:107EE00018B9FFE7039870B9FFE70699012081F8F8
:107EF0005100FFE70699002081F85000FFE70320BA
:107F00008DF81F0023E0FFE7C7E7FFE70698039916
:107F1000029A04F0F7F920B1FFE70699202048659E
:107F2000FFE70699012081F85100FFE7069900203C
:107F300081F85000FFE70698406D20B1FFE701206F
:107F40008DF81F0003E000208DF81F00FFE79DF86B
:107F50001F0008B080BD000080B584B00290019180
:107F6000ADF80220029890F85100012804D0FFE7F4
:107F700002208DF80F00B7E0019820B1FFE7BDF8AF
:107F8000020020B9FFE701208DF80F00ACE0029855
:107F90008068A0B9FFE702984068B0F5827F0ED1F3
:107FA000FFE70299042081F851000298019ABDF878
:107FB0000230114600F014FC8DF80F0094E0FFE74A
:107FC000029890F85000012804D1FFE702208DF8B4
:107FD0000F0089E00299012081F85000FFE7FFE7D8
:107FE0000299042081F85100029900204865019906
:107FF000029A9163BDF80210029A9187BDF80210AF
:10800000029AD18702990864029948640299888685
:108010000299C88602988068B0F5004F0DD1FFE73D
:1080200002980168086820F0400008600298016822
:10803000086820F480400860FFE70298C16C4CF2A9
:10804000E900C0F6000008640298C16C4CF23110DF
:10805000C0F60000C8630298C16C4CF2B500C0F6CF
:108060000000C8640298C16C00200865029B196872
:108070009A6BD86C0C31DB8FFEF70CFA78B1FFE706
:108080000299486D40F010004865FFE70299002012
:1080900081F85000FFE701208DF80F0024E00298DE
:1080A0000068006800F04000402807D0FFE7029811
:1080B0000168086840F040000860FFE7FFE70299A8
:1080C000002081F85000FFE702980168486840F0FE
:1080D0002000486002980168486840F0010048604C
:1080E00000208DF80F00FFE79DF80F0004B080BD61
:1080F00080B582B00190019804F0DCF98DF803009E
:108100009DF8030002281BD0FFE7019804F0D2F984
:10811000014640F28030C2F2000000EB411040689E
:1081200068B1FFE7019804F0C5F9014640F28030DC
:10813000C2F2000000EB411040688047FFE7FFE714
:1081400002B080BD80B582B00190019804F0B2F910
:108150008DF803009DF8030002281BD0FFE701986B
:1081600004F0A8F9014640F28030C2F2000000EBB2
:108170004110006968B1FFE7019804F09BF90146DE
:1081800040F28030C2F2000000EB411000698047ED
:10819000FFE7FFE702B080BD80B588B0069005918B
:1081A000ADF812200393FEF755FC0290BDF81200C3
:1081B000ADF80600069890F85100012804D0FFE7BA
:1081C00002208DF81F0034E1059820B1FFE7BDF8CB
:1081D000120020B9FFE701208DF81F0029E1FFE719
:1081E000069890F85000012804D1FFE702208DF88E
:1081F0001F001EE10699012081F85000FFE7FFE70C
:108200000699032081F851000699002048650599D8
:10821000069A1163BDF81210069A9186BDF81210E5
:10822000069AD18606998863069988870699C88731
:10823000069948640699086406988068B0F5004F6E
:108240000DD1FFE706980168086820F0400008603B
:1082500006980168086840F480400860FFE70698C7
:108260000068006800F04000402807D0FFE706984B
:108270000168086840F040000860FFE70698C068A1
:10828000B0F5006F51D1FFE70698406828B1FFE7CD
:10829000BDF8060001280ED1FFE706980168006BC3
:1082A0000088C8600699086B023008630699C88E7A
:1082B0000138C886FFE7FFE70698C08EA0B3FFE746
:1082C000069800688068800700280ED5FFE70698AA
:1082D0000168006B0088C8600699086B023008636B
:1082E0000699C88E0138C8861DE0FEF7B3FB0299D7
:1082F000401A0399884204D3FFE70398013018B964
:10830000FFE7039870B9FFE70699012081F8510053
:10831000FFE70699002081F85000FFE703208DF861
:108320001F0086E0FFE7C7E750E00698406828B1E5
:10833000FFE7BDF8060001280ED1FFE706980168A7
:10834000006B007808730699086B01300863069982
:10835000C88E0138C886FFE7FFE70698C08EA0B335
:10836000FFE7069800688068800700280ED5FFE7C1
:1083700006980168006B007808730699086B013055
:1083800008630699C88E0138C8861DE0FEF762FBB7
:108390000299401A0399884204D3FFE703980130F9
:1083A00018B9FFE7039870B9FFE70699012081F833
:1083B0005100FFE70699002081F85000FFE70320F5
:1083C0008DF81F0035E0FFE7C7E7FFE70698039940
:1083D000029A04F009F820B1FFE7069920204865C9
:1083E000FFE70698806870B9FFE7FFE7002000907C
:1083F00006980068C0680090069800688068009041
:108400000098FFE7FFE70699012081F85100FFE798
:108410000699002081F85000FFE70698406D20B1D2
:10842000FFE701208DF81F0003E000208DF81F00FA
:10843000FFE79DF81F0008B080BD000080B58CB03C
:10844000DDF838C00A9009910892ADF81E3001207D
:108450000390FEF7FFFA04900A9890F851008DF807
:1084600017000A9840680690BDF81E00ADF81C0081
:108470009DF81700012812D0FFE70698B0F5827F1B
:1084800009D1FFE70A98806828B9FFE79DF817002F
:10849000042804D0FFE702208DF82F009BE1099803
:1084A00038B1FFE7089820B1FFE7BDF81E0020B9FA
:1084B000FFE701208DF82F008DE1FFE70A9890F883
:1084C0005000012804D1FFE702208DF82F0082E13F
:1084D0000A99012081F85000FFE7FFE70A9890F819
:1084E0005100042805D0FFE70A99052081F85100C2
:1084F000FFE70A990020486508990A9A9163BDF838
:108500001E100A9AD187BDF81E100A9A9187099900
:108510000A9A1163BDF81E100A9AD186BDF81E1082
:108520000A9A91860A9908640A9948640A98006828
:10853000006800F04000402807D0FFE70A98016873
:10854000086840F040000860FFE70A98C068B0F58E
:10855000006F40F08180FFE70A98406828B1FFE78C
:10856000BDF81C0001280ED1FFE70A980168006BD6
:108570000088C8600A99086B023008630A99C88E9F
:108580000138C886FFE7FFE70A98C18E01200190F5
:1085900039B9FFE70A98C08F002818BF0120019061
:1085A000FFE70198C007002855D0FFE70A98006848
:1085B00080688007002818D5FFE70A98C08EA0B110
:1085C000FFE70398012810D1FFE70A980168006BC4
:1085D0000088C8600A99086B023008630A99C88E3F
:1085E0000138C88600200390FFE70A980068806879
:1085F000C007A8B1FFE70A98C08F88B1FFE70A98C3
:108600000068C0680A99896B08800A99886B0230F3
:1086100088630A99C88F0138C88701200390FFE753
:10862000FEF718FA0499401A0E99884212D3FFE710
:108630000E98013070B1FFE70A99012081F85100CE
:10864000FFE70A99002081F85000FFE703208DF82A
:108650002F00C0E098E782E00A98406828B1FFE761
:10866000BDF81C0001280ED1FFE70A980168006BD5
:10867000007808730A99086B013008630A99C88E5C
:108680000138C886FFE7FFE70A98C18E01200090F5
:1086900039B9FFE70A98C08F002818BF0120009061
:1086A000FFE70098C007002858D0FFE70A98006845
:1086B00080688007002818D5FFE70A98C08EA0B10F
:1086C000FFE70398012810D1FFE70A980168006BC3
:1086D000007808730A99086B013008630A99C88EFC
:1086E0000138C88600200390FFE70A980068806878
:1086F000C007A8B1FFE70A98C08F88B1FFE70A98C2
:108700000068C0680A99896B08700A99886B013003
:1087100088630A99C88F0138C88701200390FFE752
:10872000FEF798F90499401A0E99884204D3FFE79E
:108730000E98013018B9FFE70E9870B9FFE70A9953
:10874000012081F85100FFE70A99002081F85000CC
:10875000FFE703208DF82F003DE095E7FFE70A983B
:108760000E99049A03F040FE68B1FFE70A992020B1
:108770004865FFE70A99002081F85000FFE70120D3
:108780008DF82F0027E00A98806870B9FFE7FFE7AF
:10879000002002900A980068C06802900A98006859
:1087A000806802900298FFE7FFE70A99012081F8AC
:1087B0005100FFE70A99002081F85000FFE70A986E
:1087C000406D20B1FFE701208DF82F0003E000206D
:1087D0008DF82F00FFE79DF82F000CB080BD000042
:1087E00080B588B0069005910492ADF80E300698D9
:1087F00090F851008DF807000698406802909DF8A7
:108800000700012812D0FFE70298B0F5827F09D156
:10881000FFE70698806828B9FFE79DF8070004285D
:1088200004D0FFE702208DF81F00DFE0059838B183
:10883000FFE7049820B1FFE7BDF80E0020B9FFE77D
:1088400001208DF81F00D1E0FFE7069890F8500056
:10885000012804D1FFE702208DF81F00C6E0069929
:10886000012081F85000FFE7FFE7069890F85100DB
:10887000042805D0FFE70699052081F85100FFE79D
:108880000699002048650599069A1163BDF80E10F7
:10889000069A9186BDF80E10069AD1860499069A1A
:1088A0009163BDF80E10069A9187BDF80E10069AD6
:1088B000D1870699086406994864069890F8510093
:1088C00004280FD1FFE70698C16C4CF2E900C0F60E
:1088D000000008640698C16C4CF23110C0F600002C
:1088E000C8630EE00698C16C4CF21910C0F6000087
:1088F00008640698C16C4CF27D20C0F60000C86385
:10890000FFE70698C16C4CF2B500C0F60000C864E1
:108910000698C16C00200865069B19689A6BD86C94
:108920000C31DB8FFDF7B6FD78B1FFE70699486D96
:1089300040F010004865FFE70699002081F85000DC
:10894000FFE701208DF81F0050E006980168486895
:1089500040F0010048600698816C00200864069988
:10896000896CC8630699896CC8640699896C086526
:10897000069B1A68196B986C0C32DB8EFDF78AFD2A
:1089800078B1FFE70699486D40F010004865FFE7B1
:108990000699002081F85000FFE701208DF81F00A4
:1089A00024E006980068006800F04000402807D0E6
:1089B000FFE706980168086840F040000860FFE79C
:1089C000FFE70699002081F85000FFE7069801684C
:1089D000486840F02000486006980168486840F008
:1089E0000200486000208DF81F00FFE79DF81F007F
:1089F00008B080BD80B584B002900191ADF802202E
:108A0000029890F85100012804D0FFE702208DF869
:108A10000F00A1E0019820B1FFE7BDF8020020B9E6
:108A2000FFE701208DF80F0096E0FFE7029890F82D
:108A30005000012804D1FFE702208DF80F008BE0E1
:108A40000299012081F85000FFE7FFE70299032017
:108A500081F851000299002048650199029A11633A
:108A6000BDF80210029A9186BDF80210029AD186D2
:108A70000299886302994864029908640299888778
:108A80000299C88702988068B0F5004F0DD1FFE7C2
:108A900002980168086820F04000086002980168A8
:108AA000086840F480400860FFE70298816C4CF24F
:108AB0000110C0F6000008640298816C4CF2D510D9
:108AC000C0F60000C8630298816C4CF2B500C0F695
:108AD0000000C8640298816C00200865029B1A6837
:108AE000196B986C0C32DB8EFDF7D4FC78B1FFE784
:108AF0000299486D40F010004865FFE70299002098
:108B000081F85000FFE701208DF80F0024E0029863
:108B10000068006800F04000402807D0FFE7029896
:108B20000168086840F040000860FFE7FFE702992D
:108B3000002081F85000FFE702980168486840F083
:108B40002000486002980168486840F002004860D0
:108B500000208DF80F00FFE79DF80F0004B080BDE6
:108B600080B582B00190019803F0A4FC8DF8030059
:108B70009DF80300022815D0FFE79DF8030041018E
:108B800040F28030C2F20000405850B1FFE79DF83B
:108B90000300410140F28030C2F20000405880479B
:108BA000FFE7FFE702B080BD80B582B00190019879
:108BB00003F080FC8DF803009DF8030002281BD011
:108BC000FFE7019803F076FC014640F28030C2F2E4
:108BD000000000EB4110C06868B1FFE7019803F0A6
:108BE00069FC014640F28030C2F2000000EB411007
:108BF000C0688047FFE7FFE702B080BD80B582B064
:108C00000190019803F056FC8DF803009DF80300D5
:108C100002281BD0FFE7019803F04CFC014640F20C
:108C20008030C2F2000000EB4110806868B1FFE7BD
:108C3000019803F03FFC014640F28030C2F2000090
:108C400000EB411080688047FFE7FFE702B080BD7E
:108C500080B582B00190019803F02CFC8DF80300E0
:108C60009DF8030002281BD0FFE7019803F022FCC7
:108C7000014640F28030C2F2000000EB4110406932
:108C800068B1FFE7019803F015FC014640F280301F
:108C9000C2F2000000EB411040698047FFE7FFE7A8
:108CA00002B080BD80B582B00190019804F050FE02
:108CB00002B080BD85B003900291FFE7039890F861
:108CC0003C00012804D1FFE702208DF813007EE06C
:108CD0000399012081F83C00FFE7FFE70399022098
:108CE00081F83D000398006840680190039800688F
:108CF00080680090019820F070000190029801684F
:108D00000198084301900198039909684860039805
:108D100000680021C4F2010188423CD0FFE70398BB
:108D20000068B0F1804F36D0FFE70398006840F24A
:108D30000041C4F2000188422DD0FFE7039800688B
:108D400040F60001C4F20001884224D0FFE70398F6
:108D5000006840F60041C4F2000188421BD0FFE7E2
:108D60000398006840F20041C4F20101884212D029
:108D7000FFE70398006844F20001C4F20101884251
:108D800009D0FFE70398006841F60001C4F2000132
:108D900088420ED1FFE7009820F0800000900298F2
:108DA000416800980843009000980399096888601A
:108DB000FFE70399012081F83D00FFE703990020B8
:108DC00081F83C00FFE700208DF81300FFE79DF8D5
:108DD000130005B07047000080B582B00090009885
:108DE00020B9FFE701208DF807003FE0009890F8D8
:108DF0003D0040B9FFE70099002081F83C00009851
:108E000000F038F8FFE70099022081F83D00009952
:108E100051F8040B04F03AFE0099012081F8460055
:108E2000FFE70099012081F83E00009981F83F009A
:108E3000009981F84000009981F84100FFE7FFE7C1
:108E40000099012081F84200009981F843000099BF
:108E500081F84400009981F84500FFE7009901205E
:108E600081F83D0000208DF80700FFE79DF807001E
:108E700002B080BD83B002900298006840F60041C5
:108E8000C4F20001884212D1FFE7FFE70020019001
:108E900043F64000C4F20200016841F0080101609D
:108EA000006800F0080001900198FFE71BE00298BD
:108EB000006844F20041C4F20101884212D1FFE788
:108EC000FFE70020009043F64400C4F2020001686E
:108ED00041F400310160006800F400300090009817
:108EE000FFE7FFE7FFE703B07047000080B586B0FB
:108EF0000490039100208DF80B00FFE7049890F890
:108F00003C00012804D1FFE702208DF81700ABE0F8
:108F10000499012081F83C00FFE7FFE70499022053
:108F200081F83D000498006880680190019820F065
:108F300077000190019820F47F40019001980499F6
:108F400009688860039800680090002872D0FFE7E5
:108F5000009810286ED0FFE7009820286AD0FFE71D
:108F60000098302866D0FFE70098402855D0FFE7EA
:108F70000098502837D0FFE70098602840D0FFE7DE
:108F8000009870280BD0FFE70098B0F5805F05D0FF
:108F9000FFE70098B0F5005F16D052E055E0049866
:108FA0000068039B5A689968DB6804F05DFE0498CA
:108FB000006880680190019840F077000190019866
:108FC00004990968886040E004980068039B5A6827
:108FD0009968DB6804F048FE04980168886840F4EA
:108FE0008040886031E004980068039A5168D26834
:108FF00005F026F804980068502104F04FFE24E0A4
:1090000004980068039A5168D26805F041F8049802
:109010000068602104F042FE17E004980068039A9B
:109020005168D26805F00CF804980068402104F0FB
:1090300035FE0AE0049800680399096804F02EFEE2
:1090400003E001208DF80B00FFE70499012081F86F
:109050003D00FFE70499002081F83C00FFE79DF800
:109060000B008DF81700FFE79DF8170006B080BDD4
:1090700080B58AB00990002008900790069005906E
:1090800004900998006840F60001C4F2000188428B
:1090900023D1FFE7FFE70020039043F63000C4F23E
:1090A0000200016841F008010160006800F008005A
:1090B00003900398FFE74FF480400490022005904E
:1090C0000121069103210791089040F60040C4F267
:1090D000020004A9FDF7B2FA56E00998006840F6CC
:1090E0000041C4F20001884222D1FFE7FFE70020DF
:1090F000029043F63000C4F20200016841F08001A2
:109100000160006800F0800002900298FFE74FF4D1
:10911000E0500490022005900121069107900890EC
:1091200041F60040C4F2020004A9FDF787FA2AE0E4
:109130000998006844F20041C4F20101884221D13B
:10914000FFE7FFE70020019043F63000C4F2020081
:10915000016841F020010160006800F020000190EA
:109160000198FFE7402004900220059006900790A8
:109170000320089041F20040C4F2020004A9FDF768
:109180005DFAFFE7FFE7FFE70AB080BD80B586B074
:1091900004900391029200208DF80700FFE70498E5
:1091A00090F83C00012804D1FFE702208DF8170059
:1091B00089E00499012081F83C00FFE7FFE702986D
:1091C00000900C2800F270800099DFE801F0076D34
:1091D0006D6D206D6D6D3A6D6D6D53000498006876
:1091E000039904F071FD04980168886940F0080053
:1091F000886104980168886920F0040088610398F8
:1092000002690498016888691043886150E00498F5
:109210000068039904F0CEFD04980168886940F461
:109220000060886104980168886920F48060886122
:109230000398026904980168886940EA02208861FD
:1092400036E004980068039904F02EFE0498016843
:10925000C86940F00800C86104980168C86920F036
:109260000400C8610398026904980168C869104342
:10927000C8611DE004980068039904F08FFE04980B
:109280000168C86940F40060C86104980168C86951
:1092900020F48060C8610398026904980168C86975
:1092A00040EA0220C86103E001208DF80700FFE7D3
:1092B000FFE70499002081F83C00FFE79DF80700D4
:1092C0008DF81700FFE79DF8170006B080BD00007D
:1092D00080B582B00090009820B9FFE701208DF89A
:1092E00007003FE0009890F83D0040B9FFE7009983
:1092F000002081F83C00009800F038F8FFE7009962
:10930000022081F83D00009951F8040B04F0BEFBE7
:109310000099012081F84600FFE70099012081F8BB
:109320003E00009981F83F00009981F840000099C3
:1093300081F84100FFE7FFE70099012081F8420032
:10934000009981F84300009981F84400009981F860
:109350004500FFE70099012081F83D0000208DF8CD
:109360000700FFE79DF8070002B080BD82B00190C2
:109370000198006840F60001C4F20001884212D151
:10938000FFE7FFE70020009043F64000C4F2020030
:10939000016841F004010160006800F004000090E1
:1093A0000098FFE7FFE702B07047000080B58CB07F
:1093B0000A900991099828B9FFE70A9890F83E00A9
:1093C00007901CE00998042805D1FFE70A9890F857
:1093D0003F00069010E00998082805D1FFE70A9899
:1093E00090F84000059004E00A9890F8410005903C
:1093F000FFE705980690FFE706980790FFE70798B4
:10940000012804D0FFE701208DF82F00AFE0099874
:1094100028B9FFE70A99022081F83E001EE009986A
:10942000042806D1FFE70A99022081F83F00049042
:1094300012E00998082806D1FFE70A99022081F86E
:109440004000039005E00A99022081F84100039052
:10945000FFE703980490FFE70498FFE70A98006885
:1094600009990122019204F0E3FB01980A99096825
:109470000022C4F20102914202900CD0FFE70A9848
:1094800000684FF60041CBF6FE710844B0FA80F058
:1094900040090290FFE70298C00738B1FFE70A9839
:1094A0000168486C40F400404864FFE70A9800688F
:1094B0000021C4F2010188423CD0FFE70A9800680D
:1094C000B0F1804F36D0FFE70A98006840F20041C3
:1094D000C4F2000188422DD0FFE70A98006840F6E8
:1094E0000001C4F20001884224D0FFE70A98006816
:1094F00040F60041C4F2000188421BD0FFE70A9801
:10950000006840F20041C4F20101884212D0FFE736
:109510000A98006844F20001C4F20101884209D0AF
:10952000FFE70A98006841F60001C4F20001884292
:1095300012D1FFE70A980068806800F007000890E1
:109540000898062807D0FFE70A980168086840F0E5
:1095500001000860FFE706E00A980168086840F02B
:1095600001000860FFE700208DF82F00FFE79DF85D
:109570002F000CB080BD000080B586B0059004912E
:10958000059800680499002204F052FB05980168D0
:1095900001200022C4F20102914203900CD0FFE7A7
:1095A000059800684FF60041CBF6FE710844B0FA0A
:1095B00080F040090390FFE70398C007D8B1FFE7A8
:1095C000FFE705980068006A41F21111084210D1C6
:1095D000FFE705980068006A40F24441084207D15D
:1095E000FFE705980168486C20F400404864FFE7F5
:1095F000FFE7FFE7FFE7FFE705980068006A41F231
:109600001111084210D1FFE705980068006A40F286
:109610004441084207D1FFE705980168086820F037
:1096200001000860FFE7FFE7FFE7049828B9FFE7BC
:109630000599012081F83E001EE00498042806D117
:10964000FFE70599012081F83F00029012E004989D
:10965000082806D1FFE70599012081F84000019014
:1096600005E00599012081F841000190FFE701988C
:109670000290FFE70298FFE7002006B080BD0000DF
:1096800082B00190ADF8021002B0704780B582B090
:109690000190019805F092FB8DF803009DF80300FE
:1096A00003281BD0FFE79DF8030000EBC00140F248
:1096B000A430C2F2000000EB8100006968B1FFE74E
:1096C0009DF8030000EBC00140F2A430C2F200009C
:1096D00000EB810000698047FFE7FFE702B080BD33
:1096E00080B592B0119011980068006810901198A0
:1096F0000068C0680F901198006840690E900020C3
:109700000D900C90109800F00F000D900D9888B9F6
:10971000FFE79DF84000800600280AD5FFE79DF886
:109720003C008006002804D5FFE7119805F06AFB8D
:1097300002E2FFE70D98002800F0C280FFE79DF8E5
:109740003800C00738B9FFE7BDF83C0010F4907F3F
:1097500000F0B680FFE79DF84000C00758B1FFE772
:109760009DF83D00C00730B1FFE71199486C40F00B
:1097700001004864FFE79DF84000400700280BD532
:10978000FFE79DF83800C00730B1FFE71199486C3A
:1097900040F002004864FFE79DF840008007002881
:1097A0000BD5FFE79DF83800C00730B1FFE71199EE
:1097B000486C40F004004864FFE79DF84000000753
:1097C000002811D5FFE79DF83C008006002805D44D
:1097D000FFE79DF83800C00730B1FFE71199486CEA
:1097E00040F008004864FFE71198406C002866D0FC
:1097F000FFE79DF84000800600280AD5FFE79DF8A6
:109800003C008006002804D5FFE7119805F0FAFA1D
:10981000FFE7119800684069C0F380100C90119820
:10982000406C0007002804D4FFE70C9800283ED0C5
:10983000FFE7119805F048FA119800684069400662
:1098400000282FD5FFE7FFE7FFE71198006850E8F1
:10985000050F20F040000B90FFE70B99119802686C
:1098600042E805100028F0D1FFE7FFE71198C06B30
:1098700098B1FFE71198C16B4EF60930C0F60000B1
:1098800008651198C06BFCF79BFB28B1FFE71198A6
:10989000C06B016D8847FFE703E01198FFF7F6FE04
:1098A000FFE703E01198FFF7F1FEFFE706E01198EC
:1098B000FFF7ECFE119900204864FFE7FFE73BE16A
:1098C0001198006B012840F01781FFE79DF84000D8
:1098D000C006002840F11081FFE79DF83C00C0065B
:1098E000002840F10981FFE7FFE700200A90119866
:1098F000006800680A901198006840680A900A9809
:10990000FFE71198006840694006002840F19A80FE
:10991000FFE71198C06B00684068ADF82600BDF8FD
:109920002600002875D0FFE7BDF826001199898D23
:1099300088426EDAFFE7BDF826001199C8851198B4
:10994000C06BC069B0F5807F58D0FFE7FFE7FFE745
:109950001198006850E8030F20F480700890FFE72A
:1099600008991198026842E803100028F0D1FFE737
:10997000FFE7FFE7FFE71198006850E8050F20F0C8
:1099800001000790FFE707991198026842E8051067
:109990000028F0D1FFE7FFE7FFE7FFE71198006835
:1099A00050E8050F20F040000690FFE70699119857
:1099B000026842E805100028F0D1FFE7FFE711999F
:1099C000202081F84200119900200863FFE7FFE79B
:1099D0001198006850E8030F20F010000590FFE791
:1099E00005991198026842E803100028F0D1FFE7BA
:1099F000FFE71198C06BFCF76DFAFFE711990220A1
:109A000048631198818DC28D891A89B2FFF738FE9B
:109A100017E0BDF826001199898D884210D1FFE723
:109A20001198C06BC069B0F5807F08D1FFE711992C
:109A3000022048631198818DFFF722FEFFE7FFE7C0
:109A4000FFE779E01199888DC98D401AADF81200B1
:109A50001198C08D00284ED0FFE7BDF812000028F5
:109A600049D0FFE7FFE7FFE71198006850E8030FD0
:109A700020F490700390FFE703991198026842E880
:109A800003100028F0D1FFE7FFE7FFE7FFE7119899
:109A9000006850E8050F20F001000290FFE70299EE
:109AA0001198026842E805100028F0D1FFE7FFE7AF
:109AB0001199202081F84200119900200863FFE7E6
:109AC000FFE71198006850E8030F20F010000190A4
:109AD000FFE701991198026842E803100028F0D1CD
:109AE000FFE7FFE71199022048631198BDF81210B3
:109AF000FFF7C6FDFFE71FE09DF8400000060028C5
:109B00000AD5FFE79DF83C000006002804D5FFE7D2
:109B1000119805F061FB0FE09DF840004006002819
:109B20000AD5FFE79DF83C004006002804D5FFE772
:109B3000119805F013F9FFE712B080BD80B582B02F
:109B40000090009820B9FFE701208DF8070040E061
:109B50000098806908B1FFE700E0FFE7009890F8FF
:109B6000410040B9FFE70099002081F840000098CB
:109B700000F034F8FFE70099242081F841000098B4
:109B80000168C86820F40050C860009805F0EEF93C
:109B900000980168086920F4904008610098016805
:109BA000486920F02A00486100980168C86840F4BC
:109BB0000050C860009900204864009A202182F873
:109BC0004110009A82F84210009948638DF807000E
:109BD000FFE79DF8070002B080BD000080B590B09F
:109BE0000F9000200E900D900C900B900A900F9803
:109BF000006844F60001C4F2000188425FD1FFE72B
:109C0000FFE70020099043F64000C4F2020001681B
:109C100041F480210160006800F4802009900998D7
:109C2000FFE7FFE70020089043F63000C4F202008F
:109C3000016841F004010160006800F00400089030
:109C40000898FFE74FF440600A9002200B90002034
:109C500004900C9003200D9007200E9040F6000019
:109C6000C4F202000AA9FCF7E9FC049940F6A4003A
:109C7000C2F20000059046F22802C4F2020202601D
:109C80004FF0006242608160C1604FF48062026107
:109C900041618161C16101624162FCF743FB18B11E
:109CA000FFE7FAF763FCFFE7FFE70F9840F6A40130
:109CB000C2F20001C1630F988863FFE79CE00F9830
:109CC000006841F20041C4F20101884240F09380F3
:109CD000FFE7FFE70020079043F64400C4F20200CC
:109CE000016841F020010160006800F02000079049
:109CF0000798FFE7FFE70020069043F63000C4F224
:109D00000200016841F040010160006800F040007D
:109D100006900698FFE74FF484400A9002200B90CB
:109D2000002002900C9003200D9008200E9041F628
:109D30000000C4F202000AA9FCF780FC029940F678
:109D40000410C2F20000039046F22842C4F202025C
:109D500002604FF0206242608160C1604FF4806217
:109D6000026141618161C16101624162FCF7DAFA1D
:109D700018B1FFE7FAF7FAFBFFE7FFE70F9840F6A5
:109D80000411C2F20001C1630F988863FFE740F637
:109D90006410C2F20000019046F2A041C4F2020138
:109DA00001604FF020614160402181600021C1606D
:109DB0004FF48062026141618161C161016241626F
:109DC000FCF7B0FA18B1FFE7FAF7D0FBFFE7FFE7BF
:109DD0000F9840F66411C2F2000181630F98886306
:109DE000FFE74720009005210022FDF7CBF80098FF
:109DF000FDF7BEF8FFE7FFE710B080BD80B584B087
:109E000002900191ADF80220029890F842002028BB
:109E100017D1FFE7019820B1FFE7BDF8020020B994
:109E2000FFE701208DF80F000FE002990020086382
:109E300002980199BDF8022005F036F98DF80F005F
:109E400003E002208DF80F00FFE79DF80F0004B03B
:109E500080BD000080B582B00190019804F0AEFF93
:109E60008DF803009DF8030003281BD0FFE79DF841
:109E7000030000EBC00140F2A430C2F2000000EB8E
:109E80008100C06868B1FFE79DF8030000EBC001E6
:109E900040F2A430C2F2000000EB8100C0688047AD
:109EA000FFE7FFE702B080BD80B582B00190019866
:109EB00004F084FF8DF803009DF8030003281BD0F5
:109EC000FFE79DF8030000EBC00140F2A430C2F2AE
:109ED000000000EB8100806868B1FFE79DF8030097
:109EE00000EBC00140F2A430C2F2000000EB8100A0
:109EF00080688047FFE7FFE702B080BD80B582B091
:109F00000190019804F05AFF8DF803009DF80300BA
:109F100003281BD0FFE79DF8030000EBC00140F2CF
:109F2000A430C2F2000000EB8100406868B1FFE796
:109F30009DF8030000EBC00140F2A430C2F2000023
:109F400000EB810040688047FFE7FFE702B080BD7B
:109F5000FFE7FEE784B08DED030A9DED030AB6EE40
:109F6000001A20EE010A8DED020A03980190019873
:109F70000090009945F6DF10C5F63770A0EB610040
:109F80000090009801909DED010A9DED021A21EECE
:109F9000001A21EE002AB7EE081A31EE422A20EE0E
:109FA000020A8DED010A9DED010A9DED022A22EEC5
:109FB000002A22EE002A31EE421A20EE010A8DED2F
:109FC000010A9DED010A04B07047000083B08DEDD9
:109FD000020ACDED010A8DED001A9DED020A9DEDFC
:109FE000011A30EE410A9DED001A30EE010A40F2EE
:109FF000EC30C2F2000080ED000A9DED020A9DEDFA
:10A00000011A30EE010A9DED001A30EE010A80EDD2
:10A01000010A9DED021A9DED010A30EE411A9DEDF7
:10A02000000A30EE010A80ED020A9DED020AB1EE4F
:10A03000400A9DED011A30EE410A9DED001A30EE06
:10A04000010A80ED030A03B07047000080B586B0B6
:10A0500004908DED030A049818B9FFE700200590DD
:10A060004CE09DED030A049890ED014A90ED022A20
:10A0700090ED063A90ED071A23EE043A30EE430ACB
:10A0800021EE021A30EE410A8DED020A002028B9B5
:10A09000FFE7029805F04CF958B90DE002980BF073
:10A0A0000BFF41EC100B51EC100B05F027F918B128
:10A0B000FFE703980290FFE79DED020A049890EDF8
:10A0C000034A90ED043A90ED052A90ED061A20EE31
:10A0D000040A21EE031A30EE010A90ED071A21EE70
:10A0E000021A30EE010A8DED010A04998869C861EF
:10A0F00002980499886101980590FFE79DED050A93
:10A1000006B080BD80B588B007908DED060ACDED14
:10A11000050A079808B9FFE78BE0059807990860DA
:10A120000799002088610799C861079890ED000A97
:10A13000B5EE400AF1EE10FA0EDCFFE707994FF09A
:10A140007E50C86007990020086107994861079907
:10A150004860079988606CE09DED060A079890EDCD
:10A16000001A80EE010A8DED040A9DED041A9FEDA0
:10A17000320A80EE010A0AF015FF8DED030A9FED09
:10A180002F0A8DED000A0AF09DFDB0EE401A9DEDFC
:10A19000000A31EE011A9DED033A21EE031AB7EEE3
:10A1A000002A8DED012A31EE021A23EE033A31EE38
:10A1B000031A8DED021A9DED031A21EE011A9DED91
:10A1C000023A81EE031A079880ED031A079890ED82
:10A1D000031A31EE011A80ED041A0799C868486124
:10A1E0009DED031A21EE011A31EE421A31EE011AE9
:10A1F0009DED022A81EE021A079880ED011A0AF0FD
:10A2000061FDB0EE401A9DED010A31EE012A9DED8F
:10A21000031A22EE012A30EE420A21EE011A30EE34
:10A22000010A9DED021A80EE010A079880ED020AEC
:10A23000FFE708B080BD00BFDB0F4940DB0F493F9F
:10A2400080B584B002908DED010A029818B9FFE73D
:10A250000020039039E09DED010A029890ED031A69
:10A2600090ED043A90ED052A31EE031A31EE021A10
:10A2700080EE010A8DED000A002028B9FFE7009862
:10A2800005F024F858B911E000980BF015FE41ECE8
:10A29000100B51EC100B04F0F9FF38B1FFE70098F8
:10A2A0000299886100980299C86106E001980299B4
:10A2B000886101980299C861FFE702989DED010A43
:10A2C000FFF7C4FE8DED030AFFE79DED030A04B01E
:10A2D00080BD000080B582B08DF806009DF80600B4
:10A2E000022804DBFFE7FF208DF8070039E09DF826
:10A2F000061040F2A440C2F2000050F8210020B144
:10A30000FFE700208DF807002BE08820F8F704FE17
:10A3100001469DF8062040F2A440C2F2000040F839
:10A3200022109DF8061050F8210020B9FFE7FF2009
:10A330008DF8070015E09DF8061040F2A440C2F227
:10A340000000009050F821008821F6F7A4F8009949
:10A350009DF8060051F82010087000208DF80700C5
:10A36000FFE79DF9070002B080BD000080B588B00E
:10A370000690069820B9FFE7FE208DF81F002EE01A
:10A38000069800F049F80590059820B9FFE7FC20F1
:10A390008DF81F0023E005988088019008208DF833
:10A3A0000800FF208DF809008DF80A008DF80B00D9
:10A3B0008DF80C008DF80D008DF80E008DF80F0053
:10A3C000FC208DF810000598007801A9F8F758FBDB
:10A3D000002818BF4FF0FF308DF81F00FFE79DF9F0
:10A3E0001F0008B080BD000082B08DF803009DF80A
:10A3F0000300022803DBFFE70020019009E09DF83D
:10A40000031040F2A440C2F2000050F82100019075
:10A41000FFE7019802B0704780B586B004900498B9
:10A4200018B9FFE70020059036E004980078FFF7A0
:10A43000DBFF0390039818B9FFE7002005902BE09D
:10A4400000200290FFE70298039991F88410884257
:10A450001FDAFFE70398029900EB81004068019042
:10A46000019888B1FFE7019800780499097888423B
:10A470000AD1FFE70198408804994988884203D1AE
:10A48000FFE70198059007E0FFE70298013002908E
:10A49000D9E700200590FFE7059806B080BD0000D1
:10A4A00080B584B002900191029818B1FFE701983D
:10A4B00020B9FFE7FE208DF80F0011E00298FFF7AA
:10A4C000ABFF0090009820B9FFE7FC208DF80F004B
:10A4D00006E00098019900F049F98DF80F00FFE7B8
:10A4E0009DF90F0004B080BD80B586B00490039143
:10A4F000049818B1FFE7039820B9FFE7FE208DF814
:10A50000170090E003984178807840EA0120ADF888
:10A510000A00BDF80A009FED460ADFED460A102149
:10A5200007F0D2FB049880ED070A0399C8780979EF
:10A53000000140EA1110ADF80800BDF80800BBEEBC
:10A540000E0AF3EE0E0A0C21009107F0BDFB0099F4
:10A55000049880ED080A03980279407902F00F020E
:10A5600040EA0220ADF80600BDF80600BAEE080A7F
:10A57000F2EE080A07F0A8FB049880ED090A039898
:10A58000807900EE100AB8EE400A049880ED0A0ABD
:10A59000FFE7049890ED070AB5EE400AF1EE10FAD5
:10A5A0000ADAFFE7049890ED070A9FED231A30EED0
:10A5B000010A80ED070AECE7FFE7049890ED070A2F
:10A5C0009FED1D1AB4EE410AF1EE10FA0ADBFFE727
:10A5D000049890ED070A9FED191A30EE010A80EDFC
:10A5E000070AEAE70498C079C007C0B1FFE70498FA
:10A5F00090ED071A9FED100A30EE410A80ED070A30
:10A60000049890ED080AB1EE400A80ED080A04981B
:10A6100090ED090AB1EE400A80ED090AFFE700203B
:10A620008DF81700FFE79DF9170006B080BD00BF49
:10A63000DA0F49C1DA0F4941DB0FC940DB0FC9C04E
:10A6400080B586B00490049820B9FFE7FE208DF80D
:10A65000170087E004980078FFF73CFE20B1FFE781
:10A66000FF208DF817007DE004980078FFF7BCFE0E
:10A670000390039820B9FFE7FF208DF8170071E0E1
:10A6800000200290FFE70298039991F88410884215
:10A690001BDAFFE70398029900EB8100406878B16C
:10A6A000FFE70398029900EB810040684088049915
:10A6B0004988884204D1FFE7FD208DF8170051E05A
:10A6C000FFE7029801300290DDE7039890F88400DC
:10A6D000202804DBFFE7FF208DF8170042E0302040
:10A6E000F8F71AFC0190019820B9FFE7FF208DF8D8
:10A6F000170037E001983021F5F7CDFE0199049A53
:10A70000106852684A600860019900200872049835
:10A71000C079019900F00100087604984088ADF8EE
:10A72000020004980078BDF802100322F7F7E6FF54
:10A7300038B1FFE70198F8F7F9FAFF208DF8170014
:10A7400010E00198039991F8842001EB82014860A0
:10A75000039991F88400013081F8840000208DF87D
:10A760001700FFE79DF9170006B080BD80B58EB0D9
:10A770000C900B910C9818B1FFE70B9820B9FFE7EC
:10A78000FE208DF8370087E00C988088ADF818001F
:10A790000B9890ED020ADFED420A9FED421A10205D
:10A7A00005F0E6FBADF822000B9890ED010AFBEEF8
:10A7B0000E0AB3EE0E1A0C20019005F0D9FB0146EB
:10A7C0000198ADF820100B9991ED030ADFED360AE0
:10A7D000CDED000A9FED351A05F0CAFBDDED000A4C
:10A7E00001460198ADF81E100B9991ED040AB1EEE7
:10A7F000041A05F0BDFB01460198ADF81C100B9939
:10A8000091ED000AFAEE080AB2EE081A05F0B0FB64
:10A81000ADF81A009DF823008DF824009DF8220061
:10A820008DF82500BDF8200000098DF82600BDF840
:10A8300020109DF81F0040EA01108DF827009DF8B8
:10A840001E008DF82800BDF81C0000098DF82900B5
:10A85000BDF81C109DF81B0040EA01108DF82A007D
:10A860009DF81A008DF82B000C9880880290082023
:10A870008DF80C0009980A99CDF81110CDF80D004B
:10A880000C98007802A9F8F7FBF8002818BF4FF0E1
:10A89000FF308DF83700FFE79DF937000EB080BD1F
:10A8A000DA0F49C1DA0F4941000000000000FA4305
:10A8B00080B590B00E900E9820B9FFE7FE208DF87D
:10A8C0003F0077E00E980078FFF78EFD0D900D9811
:10A8D00020B9FFE7FC208DF83F006BE000200C90D2
:10A8E0000B90FFE70B980D9991F8841088421EDABF
:10A8F000FFE70D980B9900EB8100406890B1FFE7EE
:10A900000D980B9900EB8100406840880E994988AA
:10A91000884207D1FFE70D980B9900EB8100406852
:10A920000C9004E0FFE70B9801300B90DAE70C98ED
:10A9300020B9FFE7FC208DF83F003BE00E984088EF
:10A94000ADF82A000E980078BDF82A1003AA00235B
:10A95000F7F766FDE0B1FFE7F8F7C8FC019100905A
:10A96000009901980C9A13695269C91A904148F2EA
:10A97000A162C0F20102891A70F1000004D3FFE75E
:10A980000C9900200872FFE7FF208DF83F0011E0CE
:10A990000C9901200872F8F7A9FC0A460C994A6143
:10A9A00008610C9803A90D31FFF79EFD00208DF87A
:10A9B0003F00FFE79DF93F0010B080BD80B582B039
:10A9C0008DF806009DF80600022804DBFFE7FF2053
:10A9D0008DF8070039E09DF8061040F2AC40C2F255
:10A9E000000050F8210020B1FFE700208DF807009B
:10A9F0002BE04820F8F790FA01469DF8062040F237
:10AA0000AC40C2F2000040F822109DF8061050F849
:10AA1000210020B9FFE7FF208DF8070015E09DF821
:10AA2000061040F2AC40C2F20000009050F8210045
:10AA30004821F5F730FD00999DF8060051F82010E7
:10AA4000087000208DF80700FFE79DF9070002B0AD
:10AA500080BD000080B58EB00C900C9820B9FFE747
:10AA6000FE208DF83700A9E00C98007800F0AAF8D5
:10AA70000B900B9820B9FFE7FC208DF837009DE084
:10AA80000B9802300A900C984088ADF81600BDF87B
:10AA90001610A1F20120019104280CD3FFE70198C0
:10AAA000A0F20520042829D3FFE70198A0F209208D
:10AAB000032849D372E04FF40070069008208DF807
:10AAC0001C0000200490FFE70498032815DCFFE732
:10AAD0000A98049A00EB4200407806A9053101F873
:10AAE00012000A98049A30F8120001EB42014870F3
:10AAF000FFE7049801300490E6E753E040F2FF10CE
:10AB0000069008208DF81C0004200390FFE70398AE
:10AB1000072818DCFFE70A98039A00EB4200407808
:10AB200006A9053101EB420202F8080C0A98039AC3
:10AB300030F8120001EB420101F8070CFFE703981F
:10AB400001300390E3E72DE040F2FF20069008205B
:10AB50008DF81C000290FFE702980A2818DCFFE736
:10AB60000A98029A00EB4200407806A9053101EBF1
:10AB7000420202F8100C0A98029A30F8120001EB17
:10AB8000420101F80F0CFFE7029801300290E3E761
:10AB900000208DF823008DF8240003E0FF208DF8BD
:10ABA00037000BE00C98007806A9F7F769FF00283A
:10ABB00018BF4FF0FF308DF83700FFE79DF93700E1
:10ABC0000EB080BD82B08DF803009DF8030002280E
:10ABD00003DBFFE70020019009E09DF8031040F23D
:10ABE000AC40C2F2000050F821000190FFE701984C
:10ABF00002B0704782B08DF805009DF8050001464F
:10AC0000009140B1FFE70098012809D0FFE70098C4
:10AC100002280AD00EE042F21070ADF806000EE0F5
:10AC20004FF48040ADF8060009E047F23050ADF82F
:10AC3000060004E04FF6FF70ADF80600FFE7BDF92F
:10AC4000060002B07047000083B0ADF808008DF830
:10AC500007109DF8070001460091022804D3FFE782
:10AC60000098022813D026E0BDF80800B0F5007F58
:10AC70000CDDFFE7BDF80800B0F5027F06DAFFE75C
:10AC8000BDF8080001388DF80B0019E014E0BDF89C
:10AC90000800B0F5017F0DDDFFE7BDF8080040F2C8
:10ACA0000A21884206DCFFE7BDF8080001388DF86C
:10ACB0000B0005E000E0FFE7FF208DF80B00FFE749
:10ACC0009DF90B0003B0704780B586B004900498DE
:10ACD00018B9FFE7002005902FE004980078FFF7EF
:10ACE00071FF0390039818B9FFE70020059024E056
:10ACF00000200290FFE70298039991F844108842DF
:10AD000018DAFFE70398029900EB8100806901904F
:10AD1000019850B1FFE7019840880499498888421A
:10AD200003D1FFE70198059007E0FFE702980130A3
:10AD30000290E0E700200590FFE7059806B080BD8F
:10AD400083B08DF807009DF807000146009140B1DF
:10AD5000FFE70098012809D0FFE7009802280BD0F0
:10AD60000EE00020C4F2102002900DE04AF22C0008
:10AD7000C4F29910029007E04FF07E50029003E079
:10AD80004FF07E500290FFE79DED020A03B070473E
:10AD900080B586B00490049820B9FFE7FE208DF8B6
:10ADA000170081E004980078FFF708FE20B1FFE764
:10ADB000FF208DF8170077E004980078FFF702FF76
:10ADC0000390039820B9FFE7FF208DF817006BE090
:10ADD00000200290FFE70298039991F844108842FE
:10ADE0001BDAFFE70398029900EB8100806978B1D4
:10ADF000FFE70398029900EB81008069408804997D
:10AE00004988884204D1FFE7FD208DF817004BE008
:10AE1000FFE7029801300290DDE7039890F84400C4
:10AE20000B2804DBFFE7FF208DF817003CE05020E3
:10AE3000F8F772F80190019820B9FFE7FF208DF82C
:10AE4000170031E00199049A106852684A6008605E
:10AE5000019818302821F5F71EFB049840790199D4
:10AE600000F0010081F8280004990878498803223D
:10AE7000F7F744FC38B1FFE70198F7F757FFFF20D9
:10AE80008DF8170010E00198039991F8442001EB28
:10AE900082018861039991F84400013081F84400EF
:10AEA00000208DF81700FFE79DF9170006B080BD60
:10AEB00080B582B0019001989FED020A00F004F87D
:10AEC00002B080BD0000000080B58AB007A90191E2
:10AED00001460198089180ED000A089820B9FFE723
:10AEE000FE208DF8270078E008980078FFF76AFECA
:10AEF0000690069820B9FFE7FC208DF827006CE04B
:10AF0000019890ED000AB7EE001AB4EE410AF1EE96
:10AF100010FA04DDFFE74FF07E500790FFE701983D
:10AF200090ED000ABFEE001AB4EE410AF1EE10FAFD
:10AF300005DAFFE70020CBF680700790FFE708985E
:10AF40004079C00740B1FFE7019890ED000AB1EEEB
:10AF5000400A80ED000AFFE70898FFF7B5FE05906C
:10AF6000059820B9FFE7FC208DF8270035E0089907
:10AF700048880979FFF768FE8DF813009DF91300E2
:10AF8000B0F1FF3F04DCFFE7FF208DF8270024E04D
:10AF9000019806990231039190ED000A8DED000AA7
:10AFA00008980079FFF726FE9DED000A01EE100AD1
:10AFB000B8EEC11A20EE010ABDEEC00A10EE100A6A
:10AFC000ADF80A00BDF80A0003999DF9132021F895
:10AFD000120000208DF82700FFE79DF927000AB036
:10AFE00080BD000080B590B00E900E9820B9FFE7AC
:10AFF000FE208DF83F0072E00E980078FFF7E2FD2A
:10B000000D900D9820B9FFE7FC208DF83F0066E019
:10B0100000200C90FFE70C980D9991F8441088429D
:10B0200059DAFFE70D980C9900EB810080690B90CD
:10B030000B9800284AD0FFE70B9840880E99498862
:10B04000884243D1FFE70E990878498804AA002373
:10B05000F7F7E6F9E8B1FFE7F8F748F9039102904E
:10B06000029903980B9A136A526AC91A904140F2E6
:10B07000E932891A70F1000007D3FFE70B9900202D
:10B080000876FC208DF83F0029E0FF208DF83F0076
:10B0900025E00B9901200876F8F728F90A460B9964
:10B0A0004A6208620B9804A900F00CFC0B9901910C
:10B0B0008868CA680B69D1F814C0C1F838C04B63FE
:10B0C0000A63C86200208DF83F0008E0FFE70C9893
:10B0D00001300C909FE7FC208DF83F00FFE79DF9C1
:10B0E0003F0010B080BD000080B582B040F23470E7
:10B0F000C2F20000019046F20041C4F2000101607A
:10B100000321416000218160C1604FF4102202617F
:10B110004FF4001242610176417681760122C276B7
:10B1200001774177FAF7DAFA18B1FFE7F9F71EFA73
:10B13000FFE702B080BD000080B582B040F25C70D5
:10B14000C2F20000019046F60001C4F20001016065
:10B150000321416000218160C1604FF4102202612F
:10B160004FF4001242610176417681760122C27667
:10B1700001774177FAF7B2FA18B1FFE7F9F7F6F974
:10B18000FFE702B080BD000080B58AB0FFE7002075
:10B19000099043F63000C4F20200016841F4001146
:10B1A0000160006800F4001009900998FFE7FFE7CC
:10B1B0000020089043F63000C4F20200016841F418
:10B1C00080010160006800F4800008900898FFE7A3
:10B1D0000C2000900521059100220692FBF7D2FE7B
:10B1E0000098FBF7C5FE0599069A0D200190FBF724
:10B1F000C9FE0198FBF7BCFE0599069A392002901A
:10B20000FBF7C0FE0298FBF7B3FE0599069A3A20B9
:10B210000390FBF7B7FE0398FBF7AAFE0599069A81
:10B220003B200490FBF7AEFE0498FBF7A1FE0599C6
:10B23000069A45200790FBF7A5FE0798FBF798FEB6
:10B240000AB080BD80B582B04DF63D10C0F600005A
:10B2500046F26032C0F601020021019105F082FB46
:10B26000019940F22052C2F2000210604EF2E50055
:10B27000C0F6000046F21832C0F6010205F072FB7B
:10B2800002B080BD80B59AB0002019901890179038
:10B2900016901590FFE70020149043F63000C4F29A
:10B2A0000200016841F002010160006800F0020044
:10B2B00014901498FFE7FFE70020139043F6300046
:10B2C000C4F20200016841F040010160006800F032
:10B2D000400013901398FFE7FFE70020129043F619
:10B2E0003000C4F20200016841F001010160006811
:10B2F00000F0010012901298FFE7FFE70020119084
:10B3000043F63000C4F20200016841F00801016018
:10B31000006800F0080011901198FFE7FFE7002097
:10B32000109043F63000C4F20200016841F00401BD
:10B330000160006800F0040010901098FFE7FFE73C
:10B3400000200F9043F63000C4F20200016841F083
:10B3500080010160006800F080000F900F98FFE707
:10B36000FFE700200E9043F63000C4F202000168AF
:10B3700041F020010160006800F020000E900E985E
:10B38000FFE741F60000C4F2020001904021009165
:10B3900000220C92FBF746FB0020C4F2020003904F
:10B3A0001021029101220592FBF73CFB059A40F225
:10B3B0000040C4F2020006901146FBF733FB009AEE
:10B3C00001980599159216911791189115A9079151
:10B3D000FBF734F90198059A0799082315934FF460
:10B3E0000413049316931792FBF728F90398049B10
:10B3F000059A0799159216931792FBF71FF9029B6E
:10B400000398059A07991593169217921892FBF7CD
:10B4100015F9049A059807993023159316921790F9
:10B4200040F60000C4F20200FBF708F9059A0698FE
:10B4300007991592169217921892FBF7FFF80C9A3B
:10B440000620089005210B91FBF79CFD0898FBF75F
:10B450008FFD0B990C9A09200990FBF793FD099831
:10B46000FBF786FD0B990C9A0A200A90FBF78AFDE0
:10B470000A98FBF77DFD0B990C9A17200D90FBF7AE
:10B4800081FD0D98FBF774FD1AB080BD80B582B0C8
:10B4900040F6C410C2F20000019045F60041C4F22B
:10B4A0000001016041F68021C0F2060141600021E7
:10B4B0008160C1604FF48042026141618161C1617C
:10B4C0000162FBF7CDFA18B1FFE7F9F74FF8FFE794
:10B4D00002B080BD80B582B040F61820C2F20000F4
:10B4E000019043F20001C4F2010101604FF4827146
:10B4F000416000218160C16002220261012242613B
:10B500004FF4007282611822C2610162416281625D
:10B510000A21C162FCF7B2FA18B1FFE7F9F726F881
:10B52000FFE702B080BD000080B588B00021009127
:10B53000079106910591049103910291019140F6C2
:10B540007020C2F2000044F20042C4F20102026024
:10B550004160816041F28732C26001618161FDF723
:10B560003BFC18B1FFE7F9F701F8FFE740F6702060
:10B57000C2F20000FDF7ACFE18B1FFE7F8F7F6FFE6
:10B58000FFE760200190002202920392059240F6AC
:10B590007020C2F2000001A9FDF7F8FD18B1FFE725
:10B5A000F8F7E4FFFFE740F67020C2F20000FDF775
:10B5B0005FFD08B080BD000080B58AB00021009119
:10B5C00009910891079106910591049103910291C7
:10B5D000019140F6B820C2F2000040F60002C4F229
:10B5E00000020260416081604FF6FF72C26001613B
:10B5F0008161FDF76DFE18B1FFE7F8F7B7FFFFE7D0
:10B6000000200890099040F6B820C2F2000008A976
:10B61000FDF750FB18B1FFE7F8F7A8FFFFE7602040
:10B620000190002002900390059040F6B820C2F2ED
:10B63000000001A90822FDF7A9FD18B1FFE7F8F7FE
:10B6400095FFFFE740F6B820C2F20000FDF710FDBD
:10B650000AB080BD80B58EB0002100910D910C9193
:10B660000B910A9109910891079106910591049116
:10B6700003910291019140F60030C2F2000040F6C1
:10B680000042C4F200020260416081604FF6FF7226
:10B69000C26001618161FDF79FFB18B1FFE7F8F718
:10B6A00065FFFFE74FF480500A9040F60030C2F289
:10B6B00000000AA9FDF71AFC18B1FFE7F8F756FFDA
:10B6C000FFE740F60030C2F20000FDF701FE18B1BE
:10B6D000FFE7F8F74BFFFFE700200890099040F6DE
:10B6E0000030C2F2000008A9FDF7E4FA18B1FFE744
:10B6F000F8F73CFFFFE760200190002202920392DE
:10B70000059240F60030C2F2000001A9FDF73EFDAF
:10B7100018B1FFE7F8F72AFFFFE740F60030C2F262
:10B72000000001A90422FDF731FD18B1FFE7F8F789
:10B730001DFFFFE740F60030C2F2000001A9082219
:10B74000FDF724FD18B1FFE7F8F710FFFFE740F61B
:10B750000030C2F20000FDF78BFC0EB080BD00008F
:10B7600080B582B040F64830C2F20000019044F645
:10B770000001C4F20001016048F2A061C0F20101C1
:10B78000416000218160C16001610C2242618161E0
:10B79000C161FEF7D3F918B1FFE7F8F7E7FEFFE75D
:10B7A00002B080BD80B582B040F69030C2F2000099
:10B7B000019041F20041C4F2010101604FF4E13116
:10B7C000416000218160C16001610C2242618161A0
:10B7D000C161FEF7B3F918B1FFE7F8F7C7FEFFE75D
:10B7E00002B080BDFFE7FEE780B586B08DED050AAB
:10B7F00000200490FFE7049803283CDCFFE704984E
:10B80000C0EB001140F6BC60C2F2000000EB81000A
:10B810009DED050A40F29402C2F20002012102915C
:10B8200000F00EFB02990498C0EB001240F6DC40D9
:10B83000C2F2000000EB82009DED050A40F25402C6
:10B84000C2F2000200F0FCFA02990498C0EB001268
:10B8500040F6CC50C2F2000000EB82009DED050ADC
:10B8600040F27402C2F2000200F0EAFAFFE7049824
:10B8700001300490BFE79DED050A40F6A040C2F2FA
:10B88000000040F23402C2F200020021019100F0F7
:10B89000D7FAF6F715FE01980390FFE703980328FF
:10B8A0000EDCFFE7039940F21400C2F2000000EB47
:10B8B000C100FFF76DFAFFE7039801300390EDE751
:10B8C00006B080BD80B58AB0099008910898417B88
:10B8D000807B40EA0120ADF81E000898C17B007C07
:10B8E00040EA0120ADF81C000898417C807C40EAC9
:10B8F0000120ADF81A0009980079FFF77BF9ADF83F
:10B90000180009980079FFF71BFA8DED050ABDF8BC
:10B910001E0000EE100AB8EEC00A9FED6D1A80EE10
:10B92000010A9FED6C1A20EE010A8DED040ABDF9A3
:10B930001C0000EE100AB8EEC00A8DED030ABDF936
:10B940001A00BDF91810484300EE100AB8EEC00AFC
:10B950009FED611A80EE010A8DED020A0998807947
:10B96000C00700284CD0FFE7BDF81E000999B1F8C8
:10B970004010401A01900198B0F5805F05DDFFE7A7
:10B980000999486C013848640AE0019810F5805F15
:10B9900005DAFFE70999486C01304864FFE7FFE7E3
:10B9A000BDF81E000999A1F840000498009009987C
:10B9B00090ED110AB8EEC00A9FED461A20EE010A7A
:10B9C0009DED001A30EE010A9DED051A80EE010A88
:10B9D00080ED120A0999886C88609DED030A9DED3F
:10B9E000051A80EE010A099880ED030A9DED020A0E
:10B9F0009DED051A20EE010A099880ED040A13E076
:10BA0000099900204864BDF81E10099AA2F8401058
:10BA10000999886404980999886003980999C8600D
:10BA2000029809990861FFE7FFE7099890ED020A7B
:10BA3000B5EE400AF1EE10FA0ADAFFE7099890ED48
:10BA4000020A9FED241A30EE010A80ED020AECE7AB
:10BA5000FFE7099890ED020A9FED1E1AB4EE410A25
:10BA6000F1EE10FA0ADBFFE7099890ED020A9FED6C
:10BA70001B1A30EE010A80ED020AEAE7099890F8F5
:10BA80002800C007C0B1FFE7099890ED021A9FEDAA
:10BA9000110A30EE410A80ED020A099890ED030A7E
:10BAA000B1EE400A80ED030A099890ED040AB1EE68
:10BAB000400A80ED040AFFE70898C07C00EE100AF7
:10BAC000B8EE400A099880ED050A0AB080BD00BFB3
:10BAD00000000046DB0FC94000008046DB0FC9C0F4
:10BAE000FFE7FEE788B0079006910592079800F0FF
:10BAF000070004900498C0F10700052803D3FFE76E
:10BB00000420019004E00498C0F107000190FFE7D1
:10BB10000198039004980430062803D8FFE700201A
:10BB2000009003E0049803380090FFE7009802902B
:10BB300006980399012202FA01F101390840029B9B
:10BB4000984005999A40013A1140084308B070475F
:10BB500080B590B00E908DED0D0ACDED0C0A8DEDF7
:10BB60000B1ACDED0A1A002028B9FFE70D9803F053
:10BB7000B9FB58B943E00D980AF09EF941EC100B5F
:10BB800051EC100B03F092FBC8B3FFE7002028B97B
:10BB9000FFE70C9803F0A6FB58B930E00C980AF0C8
:10BBA0008BF941EC100B51EC100B03F07FFB30B321
:10BBB000FFE7002028B9FFE70B9803F093FB58B983
:10BBC0001DE00B980AF078F941EC100B51EC100BCA
:10BBD00003F06CFB98B1FFE7002028B9FFE70A9853
:10BBE00003F080FB78B90AE00A980AF065F941ECA5
:10BBF000100B51EC100B03F059FB20B9FFE70E9826
:10BC000080690F9016E19DED0D0ADDED0C0A0E988E
:10BC1000406890ED071AF7F751FD8DED090A9DED8B
:10BC2000090A0E98406890ED001A20EE010A8DED89
:10BC3000080A0E98406890ED000A9DED0C1A20EE5F
:10BC4000010A8DED070A0E981C309DED070AFEF7DC
:10BC5000FDF98DED060A0E9800780146019110B3AA
:10BC6000FFE70198012804D0FFE70198022817D0C8
:10BC70001CE09DED060A0E9890ED021A90ED052A43
:10BC800030EE420A9DED0A2AB4EE412AF1EE10FA96
:10BC9000C8BFB0EE421A80EE010A8DED050A05E03C
:10BCA0000B98059002E000200590FFE709980E9997
:10BCB000086106980E994861002028B9FFE70598A9
:10BCC00003F010FB70B90AE005980AF0F5F841ECB2
:10BCD000100B51EC100B03F0E9FA18B9FFE7002044
:10BCE0000590FFE79DED080A0E98406890ED011A57
:10BCF00090ED032A20EE010A9DED051A21EE021AAD
:10BD000030EE410A8DED040A0E9890ED030A9DED88
:10BD1000081A9DED0A2A21EE021A30EE010A8DED75
:10BD2000030A9DED030A0E98406890ED021A20EE7A
:10BD3000010A8DED020A0E98406890ED020A9FED0F
:10BD40003F1AB4EE410AF1EE10FA39DDFFE70020A8
:10BD500028B9FFE7039803F0C5FA58B92FE0039814
:10BD60000AF0AAF841EC100B51EC100B03F09EFA0C
:10BD700028B3FFE79DED040A9DED021A30EE010A9B
:10BD8000B0EEC00A0E98406890ED051AB4EE410A74
:10BD9000F1EE10FA12DCFFE79DED030AB0EEC00AE7
:10BDA0000E98406890ED041AB4EE410AF1EE10FAD4
:10BDB00004DCFFE703980E99C860FFE7FFE7FFE7A1
:10BDC0009DED021A9DED040A30EE010A8DED040A84
:10BDD000002028B9FFE7049803F084FA58B925E059
:10BDE00004980AF069F841EC100B51EC100B03F0C9
:10BDF0005DFAD8B1FFE70E98406890ED050A9FED17
:10BE00000F1AB4EE410AF1EE10FA0BDDFFE79DEDDB
:10BE1000040A0E984068D0ED050AF5F79BFE8DEDFB
:10BE2000040AFFE704980E998861FFE70E9880697D
:10BE30000F90FFE79DED0F0A10B080BDBD3786352E
:10BE400080B586B004908DF80F108DED020A019236
:10BE5000049820B9FFE7FF208DF81700B7E0002015
:10BE600030B9FFE70198406803F03CFA80B90BE075
:10BE7000019840680AF020F841EC100B51EC100BCF
:10BE800003F014FA20B9FFE7FF208DF817009EE0B9
:10BE9000002030B9FFE70198806803F023FA80B9E9
:10BEA0000BE0019880680AF007F841EC100B51ECA8
:10BEB000100B03F0FBF920B9FFE7FF208DF8170006
:10BEC00085E0002030B9FFE70198C06803F00AFA66
:10BED00080B90BE00198C06809F0EEFF41EC100B4F
:10BEE00051EC100B03F0E2F920B9FFE7FF208DF8C9
:10BEF00017006CE0002030B9FFE70198006903F0FB
:10BF0000F1F980B90BE00198006909F0D5FF41EC27
:10BF1000100B51EC100B03F0C9F920B9FFE7FF201B
:10BF20008DF8170053E0002030B9FFE70198406911
:10BF300003F0D8F980B90BE00198406909F0BCFF23
:10BF400041EC100B51EC100B03F0B0F920B9FFE7F6
:10BF5000FF208DF817003AE00198049948609DEDA4
:10BF6000021AB7EE000A80EE010A8DED000A0020E9
:10BF700028B9FFE7009803F0B5F958B90EE000982A
:10BF800009F09AFF41EC100B51EC100B03F08EF905
:10BF900020B1FFE700980499886003E0FF208DF846
:10BFA000170014E0049901F11C009DED020A496894
:10BFB000D1ED060AFEF7A6F89DF80F000499087067
:10BFC000049800F009F800208DF81700FFE79DF9AC
:10BFD000170006B080BD000080B584B002900298C2
:10BFE00020B9FFE7FF208DF80F0013E00299002031
:10BFF0000190C860029908610299486102998861BC
:10C0000002981C309FED050AFEF71AF901988DF889
:10C010000F00FFE79DF90F0004B080BD0000000095
:10C0200082B00090009820B9FFE7FF208DF807004C
:10C0300005E000990020C8608DF80700FFE79DF932
:10C04000070002B070470000000000000000000080
:10C05000EFF30980BFF36F8F154B1A681EF0100FB6
:10C0600008BF20ED108A20E9F04F10602DE909008B
:10C070004FF0500080F31188BFF34F8FBFF36F8FE5
:10C0800006F056FB4FF0000080F31188BDE8090070
:10C0900019680868B0E8F04F1EF0100F08BFB0EC48
:10C0A000108A80F30988BFF36F8F704700BF00BF0D
:10C0B000A010002080B582B001900198806B0090A4
:10C0C00000980168486820F0030048600099486DB6
:10C0D00040F0100048650099012081F85100009857
:10C0E000FBF7A2FC02B080BD80B582B00190019840
:10C0F000806B00900098FCF725F802B080BD00002E
:10C1000080B582B001900198806B00900098FCF798
:10C110004BFD02B080BD000080B582B00190019857
:10C12000806B00900098FCF793FD02B080BD00008A
:10C1300080B584B003900398806B0290FAF78AFC74
:10C14000019003980068006800F48070B0F5807F6B
:10C1500039D0FFE702980168486820F02000486065
:10C160000298806868B9FFE702984068B0F5827F5E
:10C1700007D1FFE702980168486820F00300486093
:10C1800006E002980168486820F001004860FFE777
:10C190000298019A642100F0B5F820B1FFE70299F6
:10C1A00020204865FFE702990020C88702990120F6
:10C1B00081F851000298406D20B1FFE70298FBF72B
:10C1C00033FC04E0FFE70298FBF792FFFFE704B0BF
:10C1D00080BD000080B584B003900398806B02900E
:10C1E000FAF738FC019003980068006800F480704A
:10C1F000B0F5807F3BD0FFE702980168486820F0E7
:10C200002000486002980168486820F002004860F9
:10C210000298019A642100F0E7F830B1FFE7029933
:10C22000486D40F020004865FFE70298806870B9CB
:10C23000FFE7FFE70020009002980068C0680090C8
:10C2400002980068806800900098FFE7FFE7029975
:10C250000020C8860299012081F851000298406DA3
:10C2600020B1FFE70298FBF7DFFB04E0FFE702984D
:10C27000FCF776FCFFE704B080BD000080B584B019
:10C2800003900398806B0290FAF7E4FB0190039807
:10C290000068006800F48070B0F5807F2BD0FFE765
:10C2A00002980168486820F0200048600298019ACE
:10C2B000642100F099F830B1FFE70299486D40F031
:10C2C00020004865FFE702980168486820F00300F5
:10C2D000486002990020C8860299C8870299012007
:10C2E00081F851000298406D20B1FFE70298FBF7FA
:10C2F0009BFB04E0FFE70298FCF780FCFFE704B03B
:10C3000080BD000080B586B004900391029204982D
:10C310004068B0F5827F13D1FFE704988068B0F5DC
:10C32000004F06D0FFE704988068B0F5806F07D112
:10C33000FFE704980168086820F040000860FFE704
:10C3400004984068B0F5827F31D1FFE70498806897
:10C35000B0F5806F15D0FFE70498039B02996A46F9
:10C3600011608021002200F0BDF848B1FFE7049978
:10C37000486D40F02000486503208DF817002FE03D
:10C3800014E00498039B02996A461160012100227F
:10C3900000F0A8F848B1FFE70499486D40F020008C
:10C3A000486503208DF817001AE0FFE714E00498B1
:10C3B000039B02996A4611600121002200F092F865
:10C3C00048B1FFE70499486D40F02000486503201C
:10C3D0008DF8170004E0FFE700208DF81700FFE755
:10C3E0009DF8170006B080BD80B586B0049003911B
:10C3F00002920498039B02996A461160022101226D
:10C4000000F070F848B1FFE70499486D40F0200053
:10C41000486503208DF8170048E040F20000C2F2A2
:10C42000000000684AF6AB21CAF6AA21A0FB011061
:10C4300000094DF68361C4F21B31A0FB0110800C92
:10C440004FF47A714843019004984068B0F5827FB8
:10C4500015D1FFE70498039B02996A461160802179
:10C46000002200F03FF848B1FFE70499486D40F022
:10C470002000486503208DF8170017E012E0FFE761
:10C48000019808B9FFE70CE0019801380190FFE737
:10C49000049800688068C1B20020B0EBD11FEFD1D2
:10C4A000FFE7FFE700208DF81700FFE79DF8170072
:10C4B00006B080BD82B000900098006843F2000191
:10C4C000C4F20101884204D1FFE700208DF8070083
:10C4D00003E002208DF80700FFE79DF8070002B097
:10C4E0007047000080B58AB0DDF830C00890079131
:10C4F0008DF81B20059305980190FAF7ABFA0246D8
:10C5000001980C99891A08440390FAF7A3FA02904B
:10C51000039840F20001C2F200010968C1F3CB3177
:10C5200048430490FFE7089800688068079908402E
:10C53000401AB0FA80F040099DF81B1088425FD085
:10C54000FFE705980130002859D0FFE7FAF782FA93
:10C550000299401A0399884204D2FFE70398002801
:10C5600042D1FFE708980168486820F0E000486081
:10C5700008984068B0F5827F13D1FFE7089880687B
:10C58000B0F5004F06D0FFE708988068B0F5806FDF
:10C5900007D1FFE708980168086820F040000860AC
:10C5A000FFE70898806AB0F5005F0FD1FFE7FFE76B
:10C5B00008980168086820F400500860089801682D
:10C5C000086840F400500860FFE7FFE70899012081
:10C5D00081F85100FFE70899002081F85000FFE73B
:10C5E00003208DF827000FE0049818B9FFE700201A
:10C5F000039003E0049801380490FFE7FFE792E717
:10C6000000208DF82700FFE79DF827000AB080BDC5
:10C61000074B19680868B0E8F04F80F30988BFF34A
:10C620006F8F4FF0000080F31188704700BF00BF8C
:10C63000A010002080B56FF00400002102F0E4FE9D
:10C6400080BD000084B003900291039890ED000A31
:10C65000029890ED001A30EE010A8DED010A9DED71
:10C66000010AB7EE001AB4EE410AF1EE10FA1BDD32
:10C67000FFE79DED011AB7EE000A80EE010A8DED8D
:10C68000000A9DED001A039890ED000A20EE010AC1
:10C6900080ED000A9DED001A029890ED000A20EE50
:10C6A000010A80ED000AFFE704B0704780B586B04C
:10C6B00004900391049828B1FFE70498B0F8A00013
:10C6C00020B9FFE7FF208DF8170060E0049890ED97
:10C6D000010A90ED271A30EE410A8DED020A049806
:10C6E000D0ED1E0A90ED310A9FED2B1AF6F7E6FF0A
:10C6F0008DED010A9DED020A0498406990ED042A2F
:10C70000B7EE001A81EE021AB4EE410AF1EE10FA09
:10C7100039DBFFE70398C078C007A0B3FFE79DEDC2
:10C72000010AB7EE001AB4EE410AF1EE10FA2ADC63
:10C73000FFE704994868C1F89C00049901F1C4001E
:10C74000496991ED030AB8EE400ADFED130A80EE65
:10C75000800AF6F771FF0498406990F834000128C8
:10C760000AD1FFE7049890ED310A9FED0C1A30EEE4
:10C77000010A80ED310AFFE70499B1F8A000013801
:10C78000A1F8A000FFE700208DF81700FFE79DF952
:10C79000170006B080BD00BFDB0FC940EBAB2B3CE0
:10C7A00084B002908DED010A029820B9FFE7FF20C6
:10C7B0008DF80F001EE00298406900780146009154
:10C7C00020B1FFE70098012808D00FE0029944F259
:10C7D0000000C4F29C50C1F8C00007E0029948F282
:10C7E0000000C4F23B50C1F8C000FFE700208DF804
:10C7F0000F00FFE79DF90F0004B0704780B586B0C9
:10C8000004900391049818B1FFE7039820B9FFE75B
:10C81000FF208DF817003BE0F6F768FD09F0A1FB5B
:10C8200000EE100A9FED1C1A8DED011A80EE010A30
:10C83000049880ED010AF6F759FD049A0292936874
:10C84000D268C01A914109F08CFB9DED011A014696
:10C85000029800EE101A80EE010A80ED040AF6F745
:10C8600045FD0A460499CA608860039800780499D7
:10C8700000F00100087004989FED080AFFF790FF90
:10C880000498039900F0B2F900208DF81700FFE733
:10C890009DF9170006B080BD00247449000069436B
:10C8A00080B58AB0089007918DED060A089858B1B6
:10C8B000FFE7079840B1FFE79DED060AB5EE400A95
:10C8C000F1EE10FA04DCFFE7FF208DF8270089E184
:10C8D000079840688DF817000798089948619DF8F7
:10C8E00017008000F6F718FB0899C1F8A4009DF81E
:10C8F00017008000F6F710FB0899C1F8A8009DF812
:10C9000017008000F6F708FB0899C1F8AC009DF805
:10C9100017008000F6F700FB0899C1F8B0009DF8F9
:10C9200017000001F6F7F8FA089908629DF8170059
:10C930008000F6F7F1FA0899C8679DF817008000A3
:10C94000F6F7EAFA0899C1F884009DF81700C0EBE1
:10C9500000108000F6F7E0FA0899C1F8C8009DF8C9
:10C960001700C0EB00108000F6F7D6FA0899C1F85E
:10C97000CC009DF817004001F6F7CEFA0899C1F8EF
:10C9800048019DF817004001F6F7C6FA0899C1F86A
:10C990004C010898006AB8B3FFE70898C06F98B3D5
:10C9A000FFE70898D0F8840070B3FFE70898D0F844
:10C9B000A40048B3FFE70898D0F8A80020B3FFE729
:10C9C0000898D0F8AC00F8B1FFE70898D0F8B000AC
:10C9D000D0B1FFE708984069C06AA8B1FFE708989E
:10C9E000D0F8C80080B1FFE70898D0F8CC0058B163
:10C9F000FFE70898D0F8480130B1FFE70898D0F871
:10CA00004C0100283ED1FFE70898006AF6F78EF93E
:10CA10000898C06FF6F78AF90898D0F88400F6F7FE
:10CA200085F90898D0F8A400F6F780F90898D0F8AE
:10CA3000A800F6F77BF90898D0F8AC00F6F776F97D
:10CA40000898D0F8B000F6F771F908984069C06A04
:10CA5000F6F76CF90898D0F8C800F6F767F9089867
:10CA6000D0F8CC00F6F762F90898D0F84801F6F74C
:10CA70005DF90898D0F84C01F6F758F9FB208DF8CD
:10CA80002700AFE0F5F71CFD00200490FFE70498B5
:10CA90009DF81710884248DAFFE70798C06A0499A2
:10CAA00001EB810100EB4100FEF772F90898D0F824
:10CAB000C8000499C1EB011100EB81009DED060A4D
:10CAC000079901F1380201210391FFF7B9F90399A0
:10CAD0000898D0F8CC00049AC2EB021200EB820056
:10CAE0009DED060A079A5832FFF7AAF9089841699E
:10CAF000D0F84801049A00EB42109DED060AD1EDF2
:10CB00003E0AFDF7FFFA08984169D0F84C01049AF3
:10CB100000EB42109DED060AD1ED3F0AFDF7F2FA57
:10CB2000FFE7049801300490B1E707983030FEF732
:10CB30002FF90898406990F8340001460291D0B16D
:10CB4000FFE7029801282CD1FFE70898D0309DED2F
:10CB5000060A079901F1B80201210191FFF770F966
:10CB60000199089800F586709DED060A079AD8325B
:10CB7000FFF766F919E00898D0309DED060A07998D
:10CB800001F1780201210091FFF75AF90099089804
:10CB900000F586709DED060A079A9832FFF750F966
:10CBA00003E0FC208DF827001CE0089901F5A8702F
:10CBB0009DED060A4969D1ED400AFDF7A3FA0899EF
:10CBC00001F5B8709DED060A4969D1ED410AFDF7FE
:10CBD00099FA08990020C1F8A000C1F89C008DF8CE
:10CBE0002700FFE79DF927000AB080BD80B584B01B
:10CBF00002900191029820B9FFE7FF208DF80F0005
:10CC0000C2E00298406990F82000C007002800F0B8
:10CC1000AB80FFE7029890F8980001460091032846
:10CC200000F29C800099DFE801F002205471029824
:10CC300090ED0E0A9FED581A80EE010A406990EDC2
:10CC4000091AB4EE410AF1EE10FA09DDFFE7029984
:10CC5000012081F8980002994868C1F89400FFE724
:10CC60000298019900F08CF97DE0029890ED0E0A8F
:10CC70009FED491A80EE010A406990ED091AB4EE61
:10CC8000410AF1EE10FA05DAFFE70299002081F877
:10CC9000980068E0029890ED010A90ED251A30EEB8
:10CCA000410A406990ED0A1AB4EE410AF1EE10FA19
:10CCB00009DBFFE70299012081F890000299022028
:10CCC00081F898004FE0FFE70298019900F058F9C9
:10CCD00049E002990020A1F8A000029890ED1E0AF8
:10CCE000416991ED031AB8EE412A9FED291A81EEB0
:10CCF000021A30EE010A80ED310A0299032081F810
:10CD0000980002994868C1F89400FFE702980199D9
:10CD100000F036F9029890ED010A90ED251A30EEF8
:10CD2000410A9FED1C1AB4EE410AF1EE10FA14DB31
:10CD3000FFE7029890ED0E0A9FED171A80EE010AA8
:10CD4000B3EE041AB4EE410AF1EE10FA05DAFFE789
:10CD50000299002081F89800FFE704E00299002082
:10CD600081F89800FFE70BE00299002081F8980015
:10CD7000029981F890000298019900F001F9FFE70B
:10CD800000208DF80F00FFE79DF90F0004B080BD73
:10CD9000DB0FC9C09A99993E00007A4480B586B0ED
:10CDA0000490049820B9FFE7FF208DF8170059E0A0
:10CDB0000498406940688DF80F0000200290FFE75A
:10CDC00002989DF80F1088422FDAFFE70498D0F8F8
:10CDD000C8000299C1EB011100EB8100FFF7FCF8DC
:10CDE0000498D0F8CC000299C1EB011100EB81004E
:10CDF000FFF7F2F80498D0F84801029900EB4110CF
:10CE00009FED1A0A8DED010AFDF71AFA9DED010A50
:10CE10000498D0F84C01029900EB4110FDF710FA8C
:10CE2000FFE7029801300290CAE70498D030FFF77C
:10CE3000D3F8049800F58670FFF7CEF8049800F553
:10CE4000A8709FED0A0A8DED000AFDF7F9F99DED36
:10CE5000000A049800F5B870FDF7F2F900208DF88B
:10CE60001700FFE79DF9170006B080BD0000000025
:10CE700080B584B00290029820B9FFE7FF208DF8BA
:10CE80000F0033E00298406940688DF807000020E9
:10CE90000090FFE700989DF80710884219DAFFE735
:10CEA0000298D0F8C8000099C1EB011100EB810095
:10CEB000FFF7B6F80298D0F8CC000099C1EB011149
:10CEC00000EB8100FFF7ACF8FFE70098013000901D
:10CED000E0E70298D030FFF7A3F8029800F58670DB
:10CEE000FFF79EF800208DF80F00FFE79DF90F0077
:10CEF00004B080BD84B00290029820B9FFE7FF2003
:10CF00008DF80F0038E00298406940688DF80700FE
:10CF100000200090FFE700989DF8071088421EDA75
:10CF2000FFE70298D0F8A410009A002041F82200F0
:10CF30000299D1F8A810009A41F822000299D1F87C
:10CF4000AC10009A41F822000299D1F8B010009A72
:10CF500041F82200FFE7009801300090DBE70299DA
:10CF60000020C1F8B4000299C1F8B8000299C1F8D4
:10CF7000BC008DF80F00FFE79DF90F0004B070476B
:10CF800080B594B012901191129818B1FFE71198E2
:10CF900020B9FFE7FF208DF84F0049E31298406960
:10CFA00040688DF843001298406980698DF842000E
:10CFB00012980078C007F0B9FFE700200F90FFE754
:10CFC0000F989DF8431088420FDAFFE712984069E6
:10CFD000C06A0F9901EB810100EB4100FDF768FF8A
:10CFE000FFE70F9801300F90EAE712984069303060
:10CFF000FDF75EFFF8E21298007E0146079150B1FE
:10D00000FFE70798012800F0B680FFE7079802289D
:10D0100000F0E981E3E200200E90FFE70E989DF812
:10D02000431088425DDAFFE71298D0F8C8000E99E5
:10D03000C1EB011100EB8100FEF7F2FF1299D1F86C
:10D04000C8000E9BC3EB031200EB8200D1F88420D2
:10D0500002EB8302D2ED000AD1ED041A9FEDE91A2A
:10D06000B0EE410AFEF774FD1298D0F8A4000E99B4
:10D0700000EB810080ED000A12990E9AD1F8A4000D
:10D08000D1F8AC1050F8220041F822001298D0F8E4
:10D09000AC10D0F84C010E9A00EB421001EB82016B
:10D0A00091ED000AFCF7D2FF1298D0F8B0000E996B
:10D0B00000EB810080ED000A12994869D1F8B010A8
:10D0C000C06A0E9A02EB820300EB430001EB82017F
:10D0D00091ED000AFDF7F8FEFFE70E9801300E9083
:10D0E0009CE7129901F1D00040F2A032C2F2000296
:10D0F00092ED000AD1ED041AD1ED1E0A9FEDC11A7E
:10D100008DED061AFEF724FD9DED061A129880EDAE
:10D110002D0A129901F58670D1ED041AD1ED230A7A
:10D1200091ED2D0AFEF714FD129880ED2E0A12994A
:10D1300001F5B87091ED2E0AFCF788FF129880ED8A
:10D140002F0A12994869303091ED2F0AFDF7BCFE85
:10D1500011988078C00768B1FFE71298FFF71EFEAC
:10D160001298FFF785FE1298FFF7C4FE129901206E
:10D170000876FFE737E200200D90FFE70D989DF855
:10D180004310884280F2B180FFE712984069C06A7C
:10D19000007A01388DF8330012984169C9699DF809
:10D1A000332001EB820191ED000A90ED301A20EE60
:10D1B000010A9FED951A80EE010A8DED0B0A129877
:10D1C00090ED300A80EE010A40F2FC30C2F200001D
:10D1D00080ED000A1299D1F8C8000D9BC3EB031231
:10D1E00000EB82009DED0B0AD1F8842002EB830254
:10D1F000D2ED000AD1ED041A9FED821A8DED051AC9
:10D20000FEF7A6FC9DED051A1298D0F8A4000D9922
:10D2100000EB810080ED000A1299D1F8CC000D9A44
:10D22000C2EB021300EB8300D1ED041A91ED220A48
:10D23000D1F8841001EB8201D1ED000AFEF788FCE1
:10D240001298D0F8A8000D9900EB810080ED000A3B
:10D2500012990D9AD1F8A400D1F8A81000EB820021
:10D2600001EB8201FFF7EEF912980D99D0F8A43086
:10D27000D0F8A820D0F8AC0003EB810393ED000AAE
:10D2800002EB810292ED001A30EE010A00EB810000
:10D2900080ED000A1298D0F8AC10D0F84C010D9A2D
:10D2A00000EB421001EB820191ED000AFCF7CEFE8B
:10D2B0001298D0F8B0000D9900EB810080ED000AC3
:10D2C00012994869D1F8B010C06A0D9A02EB820336
:10D2D00000EB430001EB820191ED000AFDF7F4FD44
:10D2E000FFE70D9801300D9048E7129901F1D00049
:10D2F00040F2A032C2F2000292ED000AD1ED041A0F
:10D30000D1ED1E0A9FEDCC1A8DED041AFEF720FC1C
:10D310009DED041A129880ED2D0A129901F5867080
:10D32000D1ED041AD1ED230A91ED2D0AFEF710FC80
:10D33000129880ED2E0A129901F5B87091ED2E0A1F
:10D34000FCF784FE129880ED2F0A1299486930305C
:10D3500091ED2F0AFDF7B8FD11988078C00750B9FC
:10D36000FFE71298FFF71AFD1298FFF7C3FD129915
:10D370000020087636E040F61B40C2F2000000783C
:10D38000C00770BBFFE71198C078C00748B3FFE73C
:10D390001299022008761298407E014603910128D6
:10D3A00008D0FFE70398022809D0FFE70398032875
:10D3B0000BD010E012990120A1F8A00010E0129902
:10D3C00048694069A1F8A0000AE0129941F60A20D4
:10D3D000A1F8A00004E012990020A1F8A000FFE746
:10D3E000FFE7FFE7FFE012981199FFF75FF90020D0
:10D3F0000A90FFE70A989DF84310884280F2AB80BC
:10D4000004E000BF0000000000C0DA451298406947
:10D41000C06A007A01388DF8270012984169C969FD
:10D420009DF8272001EB820191ED000A90ED301A62
:10D4300020EE010A9FED811A80EE010A8DED080AA7
:10D440001299D1F8C8000A9BC3EB031200EB8200CB
:10D450009DED080AD1F8842002EB8302D2ED000A88
:10D46000D1ED041A9FED741A8DED021AFEF770FBD0
:10D470009DED021A1298D0F8A4000A9900EB8100E1
:10D4800080ED000A1299D1F8CC000A9AC2EB02137F
:10D4900000EB8300D1ED041A91ED220AD1F884103B
:10D4A00001EB8201D1ED000AFEF752FB1298D0F891
:10D4B000A8000A9900EB810080ED000A12990A9AEF
:10D4C000D1F8A400D1F8A81000EB820001EB820192
:10D4D000FFF7B8F812980A99D0F8A430D0F8A8202D
:10D4E000D0F8AC0003EB810393ED000A02EB81025C
:10D4F00092ED001A30EE010A00EB810080ED000A87
:10D500001298D0F8AC10D0F84C010A9A00EB4210F7
:10D5100001EB820191ED000AFCF798FD1298D0F81A
:10D52000B0000A9900EB810080ED000A1299486969
:10D53000D1F8B010C06A0A9A02EB820300EB4300F4
:10D5400001EB820191ED000AFDF7BEFCFFE70A98AE
:10D5500001300A904EE7129901F1D000D1ED041A82
:10D56000D1ED1E0A91ED310A9FED331A8DED011AAE
:10D57000FEF7EEFA9DED011A129880ED2D0A129930
:10D5800001F58670D1ED041AD1ED230A91ED2D0A33
:10D59000FEF7DEFA129880ED2E0A129901F5B870A6
:10D5A00091ED2E0AFCF752FD129880ED2F0A129988
:10D5B0004869303091ED2F0AFDF786FC1198C0784C
:10D5C000C00758B9FFE71299012008761298806FBA
:10D5D00040F2A031C2F200010860FFE703E01299B7
:10D5E00000200876FFE7FFE712984069C06AFDF760
:10D5F00031FA129840694068052807D3FFE712986E
:10D600004069C06A2830FDF725FAFFE712984069A3
:10D610003030FDF71FFA1198C07800F0010040F695
:10D620001B41C2F20001087000208DF84F00FFE797
:10D630009DF94F0014B080BD0000000000C0DA4525
:10D6400083B001908DF80310019820B9FFE7FF2007
:10D650008DF80B000AE09DF80300019948760199C6
:10D660000020A1F8A0008DF80B00FFE79DF90B004A
:10D6700003B0704710B588B00690069820B9FFE750
:10D68000FF208DF81F004CE10020059006994969A4
:10D6900049688DF813100390FFE703989DF8131065
:10D6A000884280F29780FFE706984069C06A039934
:10D6B00001EB810100EB4100FDF794FC0698406905
:10D6C000C06A039901EB810100EB4100FDF7FCFA10
:10D6D0000290029898B1FFE70698D0F820E00398EE
:10D6E0000EEB00110401029BD3F82CC0186B5A6B8F
:10D6F0009B6B4EF804C0CB608A604860FFE70698D9
:10D70000016AD0F84801039A00EB421001EB0211C4
:10D7100091ED010AFCF79AFC0698C06F039900EBA3
:10D72000810080ED000A06980399C26FD0F884004A
:10D7300002EB810292ED000A9FED7F1A80EE010A52
:10D7400000EB810080ED000A0698D0F88400039970
:10D7500000EB810090ED000AB7EE001AB4EE410A2A
:10D76000F1EE10FA09DDFFE70698D0F88410039A6D
:10D770004FF07E5041F82200FFE70698D0F8840071
:10D78000039900EB810090ED000ABFEE001AB4EEA1
:10D79000410AF1EE10FA0ADAFFE70698D0F8841091
:10D7A000039A0020CBF6807041F82200FFE706982C
:10D7B000D0F88400039900EB810090ED001A9DEDF4
:10D7C000050A30EE010A8DED050AFFE703980130E6
:10D7D000039062E79DED050A9DF8130001EE100A23
:10D7E000B8EEC11A80EE010A069880ED220A06986A
:10D7F00040693030FDF7F6FB069800F128010191F1
:10D8000040693030FDF760FA014601985022F2F786
:10D8100008FE0698416991ED020A90ED1C1A20EE6F
:10D82000010A80ED1E0AFFE7069890ED1E0AB5EE8C
:10D83000400AF1EE10FA0ADAFFE7069890ED1E0AA8
:10D840009FED3A1A30EE010A80ED1E0AECE7FFE781
:10D85000069890ED1E0A9FED351AB4EE410AF1EEDE
:10D8600010FA0ADBFFE7069890ED1E0A9FED311AC9
:10D8700030EE010A80ED1E0AEAE7069890F85000A3
:10D88000C00750B1FFE7069890ED1E1A9FED270ADA
:10D8900030EE410A80ED1E0AFFE7069901F5A870F7
:10D8A00091ED0D0AFCF7D2FB069880ED200A069850
:10D8B00090ED0D0A9FED1E1A80EE010A80ED230AFD
:10D8C000069890ED230AB7EE001AB4EE410AF1EE85
:10D8D00010FA06DDFFE706994FF07E50C1F88C0084
:10D8E000FFE7069890ED230ABFEE001AB4EE410A56
:10D8F000F1EE10FA07DAFFE706990020CBF6807008
:10D90000C1F88C00FFE70698016A91ED010A91EDDC
:10D91000051A30EE410A80ED640A00208DF81F00E0
:10D92000FFE79DF91F0008B010BD00BFDB0FC94025
:10D9300000409C45DB0FC9C000C0DA4580B582B00D
:10D94000019003F007F803F0BBF802B080BD0000BF
:10D9500080B582B0009000980138B0F1807F03D389
:10D96000FFE70120019019E0009801384EF2140100
:10D97000CEF2000108604FF0FF300F2101F022FDD0
:10D980004EF21801CEF20001002008604EF21002A3
:10D99000CEF20002072111600190FFE7019802B06A
:10D9A00080BD000080B5F9F74BFA06F0B5F8012804
:10D9B00003D0FFE704F0CCFFFFE780BD80B594B053
:10D9C00008A83021F2F767FD002007900690059027
:10D9D00004900390FFE70020029043F64000C4F259
:10D9E0000200016841F080510160006800F0805041
:10D9F00002900298FFE7FFE70020019047F2000045
:10DA0000C4F20000016841F480410160006800F444
:10DA1000804001900198FFE7012008904FF480308A
:10DA2000099002200E904FF480010F910621109171
:10DA3000A821119112900420139008A8F9F794FCE2
:10DA400018B1FFE7F6F792FDFFE70F2003900220E1
:10DA50000490002005904FF4A05006904FF48050A1
:10DA6000079003A80521F9F7AFFA18B1FFE7F6F719
:10DA70007DFDFFE714B080BD4EF68851CEF2000167
:10DA8000086840F4700008607047000083B002909E
:10DA9000019102980068009002980021C4F20101EF
:10DAA000884225D0FFE70298B0F1804F20D0FFE7F1
:10DAB000029840F20041C4F20001884218D0FFE70A
:10DAC000029840F60001C4F20001884210D0FFE73E
:10DAD000029840F60041C4F20001884208D0FFE7F6
:10DAE000029840F20041C4F2010188420AD1FFE7E6
:10DAF000009820F070000090019841680098084359
:10DB00000090FFE702980021C4F20101884255D03D
:10DB1000FFE70298B0F1804F50D0FFE7029840F243
:10DB20000041C4F20001884248D0FFE7029840F665
:10DB30000001C4F20001884240D0FFE7029840F69D
:10DB40000041C4F20001884238D0FFE7029840F259
:10DB50000041C4F20101884230D0FFE7029844F24C
:10DB60000001C4F20101884228D0FFE7029844F284
:10DB70000041C4F20101884220D0FFE7029844F638
:10DB80000001C4F20101884218D0FFE7029841F673
:10DB90000001C4F20001884210D0FFE7029841F66C
:10DBA0000041C4F20001884208D0FFE7029842F227
:10DBB0000001C4F2000188420AD1FFE7009820F476
:10DBC000407000900198C168009808430090FFE7FA
:10DBD000009820F08000019949690843009001985D
:10DBE00080680299C8620198006802998862029868
:10DBF0000021C4F20101884208D0FFE7029840F2F8
:10DC00000041C4F20101884205D1FFE70198006993
:10DC100002990863FFE70299086840F00400086071
:10DC200002990120486100980299086003B070478A
:10DC300084B0039002910192029800F01F0101202C
:10DC400088400090009A0399086A904308620198FE
:10DC5000029901F01F0100FA01F20399086A1043CA
:10DC6000086204B07047000085B0049003910292EE
:10DC70000193049880680090009820F47F40009001
:10DC800003980299019A41EA02210143009808434E
:10DC9000009000980499886005B0704783B00290A6
:10DCA0000191029880680090009820F07000009028
:10DCB00001980099084340F00700009000980299ED
:10DCC000886003B07047000085B004900391049809
:10DCD000006A01900499086A20F001000862049823
:10DCE00040680090049880690290029820F07000CB
:10DCF0000290029820F003000290039801680298B5
:10DD000008430290019820F0020001900398816876
:10DD100001980843019004980021C4F2010188424F
:10DD200008D0FFE7049840F20041C4F201018842A4
:10DD30000ED1FFE7019820F0080001900398C16818
:10DD4000019808430190019820F004000190FFE73A
:10DD500004980021C4F20101884208D0FFE704982A
:10DD600040F20041C4F20101884213D1FFE700985C
:10DD700020F480700090009820F4007000900398C8
:10DD8000416900980843009003988169009808430E
:10DD90000090FFE700980499486002980499886110
:10DDA000039840680499486301980499086205B093
:10DDB0007047000085B0049003910498006A0190B8
:10DDC0000499086A20F010000862049840680090E6
:10DDD000049880690290029820F4E0400290029832
:10DDE00020F44070029003980168029840EA0120F4
:10DDF0000290019820F0200001900398816801981A
:10DE000040EA0110019004980021C4F20101884207
:10DE100008D0FFE7049840F20041C4F201018842B3
:10DE20000FD1FFE7019820F0800001900398C168AE
:10DE3000019840EA01100190019820F04000019003
:10DE4000FFE704980021C4F20101884208D0FFE7EF
:10DE5000049840F20041C4F20101884215D1FFE765
:10DE6000009820F480600090009820F400600090FA
:10DE700003984169009840EA810000900398816905
:10DE8000009840EA81000090FFE7009804994860FC
:10DE900002980499886103984068049988630198FE
:10DEA0000499086205B0704785B004900391049806
:10DEB000006A01900499086A20F48070086204984E
:10DEC000406800900498C0690290029820F07000A9
:10DED0000290029820F003000290039801680298D3
:10DEE00008430290019820F4007001900398816823
:10DEF000019840EA0120019004980021C4F2010138
:10DF0000884208D0FFE7049840F20041C4F20101C2
:10DF100088420FD1FFE7019820F400600190039838
:10DF2000C168019840EA01200190019820F48060C6
:10DF30000190FFE704980021C4F20101884208D053
:10DF4000FFE7049840F20041C4F20101884215D174
:10DF5000FFE7009820F480500090009820F40050D3
:10DF6000009003984169009840EA011000900398DE
:10DF70008169009840EA01100090FFE70098049939
:10DF8000486002980499C861039840680499C8637E
:10DF900001980499086205B07047000085B00490AC
:10DFA00003910498006A01900499086A20F4805053
:10DFB00008620498406800900498C0690290029832
:10DFC00020F4E0400290029820F440700290039800
:10DFD0000168029840EA01200290019820F4005064
:10DFE000019003988168019840EA013001900498FB
:10DFF0000021C4F20101884208D0FFE7049840F2F2
:10E000000041C4F2010188420BD1FFE7009820F4DF
:10E010008040009003984169009840EA8110009088
:10E02000FFE700980499486002980499C861039832
:10E0300040680499086401980499086205B0704723
:10E0400085B00490039102920498006A00900499AC
:10E05000086A20F001000862049880690190019824
:10E0600020F0F00001900299019840EA011001901F
:10E07000009820F00A00009003990098084300904F
:10E0800001980499886100980499086205B0704766
:10E0900085B00490039102920498006A009004995C
:10E0A000086A20F0100008620498806901900198C5
:10E0B00020F4704001900299019840EA01300190EB
:10E0C000009820F0A00000900399009840EA011009
:10E0D000009001980499886100980499086205B03D
:10E0E0007047000080B586B0059002F03FF84EF60C
:10E0F0003120C0F6000046F23C32C0F60102002199
:10E10000029102F02FFC029941F20C72C2F200025D
:10E11000049210604EF23920C0F6000046F2402210
:10E12000C0F6010202F01EFC0299049A50604EF201
:10E13000D940C0F6000046F26422C0F6010202F0A7
:10E1400011FC0299049A90604EF28170C0F60000B2
:10E1500046F2AC22C0F6010202F004FC0299049AD5
:10E16000D0604EF68100C0F6000046F2D022C0F624
:10E17000010202F0F7FB0299049A10614EF6791041
:10E18000C0F6000046F2F422C0F6010202F0EAFBFB
:10E190000299049A50614EF28950C0F6000046F28E
:10E1A0008822C0F6010202F0DDFB029A0499886120
:10E1B000022003900A2102F0C7F8029A0499C8616C
:10E1C000032000902C2102F0BFF8029A049B014624
:10E1D00000989963282102F0B7F8029A049B01463F
:10E1E000039859620421019102F0AEF8029A049B4F
:10E1F000014603989962182102F0A6F8029A049B3E
:10E2000001460398D9620C2102F09EF80199029A06
:10E21000DDF810C003460398CCF8303002F094F8D3
:10E220000499486301F0F8FF02F094FB02F048FC07
:10E2300006B080BD0000000080B58CB00B9001F0EE
:10E240006DFF07F0B6FB41EC100B9FED9D1B53ECEF
:10E25000112B51EC100B07F0E9F941EC100B51ECCC
:10E26000100B07F079FB0A900020089001F0D2FE15
:10E2700001F040FF099040F25840C2F200000790C0
:10E2800040F20801C2F20001F3F7E4FC0798F3F74B
:10E29000B9FC40F2D860C2F2000040F64841C2F238
:10E2A0000001F2F719FA0798F3F7ACFC0899B0EE01
:10E2B000401AB7EE000A80EE010A40F6DC30C2F2E6
:10E2C000000046F28432C0F60102FDF7B9FD0120DC
:10E2D000F4F7CAFE089841F69141C0F60101F4F73F
:10E2E000ABFD0898F4F756FDFFE70A990998084432
:10E2F0000990F3F7A3FEF3F76DFCF3F77BFCF3F75C
:10E3000093FCF3F79FFC01F031FF40F25840C2F25A
:10E3100000000690F3F762FD0698F3F7D9FD40F28E
:10E32000A040C2F200000078012865D1FFE740F26A
:10E330005841C2F2000191ED071A40F22870C2F272
:10E34000000090ED000A30EE010A80ED000A91ED28
:10E35000081A90ED010A30EE010A80ED010A91EDF4
:10E36000091A90ED020A30EE010A80ED020A40F22D
:10E370009E40C2F20000018801310180008841F214
:10E380008831884237DBFFE740F22870C2F2000094
:10E3900090ED000A9FED4C1A80EE010A40F2080150
:10E3A000C2F2000181ED000A90ED010A80EE010A3F
:10E3B00081ED010A90ED020A80EE010A81ED020A68
:10E3C00040F2A042C2F200020020107040F2584019
:10E3D000C2F200000590F3F73DFC0598F3F712FC3C
:10E3E00040F2D860C2F2000040F64841C2F200019B
:10E3F000F2F772F9FFE7FFE740F2A040C2F2000037
:10E40000007801281BD0FFE740F25840C2F200001C
:10E4100000F1100100F11C0240F2D860C2F20000CD
:10E42000049040F64843C2F20003F2F7A1FA0499BF
:10E4300040F22850C2F20000F2F7A0F8FFE701F026
:10E44000EBFE40F22851C2F2000108684A688B686E
:10E4500040F21071C2F2000101914B610A61C86083
:10E4600040F25843C2F200030393D8691A6A5B6A08
:10E470008B604A60086041F20C70C2F200000290AA
:10E48000C06A02F043F801990298C06A00231A4654
:10E4900001F0DAFF0398D0ED0A0A40F6DC30C2F250
:10E4A00000009FED0A0ADFED0A1AB0EE611AFDF7CF
:10E4B0004FFB0120F4F738FD099801F0C5FD14E782
:10E4C0000000000000407F4000409C4500002042CA
:10E4D000000000000000000080B586B0059001F04B
:10E4E0001DFE07F066FA41EC100B9FED231B53EC69
:10E4F000112B51EC100B07F099F841EC100B51EC7B
:10E50000100B07F029FA0490002001F083FD01F0C0
:10E51000F1FD03900420F4F7C9FD0220F4F7C6FDD5
:10E52000032001909FED160AF4F7FEFC0198F4F722
:10E530009BFDFFE704990398084403909DED030AAF
:10E54000B8EE400A9FED0F1A20EE010A06F062FCB9
:10E55000B7EE001A30EE010AB6EE001A20EE010AFC
:10E560008DED020A9DED020A0320F4F7DDFC03980D
:10E5700001F06AFDDEE700BF000000000000594026
:10E5800000000000A69B443B80B588B0079001F0D6
:10E59000C5FD07F00EFA41EC100B9FED771B53EC15
:10E5A000112B51EC100B07F041F841EC100B51EC22
:10E5B000100B07F0D1F90690002001F02BFD01F0BF
:10E5C00099FD0590FFE7069905980844059041F2EA
:10E5D0000C70C2F20000806B40F22C41C2F20001CC
:10E5E000039100231A4601F04FFE0398807E0146F6
:10E5F000049101282CD0FFE70498022804D0FFE7FB
:10E600000498032809D03EE040F21051C2F2000104
:10E6100000200870486088603EE040F21050C2F26E
:10E6200000000121017040F22C41C2F2000191ED85
:10E63000011AB1EE410A30EE410A80ED010A91ED76
:10E64000020ABFEE081A20EE010A80ED020A23E05A
:10E6500040F21050C2F200000121017040F22C4142
:10E66000C2F2000191ED011AB1EE410A30EE410A09
:10E6700080ED010A91ED020ABFEE081A20EE010AB0
:10E6800080ED020A08E040F21051C2F200010020C1
:10E69000087048608860FFE740F22C40C2F200003A
:10E6A000807D01460291012829D0FFE702980228C7
:10E6B00004D0FFE70298032810D030E040F22C404D
:10E6C000C2F20000007800F0010040F21C51C2F2DA
:10E6D0000001087001208870C87030E040F22C40C2
:10E6E000C2F20000007800F0010040F21C51C2F2BA
:10E6F00000010870012088700020C8701FE040F2FF
:10E700002C40C2F20000007800F0010040F21C51E1
:10E71000C2F20001087000208870C8700FE040F25B
:10E720002C40C2F20000007800F0010040F21C51C1
:10E73000C2F20001087000208870C870FFE741F243
:10E740000C70C2F200000190006B40F21051C2F256
:10E750000001002300931A4601F076FE009B019809
:10E76000406B40F21C51C2F200011A4601F06CFEEF
:10E77000059801F069FC26E70000000000407F409A
:10E780002DE9F0418EB00D9001F0C8FC07F011F9B1
:10E7900041EC100B9FED361B53EC112B51EC100B81
:10E7A00006F044FF41EC100B51EC100B07F0D4F8CD
:10E7B0000C90002001F02EFC01F09CFC0B909FEDD2
:10E7C0002E0AFDF711F8FFE70C990B9808440B90FF
:10E7D00041F20C70C2F200000890406A40F2B4416D
:10E7E000C2F200010991002307931A4601F04CFD83
:10E7F000079B0898806A40F2DC41C2F200010A914E
:10E8000004311A4601F040FDDDF824E00A9842F692
:10E81000F601C4F28401016090ED000AD0ED010A16
:10E82000DEF80000DEF80410DEF80820DEF80C3018
:10E83000DEF810C0DEF81440DEF81850DEF81C6078
:10E84000DEF82070DEF82480EE46CEF81480CEF894
:10E850001070CEF80C60CEF80850CEF80440CEF818
:10E8600000C000F011FE0B9801F0EEFBACE700BF1A
:10E870000000000000407F400000FA43000000005C
:10E8800080B588B0079001F049FC07F092F841ECA0
:10E89000100B9FED351B53EC112B51EC100B06F0B8
:10E8A000C5FE41EC100B51EC100B07F055F806902B
:10E8B000002001F0AFFB01F01DFC0590F4F74CFFC8
:10E8C00000F5847140F23850C2F200009FED280A32
:10E8D000F6F734F8FFE7069905980844059041F2E9
:10E8E0000C70C2F20000C06A40F2F861C2F200018E
:10E8F00000231A4601F0C8FC58B9FFE740F238502F
:10E90000C2F2000040F2F861C2F20001F6F78AF9A3
:10E91000FFE741F20C70C2F200000290006B40F27F
:10E92000EC61C2F200010391002301931A4601F049
:10E93000ABFC40F23850C2F200000490F6F71EF92A
:10E94000019B04990298806A01F5C0711A4601F092
:10E950007BFD03990498F5F70DFE0498F6F77CF813
:10E96000059801F071FBB6E70000000000407F4011
:10E970000000FA430000000080B586B0059001F069
:10E98000CDFB07F016F841EC100B9FED251B53EC67
:10E99000112B51EC100B06F049FE41EC100B51EC21
:10E9A000100B06F0D9FF0490002001F033FB01F0BA
:10E9B000A1FB0390F4F7D6FEF4F7CEFE014641F238
:10E9C0006050C2F2000002909FED170AFDF768FF49
:10E9D00002980221FEF734FEFFE7049903980844E9
:10E9E000039041F20C70C2F20000406B41F2F861FA
:10E9F000C2F20001009100231A4601F045FC41F2E9
:10EA00006050C2F200000190FEF734FE00990198B8
:10EA1000FDF7F4FE039801F017FBDEE700BF00BF2F
:10EA20000000000000407F400000FA4300000000AA
:10EA300080B588B0079001F071FB06F0BAFF41EC99
:10EA4000100B9FED2F1B53EC112B51EC100B06F00C
:10EA5000EDFD41EC100B51EC100B06F07DFF069024
:10EA6000002001F0D7FA01F045FB059040F200408C
:10EA7000C2F20000F4F70EFF40F2F440C2F20000D0
:10EA8000F5F738FCFFE706990598084405900A2039
:10EA9000F5F748FCB8B1FFE740F2F440C2F20000DD
:10EAA000049040F20041C2F200010391F4F72CFF00
:10EAB000039841F23851C2F20001F4F753FD049873
:10EAC000F5F718FCFFE741F20C70C2F2000002906B
:10EAD000806B40F20041C2F20001002301931A460C
:10EAE00001F0B2FC019B0298406A41F23851C2F237
:10EAF00000011A4601F0A8FC059801F0A5FAC2E74A
:10EB00000000000000407F4080B582B00190019875
:10EB1000806B009000990020C8850098FAF7B6FD38
:10EB200002B080BD80B584B00390002002900398AD
:10EB3000806B0190019800684069C0B2C0090290E2
:10EB4000019890F8410021280AD1FFE7029838B1D6
:10EB5000FFE701990020C884019800F013F9FFE74E
:10EB6000019800684069C0F380100290019890F805
:10EB7000420022280AD1FFE7029838B1FFE7019945
:10EB80000020C885019800F09FF8FFE70199486CC4
:10EB900040F0100048640198FAF778FD04B080BD99
:10EBA00080B586B005900598806B04900598006844
:10EBB0000068C00500285AD4FFE704990020C885E2
:10EBC000FFE7FFE70498006850E8030F20F4807027
:10EBD0000390FFE703990498026842E803100028B5
:10EBE000F0D1FFE7FFE7FFE7FFE70498006850E890
:10EBF000050F20F001000290FFE7029904980268D7
:10EC000042E805100028F0D1FFE7FFE7FFE7FFE744
:10EC10000498006850E8050F20F040000190FFE7DD
:10EC200001990498026842E805100028F0D1FFE736
:10EC3000FFE70499202081F842000498006B012826
:10EC400014D1FFE7FFE7FFE70498006850E8030FDF
:10EC500020F010000090FFE700990498026842E855
:10EC600003100028F0D1FFE7FFE7FFE7FFE7049973
:10EC7000002048630498006B012805D1FFE7049841
:10EC8000818DFAF7FDFC03E00498FBF7E3F8FFE75A
:10EC900006B080BD80B582B001900198806B009075
:10ECA0000099012048630098006B012806D1FFE716
:10ECB0000098818D4908FAF7E3FC03E00098FBF720
:10ECC000F3F8FFE702B080BD84B00390FFE7FFE7F1
:10ECD0000398006850E8030F20F490700290FFE75B
:10ECE00002990398026842E803100028F0D1FFE778
:10ECF000FFE7FFE7FFE70398006850E8050F20F003
:10ED000001000190FFE701990398026842E80510AD
:10ED10000028F0D1FFE7FFE70398006B012814D12A
:10ED2000FFE7FFE7FFE70398006850E8030F20F0D4
:10ED300010000090FFE700990398026842E8031072
:10ED40000028F0D1FFE7FFE7FFE70399202081F8D3
:10ED5000420003990020086304B0704780B582B078
:10ED6000019001980168C86820F04000C8600199CE
:10ED7000202081F841000198FBF7C0F8002002B084
:10ED800080BD000082B00190FFE7FFE701980068B6
:10ED900050E8030F20F0C0000090FFE700990198B1
:10EDA000026842E803100028F0D1FFE7FFE701996D
:10EDB000202081F8410002B07047000082B000902E
:10EDC0000098006844F60001C4F20001884204D1B2
:10EDD000FFE700208DF8070010E00098006841F27E
:10EDE0000041C4F20101884204D1FFE701208DF8FF
:10EDF000070003E003208DF80700FFE79DF80700F8
:10EE000002B0704780B586B0049000200390029055
:10EE1000049890F84200222840F0A080FFE7049870
:10EE20008068B0F5805F13D1FFE70498006978B976
:10EE3000FFE70498806A02900498006840686FF3C6
:10EE40005F20029908800499886A0230886223E072
:10EE50000498806A039004988068B0F5805F08D0B9
:10EE6000FFE70498806850B9FFE70498006930B95B
:10EE7000FFE70498006840680399087007E0049869
:10EE80000068406800F07F0003990870FFE704996C
:10EE9000886A01308862FFE70499C88D0138C88507
:10EEA0000004002856D1FFE704980168C86820F0E4
:10EEB0002000C86004980168C86820F48070C860A9
:10EEC00004980168486920F00100486104992020F5
:10EED00081F842000499002048630498006B0128DF
:10EEE00030D1FFE7049900200863FFE7FFE70498AB
:10EEF000006850E8030F20F010000190FFE701992F
:10EF00000498026842E803100028F0D1FFE7FFE709
:10EF1000049800680068C00600280ED5FFE7FFE7E8
:10EF20000020009004980068006800900498006831
:10EF3000406800900098FFE7FFE70498818DFAF79A
:10EF40009FFB03E00498FAF785FFFFE700208DF8A8
:10EF5000170007E000208DF8170003E002208DF86D
:10EF60001700FFE79DF8170006B080BD80B586B09A
:10EF7000059005980068006920F44050059A1168D2
:10EF8000D26810430861059988680B694A69C969A4
:10EF9000184310430843049005980068C06849F27C
:10EFA0000C6188430499084305990968C86005986D
:10EFB0000068406920F44070059A11689269104316
:10EFC00048610598006841F20001C4F201018842DD
:10EFD00009D0FFE70598006841F20041C4F2010141
:10EFE000884204D1FFE7F8F739F9039003E0F8F716
:10EFF00023F90390FFE70598C069B0F5004F29D1C8
:10F00000FFE703981921A0FB0101059A13680293F9
:10F0100053685A00DB0FF1F747F90299864648F228
:10F020001F53C5F2EB13AEFB0320420910014FF052
:10F03000640C02FB1CEC322202EBCC02A2FB03327A
:10F04000F82303EA521300EB4300C2F342121044C8
:10F05000886026E003981921A0FB0101059A136836
:10F06000019353689A009B0FF1F71EF901998446AA
:10F0700048F21F52C5F2EB12ACFB02304309642088
:10F0800003FB10CC322000EB0C10A0FB0202F0209E
:10F0900000EA521000EB0310C2F3431210448860E0
:10F0A000FFE706B080BD000080B58AB008900791E8
:10F0B000ADF81A20079808998862BDF81A000899D7
:10F0C0008885089900204864089A222182F8421015
:10F0D0000899CA6B4EF6A131C0F60001D1630899B8
:10F0E000CA6B4EF69541C0F6000111640899CA6BCF
:10F0F0004EF62531C0F60001D1640899C96B086548
:10F1000007A8059008980168C06B0431059A126839
:10F11000BDF81A30F7F7BEF958B1FFE7089910208B
:10F1200048640899202081F8420001208DF82700CA
:10F130004EE0FFE700200490089800680068049003
:10F1400008980068406804900498FFE708980069F0
:10F15000A0B1FFE7FFE7FFE70898006850E8030F5A
:10F1600040F480700390FFE703990898026842E832
:10F1700003100028F0D1FFE7FFE7FFE7FFE7FFE715
:10F180000898006850E8050F40F001000290FFE782
:10F1900002990898026842E805100028F0D1FFE7BC
:10F1A000FFE7FFE7FFE70898006850E8050F40F029
:10F1B00040000190FFE701990898026842E80510B5
:10F1C0000028F0D1FFE7FFE700208DF82700FFE7D8
:10F1D0009DF827000AB080BD83B00190019890F897
:10F1E000410021283AD1FFE701988068B0F5805F9F
:10F1F00013D1FFE70198006978B9FFE70198006A29
:10F200000090009800886FF35F20019909684860BA
:10F210000199086A0230086208E0019A106A411CEC
:10F2200011620078019909684860FFE70199C88C6C
:10F230000138C884000468B9FFE701980168C8680C
:10F2400020F08000C86001980168C86840F0400064
:10F25000C860FFE700208DF80B0003E002208DF866
:10F260000B00FFE79DF80B0003B0704780B582B03C
:10F2700040F69030C2F200000190FAF731FA01989E
:10F28000F4F7AAF802B080BDFFE7FEE782B041ECD8
:10F29000100B8DED000B0198C0F30A5040F2FF7186
:10F2A000401A18BF012002B07047000082B041EC44
:10F2B000100B8DED000B0198C0F30A5040F2FF7166
:10F2C000401A18BF012002B07047000081B000EE64
:10F2D000100A00900098C0F3C750FF3818BF0120F3
:10F2E00001B0704781B000EE100A00900098C0F3A2
:10F2F000C750FF3818BF012001B0704784B041ECFF
:10F30000100B8DED020B039A00200021CFF6E07167
:10F31000B1EB420F019006D1FFE70298B0FA80F0FE
:10F3200040090190FFE7019800F0010004B0704728
:10F3300081B000EE100A009000994FF0807000EB51
:10F340004100B0FA80F0400901B0704781B08DF8FB
:10F3500003009DF90300002812D4FFE79DF9031074
:10F3600001F01F02012090404A094EF28011CEF2B6
:10F37000000141F82200BFF34F8FBFF36F8FFFE70B
:10F3800001B0704781B08DF803009DF9030000289B
:10F390000ED4FFE79DF9031001F01F0201209040F9
:10F3A0004A094EF20011CEF2000141F82200FFE7B7
:10F3B00001B070474EF60C50CEF200000068C0F36A
:10F3C0000220704782B08DF8070000919DF9070078
:10F3D00000280AD4FFE7009800019DF907104EF2BB
:10F3E0000042CEF2000288540BE0009800019DF824
:10F3F000071001F00F014EF61452CEF200028854AD
:10F40000FFE702B07047000082B08DF8070000915E
:10F410009DF9070000280AD4FFE7009800019DF934
:10F4200007104EF20042CEF2000288540BE0009822
:10F4300000019DF8071001F00F014EF61452CEF2B4
:10F4400000028854FFE702B07047000083B00290CA
:10F45000029800F0070000904EF60C51CEF2000129
:10F460000868019001984FF6FF0210400190019842
:10F47000009A40EA02200022C0F2FA5210430190A2
:10F480000198086003B070472DE9F041A8B0339FA0
:10F49000329E319D309CDDF8BCE0DDF8B8C0CDED8A
:10F4A000270A8DED260A2597249623952294CDF8D8
:10F4B00084E0CDF880C01F931E921D911C90F3F73D
:10F4C00015FF06F04EFD00EE100A9FEDEA1A8DEDD5
:10F4D0000E1A80EE010A10EE100A06F0CBFD0A4665
:10F4E00040F69841C2F200014A600860F3F7FEFE60
:10F4F00040F62042C2F200020F9213685268C01A0E
:10F50000914106F02EFD9DED0E1A00EE100A80EEE0
:10F51000010A40F22450C2F2000080ED000AF3F725
:10F52000E5FE0A460F994A60086000201890FFE740
:10F53000189803282DDCFFE7189940F21400C2F256
:10F5400000000D9000EBC100FBF74CFD0D981899E1
:10F5500000EBC100FBF7B8FB17901798A0B1FFE7CD
:10F56000189840F6544EC2F2000E0EEB0011040142
:10F57000179BD3F82CC0186B5A6B9B6B4EF804C0CA
:10F58000CB608A604860FFE7FFE718980130189069
:10F59000CEE79DF9710001460C91032800F20A8123
:10F5A0000C99DFE801F0021368C148F29861C2F2D9
:10F5B00000010020086048F29C61C2F2000108606E
:10F5C00048F2A061C2F200010860F4E09DED261A45
:10F5D0009DED270A30EE410A8DED1B0A9DED1B0AB9
:10F5E00005F070FB8DED1A0A9DED1B0A05F012FC6B
:10F5F0008DED190A9DED1A0A9DED211A9DED222A25
:10F6000020EE010A9DED191A21EE021A30EE410A90
:10F6100048F29860C2F2000080ED000A9DED190AE0
:10F620009DED211A9DED222A20EE010A9DED1A1A68
:10F6300021EE021A30EE010A48F29C60C2F200008C
:10F6400080ED000A9DED260ADDED270A40F22450E8
:10F65000C2F20000D0ED001A40F6A040C2F2000055
:10F660009FED851AFCF774FA48F2A060C2F2000020
:10F6700080ED000A9FE040F6A040C2F200000B902F
:10F68000FCF7CEFC9DED261A9DED270A30EE410ACF
:10F690008DED1B0A9DED1B0A05F014FB8DED1A0A7A
:10F6A0009DED1B0A05F0B6FB0B988DED190A9DED3B
:10F6B0001A0A9DED211A9DED222A20EE010A9DEDE8
:10F6C000191A21EE021A30EE410A48F29861C2F28C
:10F6D000000181ED000A9DED190A9DED211A9DEDB5
:10F6E000222A20EE010A9DED1A1A21EE021A30EEAE
:10F6F000010A48F29C61C2F2000181ED000A9DED11
:10F70000260ADDED270A40F22451C2F20001D1EDB4
:10F71000001A9FED591AFCF71BFA48F2A060C2F2DA
:10F72000000080ED000A46E09DED261A9DED270AB7
:10F7300030EE410A8DED1B0A9DED1B0A05F0C2FA61
:10F740008DED1A0A9DED1B0A05F064FB8DED190A7B
:10F750009DED1A0A9DED211A9DED222A20EE010A47
:10F760009DED191A21EE021A30EE410A48F2986016
:10F77000C2F2000080ED000A9DED190A9DED211AEC
:10F780009DED222A20EE010A9DED1A1A21EE021AA1
:10F7900030EE010A48F29C60C2F2000080ED000ADF
:10F7A00048F2A061C2F2000149F69A10C3F619703E
:10F7B000086000E0FFE748F29860C2F2000090EDB8
:10F7C000000A48F29C60C2F20000D0ED000A48F244
:10F7D000A060C2F2000090ED001AFAF7F7FB0020DB
:10F7E00016908DF85700FFE79DF9570003282DDC90
:10F7F000FFE79DF9571040F2EC30C2F2000000EB39
:10F80000810090ED000AB0EEC00A8DED140A9DED66
:10F81000140A9DED161AB4EE410AF1EE10FA05DD58
:10F82000FFE79DED140A8DED0A0A04E09DED160A2E
:10F830008DED0A0AFFE79DED0A0A8DED160AFFE736
:10F840009DF8570001308DF85700CDE79DED160A61
:10F85000B7EE001AB4EE410AF1EE10FA30DDFFE720
:10F8600000208DF84F00FFE79DF94F00032826DCAC
:10F870000EE000BF002474490000000000BF00BF7C
:10F88000158C4AEA04343340000000000058BB40A5
:10F890009DED161A9DF94F1040F2EC30C2F20000B7
:10F8A00000EB810090ED000A80EE010A80ED000A75
:10F8B000FFE79DF84F0001308DF84F00D4E7FFE7D8
:10F8C0009DF9710001460991032800F28D82099982
:10F8D000DFE811F0040021001001CD0140F6BC600A
:10F8E000C2F200000890FCF79BFB08983C30FCF744
:10F8F00097FB08987830FCF793FB0898B430FCF736
:10F900008FFB40F2E441C2F2000100200860486031
:10F910008860C86069E240F6BC60C2F200000790EF
:10F92000FCF77EFB07983C30FCF77AFB07987830B1
:10F93000FCF776FB0798B430FCF772FB00201290BE
:10F94000FFE71298032800F3D480FFE7129906918D
:10F9500040F65440C2F2000000EB0110406806F08F
:10F96000ABFA41EC100B51EC100B1FED3B0B53ECC1
:10F97000102B06F0A9F841EC100B51EC100B1FED09
:10F980003E0B53EC102B05F051FE41EC100B51ECEB
:10F99000100B05F065FD069A014641F2FC60C2F2CB
:10F9A000000040F82210129900EB810090ED000A4F
:10F9B000B7EE001AB4EE410AF1EE10FA0ADDFFE7E5
:10F9C000129A41F2FC61C2F200014FF07E5041F800
:10F9D00022001CE0129941F2FC60C2F2000000EB30
:10F9E000810090ED000ABFEE001AB4EE410AF1EE7C
:10F9F00010FA0BDAFFE7129A41F2FC61C2F2000141
:10FA00000020CBF6807041F82200FFE7FFE7129A52
:10FA1000C2EB021140F6DC40C2F2000000EB8100B4
:10FA200040F62841C2F2000101EB820191ED000A8B
:10FA300040F65441C2F2000101EB0211D1ED000A7F
:10FA400040F22451C2F200010491D1ED001A1FEDE1
:10FA5000761A8DED051AFCF77BF804999DED051AD1
:10FA6000129840F63842C2F2000202EB800080EDAC
:10FA7000000A129BC3EB031C40F6CC50C2F20000FC
:10FA800000EB8C0002EB830292ED000A41F2FC6273
:10FA9000C2F2000202EB8302D2ED000AD1ED001A9D
:10FAA000FCF756F8129940F2E440C2F2000000EB75
:10FAB000810181ED000A129900EB810090ED000AAE
:10FAC0009FEDE41AB4EE410AF1EE10FA0CDDFFE707
:10FAD000129A40F2E441C2F200014CF6CD40C3F666
:10FAE0004C7041F82200FFE7FFE7129801301290B6
:10FAF00027E77AE100201190FFE71198032800F32F
:10FB0000B580FFE7119B190140F65440C2F2000096
:10FB1000415840F62842C2F2000242F823101199DF
:10FB2000039100EB0110406806F0C6F941EC100BA0
:10FB300051EC100B9FEDC20B53EC102B05F0C4FFE2
:10FB400041EC100B51EC100B9FEDBF0B53EC102B45
:10FB500005F06CFD41EC100B51EC100B05F080FC36
:10FB6000039A014641F2FC60C2F2000040F8221004
:10FB7000119900EB810090ED000AB7EE001AB4EE87
:10FB8000410AF1EE10FA0ADDFFE7119A41F2FC6139
:10FB9000C2F200014FF07E5041F822001CE01199A2
:10FBA00041F2FC60C2F2000000EB810090ED000A1F
:10FBB000BFEE001AB4EE410AF1EE10FA0BDAFFE7DD
:10FBC000119A41F2FC61C2F200010020CBF6807074
:10FBD00041F82200FFE7FFE7119AC2EB021140F65D
:10FBE000BC60C2F2000000EB810040F2EC31C2F2D6
:10FBF000000101EB820191ED000A41F2FC61C2F2C9
:10FC0000000101EB8201D1ED000A40F22451C2F261
:10FC10000001D1ED001A9FED8E1AFBF799FF1199A3
:10FC200040F2E440C2F2000000EB810181ED000AE5
:10FC3000119900EB810090ED000A9FED861AB4EE59
:10FC4000410AF1EE10FA0CDDFFE7119A40F2E441AF
:10FC5000C2F200014CF6CD40C3F64C7041F82200D0
:10FC6000FFE7FFE711980130119046E7BDE0002063
:10FC70001090FFE71098032800F3B580FFE7109B72
:10FC8000190140F65440C2F20000415840F62842A3
:10FC9000C2F2000242F823101099029100EB011009
:10FCA000406806F009F941EC100B51EC100B9FED88
:10FCB000640B53EC102B05F007FF41EC100B51ECDB
:10FCC000100B9FED610B53EC102B05F0AFFC41ECDA
:10FCD000100B51EC100B05F0C3FB029A014641F2E8
:10FCE000FC60C2F2000040F82210109900EB810085
:10FCF00090ED000AB7EE001AB4EE410AF1EE10FAE8
:10FD00000ADDFFE7109A41F2FC61C2F200014FF0F8
:10FD10007E5041F822001CE0109941F2FC60C2F2D2
:10FD2000000000EB810090ED000ABFEE001AB4EE77
:10FD3000410AF1EE10FA0BDAFFE7109A41F2FC618A
:10FD4000C2F200010020CBF6807041F82200FFE7EC
:10FD5000FFE7109AC2EB021140F6BC60C2F200004D
:10FD600000EB810040F2EC31C2F2000101EB8201B4
:10FD700091ED000A41F2FC61C2F2000101EB820147
:10FD8000D1ED000A40F22451C2F20001D1ED001A77
:10FD90009FED2F1AFBF7DCFE109940F2E440C2F20F
:10FDA000000000EB810181ED000A109900EB810059
:10FDB00090ED000A9FED271AB4EE410AF1EE10FA19
:10FDC0000CDDFFE7109A40F2E441C2F200014CF66C
:10FDD000CD40C3F64C7041F82200FFE7FFE71098D2
:10FDE0000130109046E700E0FFE740F2E440C2F245
:10FDF0000000009090ED000A40F21400C2F20000F2
:10FE00000190FBF761F80099019891ED010A083023
:10FE1000FBF75AF80099019891ED020A1030FBF7B0
:10FE200053F80099019891ED030A1830FBF74CF84C
:10FE30000198FAF70FFE28B0BDE8F08100BF00BFBF
:10FE4000158C4AEA04343340000000000058BB40DF
:10FE500000000000CDCC4C3F82B08DED010ACDED0D
:10FE6000000A01980099C90F61F3DF7001909DEDC0
:10FE7000010A02B07047000080B588B0069006986D
:10FE80000190019858B9FFE74FF0500080F31188B6
:10FE9000BFF36F8FBFF34F8F0790FFE7FEE7019827
:10FEA00041F2A001C2F200010968884204D1FFE7D3
:10FEB00000208DF8170056E001F0FEFF0198406920
:10FEC000049041F2A800C2F200000068039041F2E1
:10FED000B000C2F200000068029002F019F8049825
:10FEE0000399884205D0FFE704980299884204D11B
:10FEF000FFE702208DF8170034E0049848F278718B
:10FF0000C2F20001884218D1FFE70198806A78B9EF
:10FF1000FFE7019890F85800012804D1FFE702207C
:10FF20008DF8170003E003208DF81700FFE703E0CA
:10FF300002208DF81700FFE713E0049848F28C7157
:10FF4000C2F20001884203D0FFE7049820B9FFE71E
:10FF500004208DF8170003E001208DF81700FFE75B
:10FF6000FFE7FFE7FFE79DF8170008B080BD00003E
:10FF700086B08DED050ACDED040A8DED031A0290D1
:10FF80009DED030A9DED041A30EE410A8DED010A44
:10FF9000049800909DED050A9DED001A30EE410A8F
:10FFA000029901208840013801EE100AB8EEC11A0A
:10FFB00020EE010A9DED011A80EE010ABDEEC00A95
:10FFC00010EE100A06B0704780B582B00020019094
:10FFD000F6F744FFFDF7F2FCFBF754F9FBF7D4F812
:10FFE000FBF782F8FBF7A8F8FBF750FAFBF79CFA4F
:10FFF000FBF770FAFBF7B4FBFBF7D4FBFBF7DCFA7B
:020000040801F1
:10000000FBF728FB00F08EF8FBF71CF900F0DAF89C
:10001000FFE7FEE780B584B00290EFF30580039020
:10002000039820B1FFE76FF00500019009E0002080
:100030000190029820B1FFE7029802F0B7F8FFE7BD
:10004000FFE7019804B080BD80B586B00490EFF35F
:1000500005800590059820B1FFE76FF0050001903D
:100060001BE00020019003F073FD039004980399B6
:10007000401A0290029858B1FFE702990020B0EBB5
:10008000D17F05D1FFE7029903A802F0C7F803E08A
:100090006FF003000190FFE7FFE7019806B080BD15
:1000A00080B582B003F038FD0146009158B1FFE7FA
:1000B000009801280AD0FFE70098022807D1FFE73F
:1000C0000220019012E0032001900FE0FFE740F2D0
:1000D0007C30C2F200000068012803D1FFE7012054
:1000E000019002E000200190FFE7FFE7019802B0D5
:1000F00080BD000080B582B0EFF3058001900198CB
:1001000020B1FFE703F02EFD009003E003F020FD97
:100110000090FFE7009802B080BD00004FF47A70B5
:100120007047000082B0EFF305800190019820B184
:10013000FFE76FF00500009014E040F27C30C2F25F
:100140000000006848B9FFE740F27C31C2F20001CC
:10015000012008600020009003E04FF0FF30009085
:10016000FFE7FFE7009802B07047000080B584B059
:10017000EFF305800390039820B1FFE76FF00500CF
:1001800002901BE003F0C8FC0146019140B1FFE77B
:10019000019801280CD0FFE70198022803D008E05D
:1001A0000120029009E002F0BBFA0020029004E076
:1001B000FFE74FF0FF300290FFE7FFE7029804B03F
:1001C00080BD000080B582B0EFF3058001900198FA
:1001D00020B1FFE76FF00500009019E040F27C309D
:1001E000C2F20000006801280DD1FFE7FCF722FAF7
:1001F00040F27C31C2F200010220086002F020FAD5
:100200000020009003E04FF0FF300090FFE7FFE791
:10021000009802B080BD000080B584B0EFF3058087
:100220000390039820B1FFE76FF00500029027E0EC
:1002300003F072FC0146019140B1FFE701980128EB
:1002400018D0FFE70198022811D014E00120029095
:1002500003F04CFF012809D0FFE703F05DFC20B953
:10026000FFE74FF0FF300290FFE7FFE707E00020D5
:10027000029004E0FFE74FF0FF300290FFE7FFE756
:10028000029804B080BD000080B588B0069005914A
:10029000049203930698029000200190EFF30580EA
:1002A0000790079868B3FFE7029830B1FFE7059819
:1002B00018B1FFE7039820B1FFE76FF0030001904A
:1002C0001EE000200090029805996A4602F08CFF1B
:1002D000012804D0FFE76FF0020001900FE00098C2
:1002E00060B1FFE74EF60451CEF200014FF08050AE
:1002F0000860BFF34F8FBFF36F8FFFE7FFE7FFE7A4
:100300001FE0029818B1FFE7059820B9FFE76FF0EA
:100310000300019014E002980599039A02F076FE1A
:1003200001280CD0FFE7039820B1FFE76FF0010030
:10033000019003E06FF002000190FFE7FFE7FFE7A5
:10034000FFE7019808B080BD80B588B006900591A0
:10035000049200200390EFF305800790079800288F
:100360006ED1FFE7069800286AD0FFE705980028BD
:1003700066D0FFE74FF0FF300290049868B3FFE7C4
:1003800004988068A0B1FFE70498C06850280FD394
:10039000FFE70498006958B1FFE70498406906999F
:1003A000059A5143884203D3FFE70120029013E0EE
:1003B0000498806878B9FFE70498C06858B9FFE7E7
:1003C0000498006938B9FFE70498406918B9FFE755
:1003D00000200290FFE7FFE702E000200290FFE725
:1003E000029801280ED1FFE706980599049A9368B0
:1003F0001269EE464FF0000CCEF800C002F02EFB62
:1004000003900AE0029838B9FFE7069805990022A0
:1004100002F0EAFA0390FFE7FFE7039878B1FFE7FD
:10042000049820B1FFE704980068019002E00020E2
:100430000190FFE70398019901F05CFEFFE7FFE7F9
:10044000039808B080BD000080B588B00690059183
:100450008DF8132003930698029000200190EFF38B
:1004600005800790079868B3FFE7029830B1FFE76F
:10047000059818B1FFE7039820B1FFE76FF003007C
:1004800001901EE000230093029805996A4602F04D
:10049000E1FC012804D0FFE76FF0020001900FE0BB
:1004A000009860B1FFE74EF60451CEF200014FF024
:1004B00080500860BFF34F8FBFF36F8FFFE7FFE7F8
:1004C000FFE720E0029818B1FFE7059820B9FFE7A1
:1004D0006FF00300019015E002980599039A00233C
:1004E00002F0A2FB01280CD0FFE7039820B1FFE740
:1004F0006FF00100019003E06FF002000190FFE750
:10050000FFE7FFE7FFE7019808B080BD80B584B042
:10051000029002980190EFF305800390039820B1B8
:10052000FFE76FF0050000900DE0019820B9FFE7AC
:100530006FF00300009005E000210091019802F0A7
:1005400015FBFFE7FFE7009804B080BD80B586B0DB
:1005500004900391049820F001000290049800F0A8
:100560000100009000200190EFF3058005900598B0
:1005700020B1FFE76FF00500019033E0029820B949
:10058000FFE76FF0030001902BE00098A0B1FFE7B8
:100590000298039902F0C2FF01280CD0FFE70398EC
:1005A00020B1FFE76FF00100019003E06FF002005F
:1005B0000190FFE7FFE713E00298039902F098FE2D
:1005C00001280CD0FFE7039820B1FFE76FF001008E
:1005D000019003E06FF002000190FFE7FFE7FFE703
:1005E000FFE7FFE7019806B080BD000080B588B046
:1005F000069000200590EFF30580079007980028EB
:1006000040F08580FFE7069820B1FFE70698406834
:10061000049002E000200490FFE79DF81000C0075E
:1006200018B1FFE70120039002E000200390FFE7EC
:10063000049800F00800082868D0FFE74FF0FF306A
:1006400002900698C8B1FFE70698806840B1FFE7BE
:100650000698C068502803D3FFE7012002900BE002
:100660000698806838B9FFE70698C06818B9FFE7B0
:1006700000200290FFE7FFE702E000200290FFE782
:100680000298012812D1FFE7039838B1FFE70698D6
:100690008168042002F08EF9059006E006988168D2
:1006A000012002F087F90590FFE711E0029870B988
:1006B000FFE7039828B1FFE7042002F067F90590EF
:1006C00004E0012002F062F90590FFE7FFE7FFE791
:1006D000059878B1FFE7069820B1FFE70698006813
:1006E000019002E000200190FFE70598019901F0D8
:1006F00001FDFFE7059840B1FFE7039828B1FFE748
:10070000059840F001000590FFE7FFE7FFE7059837
:1007100008B080BD80B586B00490049820F0010038
:100720000390049800F00100019000200290EFF384
:1007300005800590059820B1FFE76FF00500029055
:1007400024E0039820B9FFE76FF0030002901CE05B
:10075000019858B1FFE7039802F022FC012804D069
:10076000FFE76FF002000290FFE70DE0039800231F
:1007700019461A4602F058FA012804D0FFE76FF034
:1007800002000290FFE7FFE7FFE7FFE7029806B0ED
:1007900080BD000080B58AB0089007910898069047
:1007A000069830B1FFE79DF81F000006002804D529
:1007B000FFE76FF0030005903BE04FF0FF3005903E
:1007C000EFF305800990099820B3FFE70023039316
:1007D000049306980799EC4604AACCF8002001225D
:1007E00003F0AEF8039A069869460A6005AB114615
:1007F00003F0A6F8049860B1FFE74EF60451CEF27C
:1008000000014FF080500860BFF34F8FBFF36F8F30
:10081000FFE70DE00698079901220023029302F0FA
:10082000D3FF029A069805AB114602F0CDFFFFE711
:10083000FFE705980AB080BD80B58CB00A90099199
:100840000892EFF305800B900B9820B1FFE76FF053
:10085000050007907AE09DF82B000006002804D5DB
:10086000FFE76FF0030007906FE09DF8240080071A
:10087000002803D5FFE70020059002E00A980590C4
:10088000FFE7002007900898029003F061F90490B8
:10089000FFE70599029B002006AA03F055FA019094
:1008A000019801283FD1FFE70A990798084007906F
:1008B00006990798084307909DF82400C00780B167
:1008C000FFE70A9907980840884201D1FFE73BE01B
:1008D000089820B9FFE76FF00200079034E0FFE7C7
:1008E0000EE00A980799084201D0FFE72CE008982B
:1008F00020B9FFE76FF00200079025E0FFE7FFE770
:1009000003F026F90499401A03900398029988424B
:1009100003D9FFE70020029004E003990298401AEF
:100920000290FFE70BE0089820B9FFE76FF00200A4
:10093000079003E06FF001000790FFE7FFE7FFE794
:1009400001980028A5D1FFE7FFE7FFE707980CB063
:1009500080BD000080B582B003F0D4F8019001980A
:1009600002B080BDB0B58EB00B900A910992002004
:100970000690EFF305800D900D98002840F09980C7
:10098000FFE70B98002800F09480FFE78020079095
:1009900018200590002008904FF0FF30049009982F
:1009A00000284DD0FFE70998006820B1FFE70998BB
:1009B00000680890FFE70998806920B1FFE709986F
:1009C00080690590FFE7059848B1FFE7059838284A
:1009D00005D8FFE709980079C00718B1FFE70020A4
:1009E0000C9069E00998406928B1FFE709984069CF
:1009F00080080790FFE70998806880B1FFE70998B1
:100A0000C0685C280BD3FFE70998006938B1FFE79D
:100A10000998406918B1FFE7012004900FE0099898
:100A2000806858B9FFE70998C06838B9FFE70998A6
:100A3000006918B9FFE700200490FFE7FFE702E034
:100A400000200490FFE70498012817D1FFE70B98D6
:100A50000899079A0A9BDDF814C0DDF824E0DEF857
:100A60000850DEF81040EE46CEF80850CEF80440AC
:100A7000CEF800C002F040FE069019E00498B0B92C
:100A8000FFE70B980899BDF81C200A9BDDF814C0FD
:100A9000EE4606ACCEF80440CEF800C002F0DCFD15
:100AA000012803D0FFE700200690FFE7FFE7FFE7FC
:100AB000FFE706980C90FFE70C980EB0B0BD000061
:100AC00080B586B0049004980390EFF305800590FC
:100AD000059820B1FFE76FF0050002901CE0039835
:100AE00020B9FFE76FF00300029014E00398FFF7CE
:100AF000C3F98DF807009DF80700042806D0FFE72A
:100B000000200290039801F013FC03E06FF0020054
:100B10000290FFE7FFE7FFE7029806B080BD000004
:100B200080B584B00390029148F2A070C2F2000038
:100B30000068009041F2A000C2F20000006804309A
:100B400001F0ECF808B9FFE700E0FFE70398013097
:100B500080B9FFE7029868B1FFE741F2A000C2F256
:100B600000000068011D48F27870C2F2000001F038
:100B70007BF93DE00098039908440190019841F207
:100B8000A001C2F2000109684860019800998842FA
:100B90000ED2FFE741F2B000C2F20000006841F25D
:100BA000A001C2F200010968043101F027F91EE03A
:100BB00041F2A800C2F20000006841F2A001C2F2B6
:100BC00000010968043101F019F9019848F2047133
:100BD000C2F200010968884207D2FFE7019848F293
:100BE0000471C2F20001086000E0FFE7FFE7FFE7E1
:100BF00004B080BD80B582B0019001F05DF947F688
:100C0000CC71C2F2000108680130086041F2A00016
:100C1000C2F20000006898B9FFE7019841F2A00114
:100C2000C2F20001086047F6CC70C2F20000006812
:100C3000012803D1FFE700F021FB00E0FFE71CE003
:100C400048F26C70C2F200000068A0B9FFE741F200
:100C5000A000C2F200000068C06A0199C96A884217
:100C600007D8FFE7019841F2A001C2F20001086035
:100C700000E0FFE700E0FFE7FFE747F6D870C2F2C9
:100C80000000016801310160006801994864019821
:100C9000C06A47F6DC71C2F200010968884208D9CF
:100CA000FFE70198C06A47F6DC71C2F200010860F4
:100CB000FFE70199C86A00EB800241F2B800C2F276
:100CC000000000EB8200043101F0CEF801F020F9C1
:100CD00048F26C70C2F200000068C8B1FFE741F250
:100CE000A000C2F200000068C06A0199C96A884287
:100CF0000CD2FFE74EF60451CEF200014FF08050C7
:100D00000860BFF34F8FBFF36F8F00E0FFE700E095
:100D1000FFE702B080BD000080B584B001F0CCF8E0
:100D200048F2A470C2F200000068002840D1FFE73A
:100D300048F2A460C2F20000029001F03FF848F2CD
:100D4000B860C2F20000039001F038F802990398ED
:100D500041F2A402C2F20002116041F2B401C2F2F7
:100D60000001086069460020086040F6AC72C2F2DB
:100D7000000241F24C03C2F200030A20102101F0EC
:100D80006DFE014648F2A470C2F2000001600068E6
:100D900060B1FFE748F2A470C2F20000006846F2BA
:100DA000B531C0F6010101F0A5F900E0FFE700E070
:100DB000FFE701F0ADF804B080BD000080B582B05F
:100DC000FFE747F6D070C2F20000006808B3FFE703
:100DD00001F072F848F28C70C2F20000C068C0687E
:100DE00001900198043000F099FF47F6CC71C2F2EF
:100DF000000108680138086047F6D071C2F20001AE
:100E000008680138086001F083F8019800F08CF858
:100E1000D7E702B080BD000080B582B0019000919C
:100E20000198006CB8B1FFE70199C8680A6C1044DA
:100E3000C86001988168C068884204D3FFE70199BF
:100E40000868C86000E0FFE70098019AD168126C5A
:100E5000EFF7A2FAFFE702B080BD000080B586B0D0
:100E6000059004910392002002900598806B0190F8
:100E70000598006C78B9FFE70598006848B9FFE766
:100E80000598806802F0CCFF0290059900208860E8
:100E900000E0FFE741E00398B8B9FFE7059A04993D
:100EA0005068126CEFF778FA059948680A6C10449C
:100EB0004860059948688968884204D3FFE7059926
:100EC0000868486000E0FFE726E0059A0499D068CA
:100ED000126CEFF761FA0599C8680A6C801AC8604D
:100EE00005980168C068884206D2FFE705998868BE
:100EF0000A6C801AC86000E0FFE70398022809D155
:100F0000FFE7019820B1FFE701980138019000E068
:100F1000FFE700E0FFE7FFE7FFE7019801300599F1
:100F20008863029806B080BD80B582B000900098BA
:100F300090F8590040B9FFE70098006B01F00EF8F7
:100F4000009801F00BF81CE0009890F85900012877
:100F500004D1FFE7009801F001F811E0009890F843
:100F6000590002280BD0FFE74FF0500080F31188A2
:100F7000BFF36F8FBFF34F8F0190FFE7FEE7FFE7EF
:100F8000FFE702B080BD000082B001900198406A86
:100F900038B1FFE70198006B0068C0F1380000909D
:100FA00002E000200090FFE7009802B070470000C8
:100FB00082B0019041F2A400C2F200000068006813
:100FC000B0FA80F04009019908600198006848B9BA
:100FD000FFE741F2A400C2F200000068C0680068A8
:100FE000009002E000200090FFE7009802B07047F8
:100FF00084B04FF4C040009041F6C070C2F20000CF
:1010000001909DF80400400788B1FFE70198073080
:101010000190019820F007000190019A41F6C071FB
:10102000C2F200010098891A08440090FFE7019875
:101030000290029948F27070C2F200000160002133
:1010400041600298009A104401900198083801907C
:10105000019820F007000190019A41F2AC00C2F221
:1010600000000260026851600268116002990391F9
:101070000199039A891A51600068039908600398DE
:10108000406848F20071C2F20001086003984068AD
:1010900048F2F861C2F20001086048F2CC61C2F285
:1010A00000014FF00040086004B0704780B582B086
:1010B0000190FFE7FFF782FE41F2B800C2F20000A4
:1010C000006802280CD3FFE74EF60451CEF200016F
:1010D0004FF080500860BFF34F8FBFF36F8F00E079
:1010E000FFE7E7E780B582B00190019868B1FFE7BC
:1010F000019800238360019803600198C360019800
:1011000019461A4601F090FD00E0FFE702B080BDED
:1011100080B584B0DDF818C00390029101928DF87B
:101120000330029818B9FFE70698006003E00198C1
:1011300006990860FFE703980699C8630298069924
:1011400008640698012101F011FD9DF8030006993D
:1011500081F84C0004B080BD80B588B0DDF834C0A3
:10116000DDF830C0DDF82CC0DDF828C00690059110
:10117000049203930C98006B04998900A522EFF761
:1011800082F90C98006B049900EB810004380290FE
:10119000029820F0070002909DF80800400758B11F
:1011A000FFE74FF0500080F31188BFF36F8FBFF35C
:1011B0004F8F0790FFE7FEE70598F8B1FFE70020A3
:1011C0000190FFE701980F2813D8FFE70598019ACF
:1011D000805C0C99114481F8340005980199405CB9
:1011E00008B9FFE705E0FFE7FFE70198013001904C
:1011F000E8E70C99002081F8430004E00C990020F6
:1012000081F83400FFE70A98382803D3FFE7372036
:101210000A9000E0FFE70A980C99C8620A980C99B6
:10122000C8640C990020009008650C98043000F008
:10123000DDFD0C98183000F0D9FD00980C9909617B
:101240000A99C1F138010C9A91610C9949620C9983
:1012500048650C9981F8580002980699039A00F0A5
:10126000E7FC0C9908600B9820B1FFE70C980B99EC
:10127000086000E0FFE708B080BD000080B584B0E2
:1012800000200390FFE70398372810D8FFE7039862
:1012900000EB800141F2B800C2F2000000EB8100D7
:1012A00000F08CFDFFE7039801300390EBE748F274
:1012B000D060C2F20000019000F080FD48F2E460CE
:1012C000C2F20000029000F079FD48F21870C2F2FC
:1012D000000000F073FD48F28C70C2F2000000F0D4
:1012E0006DFD48F27870C2F2000000F067FD0199D0
:1012F000029841F2A802C2F20002116041F2B0016C
:10130000C2F20001086004B080BD000083B002900A
:1013100048F27070C2F200000190FFE70198006887
:101320000299884205D2FFE7FFE701980068019023
:10133000F4E70198009000980199496808440299DF
:10134000884209D1FFE70298426801994868104431
:1013500048600198029000E0FFE702980090009832
:1013600002994968084401990968884220D1FFE739
:101370000198006841F2AC01C2F20001096888429C
:101380000DD0FFE701980068426802994868104450
:1013900048600198006800680299086007E041F21F
:1013A000AC00C2F20000006802990860FFE704E0A8
:1013B0000198006802990860FFE701980299884245
:1013C00004D0FFE702980199086000E0FFE703B04E
:1013D0007047000080B586B0059004910392029397
:1013E00000200190049805994860059800610498D0
:1013F0000399884216D8FFE703980299401A059985
:101400008969884203D3FFE70120019009E041F296
:10141000B400C2F2000000680599043100F0EEFC4F
:10142000FFE717E003980299884208D2FFE7049883
:101430000299884203D3FFE70120019009E041F2BD
:10144000A400C2F2000000680599043100F0D6FC47
:10145000FFE7FFE7019806B080BD000080B582B0CD
:10146000019000F029FD0198806B18B9FFE7012079
:10147000009002E000200090FFE700F049FD009896
:1014800002B080BD80B582B0019000F015FD0198DA
:10149000806B0199C96B884203D1FFE7012000905E
:1014A00002E000200090FFE700F032FD009802B05B
:1014B00080BD000008480068006880F308884FF08D
:1014C000000080F3148862B661B6BFF34F8FBFF39C
:1014D0006F8F00DF00BF00BF08ED00E080B586B071
:1014E0000490039141F2A400C2F200000068C068B9
:1014F000C06801900198043000F010FC019890F849
:1015000028004007002823D5FFE70198049B816944
:101510001944039AFFF75EFFC0B1FFE70198049AF0
:10152000694600230B60194602F0EEFE0290029815
:1015300058B9FFE74FF0500080F31188BFF36F8F69
:10154000BFF34F8F0590FFE7FEE700E0FFE707E0FE
:10155000019991F8280000F0FE0081F82800FFE7CB
:101560000198016A884706B080BD000080B58EB042
:10157000FFE748F2A470C2F20000006807A9002249
:1015800001F044FD002800F0B880FFE70798B0F1B3
:10159000FF3F17DCFFE707A804300290029858B914
:1015A000FFE74FF0500080F31188BFF36F8FBFF358
:1015B0004F8F0B90FFE7FEE702990A684868896839
:1015C000904700E0FFE70798002800F19580FFE7CB
:1015D000099806900698406928B1FFE706980430FC
:1015E00000F09CFB00E0FFE705A800F0FBF803908B
:1015F00007980190092800F27D800199DFE801F049
:101600000505053D456605053D45069991F8280007
:1016100040F0010081F828000698089B8169194470
:10162000039AFFF7D7FE30B3FFE70698016A8847B1
:10163000069890F82800400700281AD5FFE706987A
:10164000089982690A44694600230B60194602F032
:101650005BFE0490049858B9FFE74FF0500080F308
:101660001188BFF36F8FBFF34F8F0C90FFE7FEE73A
:1016700000E0FFE700E0FFE73DE0069991F8280071
:1016800000F0FE0081F8280035E0069991F8280066
:1016900040F0010081F828000898069988610698B2
:1016A000806958B9FFE74FF0500080F31188BFF30D
:1016B0006F8FBFF34F8F0D90FFE7FEE70698039BF8
:1016C000816919441A46FFF785FE14E0069890F8E0
:1016D00028008007002804D4FFE7069800F03EFCAD
:1016E00007E0069991F8280000F0FE0081F8280034
:1016F000FFE700E0FFE7FFE73BE70EB080BD00003B
:1017000080B584B00390029101F00AF8684600F0B9
:1017100069F801900098D8BBFFE7029860B9FFE72D
:1017200003980199884207D8FFE702F0DFFC03988D
:101730000199FFF7D3FE2AE0029858B1FFE741F282
:10174000B400C2F2000000680068B0FA80F04009FE
:101750000290FFE748F2A470C2F20000006803990B
:10176000019A891A029A00F0EFFC02F0BFFC60B9FE
:10177000FFE74EF60451CEF200014FF080500860B2
:10178000BFF34F8FBFF36F8F00E0FFE7FFE702E08B
:1017900002F0ACFCFFE704B080BD000081B041F274
:1017A000A800C2F200000068006840B9FFE748F2F4
:1017B0000471C2F200014FF0FF3008600FE041F207
:1017C000A800C2F200000068C068C06800900098DD
:1017D000406848F20471C2F200010860FFE701B0FE
:1017E0007047000080B582B0019002F0B1F900901E
:1017F000009841F29C01C2F200010968884206D2B9
:10180000FFE700F011F801990120086003E0019959
:1018100000200860FFE7009841F29C01C2F200013D
:101820000860009802B080BD80B588B0FFE741F243
:10183000A400C2F200000068006800284ED0FFE754
:1018400041F2A400C2F200000168C968096806916B
:101850000068C068C06803900398043000F05EFA26
:101860000398016A8847039890F8280040070028E9
:1018700032D5FFE7069803998969084405900598D1
:10188000069988420FD9FFE70598039948600398A5
:10189000006141F2A400C2F2000000680399043123
:1018A00000F0ACFA17E00398069A694600230B6033
:1018B000194602F029FD0290029858B9FFE74FF04F
:1018C000500080F31188BFF36F8FBFF34F8F0790E5
:1018D000FFE7FEE7FFE700E0FFE7A8E741F2A40229
:1018E000C2F200021068049041F2B401C2F2000199
:1018F000086810600498086008B080BD83B00020BC
:10190000009040F26C20C2F200000068013058B133
:10191000FFE74FF0500080F31188BFF36F8FBFF3E4
:101920004F8F0190FFE7FEE74FF0500080F31188E2
:10193000BFF36F8FBFF34F8F0290FFE7009808B996
:10194000FFE7FBE703B0704780B584B00390FFE783
:1019500001A8FFF72DFB029002980199FFF7D0FE36
:10196000FFF704FEF4E7000080B582B0019000F0BC
:10197000A3FA019890F845008DF80300FFE79DF960
:101980000300012816DBFFE70198406A58B1FFE722
:101990000198243002F042FB18B1FFE700F062FD2D
:1019A00000E0FFE700E005E09DF8030001388DF856
:1019B0000300E4E70199FF2081F8450000F0A8FA50
:1019C00000F07AFA019890F844008DF80200FFE7E1
:1019D0009DF90200012816DBFFE70198006980B13C
:1019E000FFE70198103002F019FB18B1FFE700F093
:1019F00039FD00E0FFE79DF8020001388DF8020094
:101A000000E000E0E4E70199FF2081F8440000F0E5
:101A10007FFA02B080BD000080B58AB00690002039
:101A2000029000F07DFE41F2AC00C2F200000068BE
:101A300018B9FFE7FFF7DCFA00E0FFE7069848F285
:101A4000CC61C2F200010968084240F0C580FFE79E
:101A5000069800B3FFE70698083006909DF8180036
:101A60004007B0B1FFE7069820F007000830069065
:101A70009DF81800400758B1FFE74FF0500080F381
:101A80001188BFF36F8FBFF34F8F0790FFE7FEE71B
:101A900000E0FFE700E0FFE70698002800F09A80EA
:101AA000FFE7069848F2F861C2F20001096888422F
:101AB00000F29080FFE748F27070C2F200000490DC
:101AC00000680590FFE705984168069A002091425A
:101AD000019007D2FFE705980068002818BF012091
:101AE0000190FFE70198C00730B1FFE70598049027
:101AF000059800680590E6E7059841F2AC01C2F24E
:101B000000010968884263D0FFE704980068083044
:101B10000290059800680499086005984068069945
:101B2000401A112821D3FFE705980699084403902D
:101B30009DF80C00400758B1FFE74FF0500080F3CC
:101B40001188BFF36F8FBFF34F8F0890FFE7FEE759
:101B5000059840680699401A0399486006980599C7
:101B600048600398FFF7D2FB00E0FFE70598426862
:101B700048F2F860C2F200000168891A016000684A
:101B800048F20071C2F20001096888420BD2FFE7F7
:101B900048F2F860C2F20000006848F20071C2F238
:101BA0000001086000E0FFE748F2CC60C2F20000EC
:101BB000026805994868104348600599002008604C
:101BC00048F20C71C2F2000108680130086000E0C0
:101BD000FFE700E0FFE700E0FFE702F087FA9DF88B
:101BE0000800400758B1FFE74FF0500080F311881C
:101BF000BFF36F8FBFF34F8F0990FFE7FEE70298A7
